:020000040800F2
:10400000A04D002045410008E9BD00084D82000890
:10401000F1A300089D520008A14001080000000023
:1040200000000000000000000000000041E6000861
:10403000D9550008000000005B4100081116010876
:104040005F4100085F4100085F4100085F410008D0
:104050005F4100085F4100085F4100085F410008C0
:104060005F41000885570008D55700085F410008E8
:10407000BD5500085F410008BF5500085F410008BA
:104080005F4100085F4100085F4100085F41000890
:104090005F4100085F4100085F4100086158000867
:1040A0005F4100085F4100085F4100085F41000870
:1040B000811601085F4100085F4100085F41000868
:1040C0005F4100085F4100085F4100085F41000850
:1040D0005F41000809360108113601081936010848
:1040E0005F4100085F4100085F4100085F41000830
:1040F0005F4100085F4100085F4100085F41000820
:104100005F4100085F4100085F4100085F4100080F
:104110005F4100085F4100085F4100085F410008FF
:104120005F4100085F4100085F4100085F410008EF
:10413000DFF80CD000F0B6FB0048004741620108F0
:10414000A04D00200648804706480047FEE7FEE7EE
:10415000FEE7FEE7FEE7FEE7FEE7FEE7FEE7FEE737
:10416000211601083141000840EA01039B0703D0F2
:1041700009E008C9121F08C0042AFAD203E011F8A6
:10418000013B00F8013B521EF9D27047D2B201E068
:1041900000F8012B491EFBD270470022F6E710B54C
:1041A00013460A4604461946FFF7F0FF204610BDA5
:1041B000421E12F8013F002BFBD111F8013B02F81F
:1041C000013B002BF9D1704730B505462A460B4616
:1041D00012F8010B13F8014B08B1A042F8D01CB142
:1041E000002802D06D1CF1E7284630BD10B504460A
:1041F00004E00B7800F8013B03B1491C521EF8D2D1
:10420000204610BD421C10F8011B0029FBD1801A6A
:10421000704710B5002200E0521C835C8C5CA34206
:1042200001D1002BF8D1D8B2E1B2401A10BD30B59F
:1042300004460020034600E05B1C934203D2E05C8E
:10424000CD5C401BF8D030BD034611F8012B00F8BF
:10425000012B002AF9D11846704730B505460020D9
:10426000034600E05B1C934205D2EC5CC85C201A5C
:1042700001D1002CF6D130BD2DE9F04791460F4613
:1042800080460446002614F8015B2DB100F05AFA6E
:104290000068405DC007F6D12B2D02D02D2D18D01F
:1042A000641E4A463946204600F050FA27B1396864
:1042B000A14201D1C7F8008071054FF002040BD56F
:1042C0004042002803DD10F0F1F80460A007BDE8CB
:1042D000F08746F48066E4E70028F8DA10F0E6F8A4
:1042E00004606FF00040F2E770B5064610F0DEF8AB
:1042F000046805460A2200213046FFF7BDFF2C6006
:1043000070BD70B5064610F0D1F8046805460A2263
:1043100000213046FFF7B0FF2C6070BD2DE9FE4F45
:10432000804681EA0300C00F0C46009021F0004156
:1043300023F00045B8EB0200A94105D240462146D2
:1043400090461C460B46024623F00040104347D0DF
:10435000270DC7F30A00C3F30A510290401A0190D7
:1043600040286BDAC3F3130040F4801B0098924698
:1043700020B10023D2EB030A63EB0B0B01985946E3
:10438000C0F14002504600F0ACF906460D465046DA
:104390005946019A00F0C4F910EB0800614100246D
:1043A00087EA115284EAE7731A4340D0009A62B355
:1043B000019A012A4FEA075215DC001B61EB02014A
:1043C0004FF0004202EA0752CDE90042001C41F5DD
:1043D000801132462B4600F017FA03B0BDE8F08F8B
:1043E00040462146F9E7001B61EB0201001C41F544
:1043F000801300185B412018A2F5001747EB03015A
:1044000040EAD570B6196D4111E06D084FEA3606E5
:1044100045EAC0754FEA0752001B61EB0201001C20
:1044200041F5801149084FEA3000001951413246E8
:104430002B4603B0BDE8F04F00F0D7B90098012239
:1044400040000023D0EB020263EBE07300982146AA
:104450004FEAE074B8EB000061EB0401E9E783F098
:1044600000435BE781F0004158E72DE9FE4F81EA08
:10447000030404F0004421F0004100944FF0000BCD
:1044800023F0004350EA01045ED052EA03045BD0FB
:10449000C3F30A54C1F30A552C44A4F2F334019433
:1044A000A0FB0254C1F3130141F48011C3F31303C1
:1044B00043F4801301FB024400FB034E840A970A75
:1044C00044EA815447EA8357A4FB076802958D0AA2
:1044D00005FB07854FEA932C04FB0C542705029D2E
:1044E0004FEA065847EA1637B5EB08056EEB070C9E
:1044F000870E920E47EA811742EA8312A7FB020158
:10450000B6EB0B0164EB00042B0D43EA0C335E1891
:1045100044EB1C50DA465146E7FB0201C5F3130495
:104520004FEA0B3343EA14534FEA0432019C43EA47
:104530000603A4F10C040294009CCDE900B400F041
:1045400063F903B0BDE8F08F00200146F9E72DE9DB
:10455000F04D81EA030404F0004B21F000451446BD
:104560004FF0000A23F0004150EA050220D054EA3F
:1045700001021DD0C5F30A570246C5F31303C1F368
:104580001300C1F30A5640F4801543F48013A7EBDF
:104590000608101BD64608F2FD3873EB050002D35F
:1045A00008F1010801E092185B41B8F1000F03DA4D
:1045B00000200146BDE8F08D00204FF48011064632
:1045C00084460EE0171B73EB050705D3121B63EB44
:1045D000050306434CEA010C49084FEA30009218E3
:1045E0005B4150EA0107EDD152EA030012D082EAA2
:1045F000040083EA0501084305D0101BAB4106D235
:104600000122002306E000224FF0004302E06FF099
:10461000010253101AEB06004CEB085110EB0A0094
:1046200041EB0B01BDE8F04D00F0DFB80EB5C10F56
:1046300080EAE0700844CA07002140F233438DE865
:104640000E000A460B4600F0DFF803B000BDC1F3D0
:104650000A5210B5C1F3130140F2FF3341F4801147
:104660009A4201DA002010BD40F233439A42A2F28E
:10467000334203DC524200F043F810BD904010BDBD
:104680002DE9F05F0546002092469B468846064687
:10469000814640241BE0284641464746224600F01A
:1046A0002FF853465A46C01A914110D31146184666
:1046B000224600F016F82D1A67EB01084F462246F5
:1046C0000120002100F00DF817EB00094E41201EDB
:1046D000A4F10104DFDC484631462A464346BDE8E2
:1046E000F09F202A04DB203A00FA02F100207047F4
:1046F0009140C2F1200320FA03F319439040704720
:10470000202A04DB203A21FA02F00021704721FA26
:1047100002F3D040C2F1200291400843194670478D
:10472000202A06DBCB17203A41FA02F043EAE07375
:1047300006E041FA02F3D040C2F120029140084362
:1047400019467047004870476C9001082DE9F05FEA
:1047500082460078002715468B460AF10104B946C7
:10476000302801D09DB113E014F8010B01277828FF
:1047700003D0582801D045B10AE00DB1102D07D162
:104780000027102514F8010B02E0082500E00A2597
:104790000026B0460EE005FB080005FB06F10127E8
:1047A00001EB10461FFA80F8B6F5803F00D3B946FA
:1047B00014F8010B294600F087F80028EBDABBF16A
:1047C000000F05D00FB1641E00E05446CBF8004046
:1047D000B9F1000F06D00FF069FE02210160C81E7A
:1047E000BDE8F09F48EA0640FAE710B5141E73F1E1
:1047F000000408DA401C41F1000192185B411A43A1
:1048000001D120F0010010BD2DE9F04D92469B46EC
:1048100011B1B1FA81F202E0B0FA80F22032904692
:10482000FFF75FFF04460F4640EA0A0041EA0B012A
:1048300053465A46084313D0114653EA010019D093
:10484000C8F140025046FFF75BFF05460E46504652
:1048500059464246FFF745FF084305D0012004E0D2
:1048600020463946BDE8F08D0020054346EAE07653
:104870002C4337430A986305E40AA0EB08000022A2
:10488000FD0A44EA47540A3002D500200146E9E710
:10489000010510196941DDE9084500196941BDE8C4
:1048A000F04DA2E7064C074D06E0E06840F001033A
:1048B00094E8070098471034AC42F6D3FFF73CFC6D
:1048C000CC9A0108EC9A01083A2800D2303820F03E
:1048D0002002412A01D3A2F13700884201D34FF0D0
:1048E000FF30704770B58C1810F8015B15F00703A6
:1048F00001D110F8013B2A1106D110F8012B03E079
:1049000010F8016B01F8016B5B1EF9D12B0705D480
:104910000023521E0DD401F8013BFAE710F8013BC9
:10492000CB1A921C03E013F8015B01F8015B521EE5
:10493000F9D5A142D8D3002070BD000000B587B0E2
:104940000121480209F0B0F901210C2009F0ACF96D
:104950000120ADF8040000208DF8070001A91248DD
:1049600001F0BCFD0120ADF8040000208DF8070027
:1049700001A90E4801F0B2FD002002908DF80C0054
:104980008DF80D004FF46020049000200590012068
:104990008DF8180002A9064800F024F80121044807
:1049A00000F008F807B000BD00080140000C01400D
:1049B0000024014021B1826842F00102826003E0DC
:1049C000826822F00102826070470146C86C80B2A2
:1049D00070470246002013680B400BB1012000E035
:1049E0000020704730B502460020002350680F4C6D
:1049F00020400D790C6844EA0524204350609068FB
:104A00000B4C2040D1E902542C434D7944EA450433
:104A100020439060D06A20F470000C7C641EE4B2E5
:104A2000234340EA0350D06230BD0000FFFEF0FF98
:104A3000FDF7F1FFF0B504460D4600200021092DD9
:104A400011DDE068A5F10A0606EB4607072606FA1F
:104A500007F18843A5F10A0606EB460603FA06F1BC
:104A60000843E0600CE0206905EB4507072606FADD
:104A700007F1884305EB450603FA06F10843206178
:104A8000072A0FDA606B561E06EB86071F2606FA0A
:104A900007F18843561E06EB860605FA06F1084321
:104AA000606322E00D2A0FDA206BD61F06EB860723
:104AB0001F2606FA07F18843D61F06EB860605FA7D
:104AC00006F10843206310E0E06AA2F10D0606EB50
:104AD00086071F2606FA07F18843A2F10D0606EBAA
:104AE000860605FA06F10843E062F0BD21B182684E
:104AF00042F4A002826003E0826822F4A002826095
:104B00007047F0B504460A4625460CE003F00F074F
:104B10001E11304600F04DF802F8010B384600F047
:104B200048F802F8010B15F8013B002BEED10020EC
:104B30001070F0BD2DE9F04707460C461546B84603
:104B400011E018F8016B06F00F0A4FEA26194846E3
:104B500000F02FF804F8010B504600F02AF804F892
:104B6000010B681EC5B2002DEBD100202070BDE8FE
:104B7000F0872DE9F04104460A4625464FF0040827
:104B800010E015F8013B03F00F061F11384600F046
:104B900010F802F8010B304600F00BF802F8010B98
:104BA000A8F10108B8F1000FEBD100201070BDE8AA
:104BB000F081002805DB092803DC00F13001C8B2D0
:104BC00008E00A2805DB0F2803DC00F15701C8B212
:104BD00000E0FF2070472DE9F84307468846384635
:104BE000FFF710FB0646304606EBD0714910A6EBE6
:104BF000410111B10020BDE8F883002546E017F817
:104C000015008DF800006800401C385C8DF801002C
:104C100000242DE01DF8040030280ADB1DF80400F4
:104C2000392806DC1DF804003038C0B20DF8040045
:104C30001CE01DF8040061280ADB1DF8040066284A
:104C400006DC1DF804005738C0B20DF804000DE072
:104C50001DF80400412809DB1DF80400462805DC86
:104C60001DF804003738C0B20DF80400601CC4B24F
:104C7000022CCFDB9DF80000F02101EA00109DF826
:104C80000110084308F80500681CC5B206EBD67190
:104C9000B5EB610FB3DB2846ADE700002DE9F0412D
:104CA00096B004465022D14902A8FFF75DFAD0A180
:104CB000204606F025FF90B9E07B2C2807D004F1B0
:104CC0000F00FFF711FB40B2CC4908708AE104F1F4
:104CD0001000FFF709FB40B2C849087082E1C8A183
:104CE000204606F00DFF28B9A01DFFF7FDFAC649C2
:104CF000086077E1C5A1204606F002FFB8B9607AE6
:104D0000312803D10120C449087002E00220C249C1
:104D10000870C24800780028D8D1BF480078012820
:104D2000D4D1BE490870BEA006F064FD5AE1BFA10F
:104D3000204606F0E5FEB8B9E07A312803D101201B
:104D4000B549087002E00220B3490870B348007802
:104D50000028BBD1B04800780128B7D1AF4908700E
:104D6000AFA006F047FD3DE1B3A1204606F0C8FE26
:104D700028B9617BE07A002212F006FF32E1B1A18E
:104D8000204606F0BDFE88BB012003469AA20D21F5
:104D90000090204601F007FA0546B0F1FF3F95D09C
:104DA0006019FFF7A1FAC6B201200346A8A20D219F
:104DB0000090204601F0F7F90546B0F1FF3F85D09D
:104DC0006019FFF791FA87B202200123A0A20D21FA
:104DD0000090204601F0E7F90546B0F1FF3F88D08A
:104DE00061193A46304612F02DFEFBE0FFE799A12B
:104DF000204606F085FE28B9E17A607A002212F09A
:104E0000C3FEEFE096A1204606F07AFE28B9A07A0C
:104E10000122002112F0B8FEE4E094A1204606F041
:104E20006FFE18B9204606F053F8DBE091A120464A
:104E300006F066FE002846D1A079202803D1E0794B
:104E40008DF8040002E0A0798DF804009DF804308C
:104E50008AA2502102A80FF001FB9DF8040030380F
:104E60000A2824D2DFE800F005230A0F14192323AF
:104E7000231E85A102A8FFF79BF91DE085A102A8CA
:104E8000FFF796F918E086A102A8FFF791F913E061
:104E900084A102A8FFF78CF90EE086A102A8FFF713
:104EA00087F909E085A102A8FFF782F904E084A14F
:104EB00002A8FFF77DF900BF00BF012202A9002070
:104EC0000CF04CF98EE080A1204606F019FE30B9B6
:104ED0000120804981F862020020087282E07EA1F0
:104EE000204606F00DFE70B97D4890F89C0003281E
:104EF00004D07B4890F89C00022873D10121204601
:104F000010F092FA6EE077A1204606F0F9FD70B934
:104F1000734890F89C00032804D0714890F89C00D6
:104F200002285FD10021204610F07EFA5AE06FA1DE
:104F3000204606F0E5FD38B9A01D01F043FA0A212C
:104F40006C4812F0F7FE4DE06BA1204606F0D8FD4C
:104F500010B910F0F3FB45E06AA1204606F0D0FD41
:104F600018B9601D02F02CFB3CE068A1204606F059
:104F7000C7FD00B367A1204606F0C2FDE0B9E01D01
:104F8000FFF7B2F940B265490870554890F8F6024B
:104F900091F90010884225D0514890F8F60200900F
:104FA0005E4890F900305EA2502102A80FF056FA38
:104FB00002A806F01FFC15E05DA1204606F0A0FD4A
:104FC00060B902AB03222C21204601F0C9F88046CB
:104FD000FFF78AF940B20949087003E056A120465C
:104FE00006F08EFD16B0BDE8F0810000E47E0108F9
:104FF0005E535953494E464F3A0000004403002087
:105000002B4353513A000000F80200202B504F432D
:105010005F5050503A000000E901002030030020AA
:1050200041542B43434C4B3F0D0A00002B504F4340
:105030003A6E706F6E672C002B544350535441549A
:1050400055533A002B544350524543563A00000002
:105050002C0000002B5443504F50454E3A000000A6
:105060002B544350434C4F53453A00002B43434C81
:105070004B3A00005E4D4F44453A00005B4D6F6473
:10508000652025635D0000004E6F207365727665B4
:105090007200000043444D41204D6F6465000000E4
:1050A00047534D0054442D5343444D412F455644DE
:1050B0004F0000005743444D410000004C54450050
:1050C000556E6B6E6F7700002B504F433A5354412F
:1050D000525400005C0800202B474749503A00001A
:1050E000DE1B00202B475049503A00002B464F54FE
:1050F000413A0000400100202B504F433A57414BAA
:10510000455550002B5544503A0000002B41554462
:10511000434800002B435445433A00004503002018
:1051200041542B435445433D25642C25640D0A000E
:105130002B434F50530000002B48454144534554E6
:105140003A0000002DE9F04707468846DFF8D8907E
:10515000B8F1000F33D1B86A00F58055334E002402
:1051600011E04FF480622946484612F0DBF94FF413
:1051700080623146484612F04BFA05F5806506F527
:105180008066601CC4B2042CEBDBBD6A4FF4FF16D2
:10519000002411E04FF480622946484612F0C2F91B
:1051A0004FF480623146484612F032FA05F58065C8
:1051B00006F58066601CC4B2042CEBDB32E01B4DAC
:1051C000B86A00F58056002411E04FF48062294649
:1051D000484612F0A7F94FF480623146484612F073
:1051E00017FA05F5806506F58066601CC4B2042CCC
:1051F000EBDB4FF4FF15BE6A002411E04FF4806230
:105200002946484612F08EF94FF4806231464846EE
:1052100012F0FEF905F5806506F58066601CC4B2E3
:10522000042CEBDBBDE8F0879C33002000F01F006E
:1052300070B502F0C5FA044602F096F90546294613
:1052400005A00FF0FBF8002C01DD084804600748BA
:10525000006800F027F870BD766F6C564241543DEF
:105260003D3D3D3D25640D0A00000000EC0100209D
:1052700008B50121092008F017FD4FF40070ADF8C2
:10528000000018208DF8030003208DF80200694605
:10529000014801F023F908BD000C014000BFFEE702
:1052A0007047000010B50446B4F59D7F18DC01225C
:1052B0001DA100200BF052FF21A006F09BFA012057
:1052C000234981F8310009F0BDF9012010F03AF9C5
:1052D0000CF020F84FF480701E49086000BFFEE714
:1052E000B4F5A27F1CDC1C4800783C280DD11BA122
:1052F000032005F055F8012003F060FF0020194954
:105300000880012218A10BF029FF13480078401CE7
:10531000C0B211490870B42805DD0020087002E011
:1053200000200D49087010BD56626174206C6F77C3
:105330002173687574646F776E206E6F772100003B
:105340004154244D59504F5745524F46460D0A007F
:105350009C1B0020140C0140F4010020C7EBB3E4B7
:10536000B5E70000B0000020436861726765206205
:10537000617421210000000000B585B00F4800785D
:1053800020B1012807D002280FD109E00CA16846FE
:105390000FF078F80BE00DA168460FF073F806E007
:1053A0000DA168460FF06EF801E005B000BD00BF2A
:1053B000684601F055F800BFF7E700001101002032
:1053C000455652435F48414C460000004556524303
:1053D0005F46554C4C000000414D524E422D31323B
:1053E0003200000010B5044624B1012C36D0022C46
:1053F00033D167E0012258A100200BF0AFFE5948DD
:105400000470002240F2255157480EF06DF9012238
:1054100040F2244154480EF067F90122802152489D
:105420000EF022F9012240214F480EF01DF9002212
:1054300040F225514D480EF057F9012240F2244127
:105440004A480EF051F90022802148480EF00CF92C
:105450000122402145480EF007F97AE0012244A1DB
:1054600000200BF07BFE3F480470012240F22551E2
:105470003D480EF039F9002240F224413A480EF03E
:1054800033F90022802138480EF0EEF80122402145
:1054900035480EF0E9F8012240F2255137480EF068
:1054A00023F9002240F2244134480EF01DF9002275
:1054B000802132480EF0D8F8002240212F480EF00B
:1054C000D3F846E001222EA100200BF047FE25482C
:1054D0000470012240F2255123480EF005F9002204
:1054E00040F2244120480EF0FFF8002280211E489F
:1054F0000EF0BAF8002240211B480EF0B5F800214A
:10550000234800F05DF800212148143000F058F8DD
:10551000012240F2255115480EF0E6F8002240F233
:10552000244112480EF0E0F8002280210F480EF0CE
:105530009BF8002240210D480EF096F800211448F7
:10554000283000F03DF8002111483C3000F038F8D8
:1055500000BF00BF10BD0000434F4D3C2D2D3E4D00
:10556000435521002C000020003801400044004039
:10557000434F4D3C2D2D3E475053210000480040E5
:10558000434F4D3C2D2D3E4D6F64656D2100000055
:105590004400024010B50648008838B1054806F0BE
:1055A000D9FF0020024908800349088010BD00008F
:1055B00030000020340400202E0000207047704787
:1055C00021B1026842F00102026004E002684FF675
:1055D000FE731A4002607047704710B54FF42F7386
:1055E000002109E0002201E000BF521C03F596549F
:1055F000A242F9D34C1CA1B28142F3DB10BD01469B
:105600001CE000BF00BF00BF00BF00BF00BF00BF65
:1056100000BF00BF00BF00BF00BF00BF00BF00BF92
:1056200000BF00BF00BF00BF00BF00BF00BF00BF82
:1056300000BF00BF00BF00BF00BF00BF0A1EA1F136
:10564000010399B2DDD1704770B586B002AC02AEED
:105650004A48C1884A4800EB810000680090102247
:105660002046009911F05EFF9DF80900012812D133
:1056700043481638808870B1414816388088401EEB
:105680003F49163988800846808820B90846007846
:1056900020F0010008703A481638408830B1384888
:1056A00016384088401E3649163948803448163826
:1056B0000078C0F3800060B1314816380078800867
:1056C000401E2F491639097860F382012C4816389C
:1056D00001702B481638D0F80600009988420FD088
:1056E00005AD049800F10C010422284611F090FF4A
:1056F00004AD059800F108010422284611F088FF46
:1057000000200190012201A8009911F081FF1C489E
:105710001638D0F806000099884228D01848163864
:10572000D0F806101022204611F0FCFE144816385E
:10573000D0F8060000F108010422684611F068FF65
:10574000049800F10C010422684611F061FF0098F2
:1057500000F10801042204A811F05AFF009800F19A
:105760000C0104220648103811F052FF04E00449ED
:1057700016390598C1F8060006B070BDC024002097
:10578000BE21002010B5082000F0D2F801280FD16A
:1057900008A00EF053FE0C480078012805D1000245
:1057A0000A49086001200A490870082000F0B4F88E
:1057B00010BD0000506F77657220646F776E2D2DDD
:1057C0002D2D0D0A0000000001030020100C0140E7
:1057D000DB02002010B5102000F0B6F8A0B11C4884
:1057E000006800F0100030B11A48007840F0010065
:1057F0001849087005E01748007820F001001549A5
:105800000870102000F08EF81248007810B10328BC
:1058100017D10AE010480078012802D10F4908701A
:1058200002E002200D4908700BE00B4800780128C7
:1058300003D102200949087002E0012007490870DD
:1058400000BF00BF034800780349087010BD000086
:10585000080C01404A0000204B00002048000020B6
:1058600010B5202000F070F8F0B12148006800F079
:10587000200030B11F48007840F002001D49087038
:1058800005E01C48007820F002001A49087020202A
:1058900000F048F81848007C30B918488078012892
:1058A00002D117A005F0A6FF1248007810B1032816
:1058B00017D10AE016480078012802D1154908706E
:1058C00002E00220134908700BE01148007801281B
:1058D00003D102200F49087002E001200D49087031
:1058E00000BF00BF034800780949087010BD0000E0
:1058F000080C01404A0000205C080020DE1B00204C
:1059000041542B504F433D3345303030300D0A0069
:105910004B0000204800002001490860704700004B
:10592000140401400149086070470000140401405C
:1059300001460020034A12680A400AB1012000E033
:105940000020704714040140014600200022074B4C
:105950001B6803EA0102054B14331B680B4013B1AB
:105960000AB1012000E0002070470000000401405F
:10597000002123498279002A3AD00A461268036836
:105980009A430B461A600A1D126803689A430B1D5E
:105990001A60027911440A6803681A430A60184AB7
:1059A0000832126803689A43154B08331A601A1DAF
:1059B000126803689A43124B0C331A604279102A1A
:1059C0000ED11A1F126803681A430D4B08331A6070
:1059D0001A1D126803681A43094B0C331A600DE054
:1059E0000749427911440A6803681A430A6005E0CE
:1059F000027911440A6803689A430A6070470000FC
:105A0000000401400EB504208DF80B0003208DF832
:105A10000A003020ADF8080002A90D4800F05EFD34
:105A20000421012000F03AFD0521012000F036FD9F
:105A30003020009000208DF8040010208DF8050023
:105A400001208DF806006846FFF792FF0EBD0000AA
:105A5000000C014000B589B057480078002874D088
:105A6000012802D0022871D149E0012003F0A6FBF1
:105A70000020524908800320514908745148807819
:105A800010B1012839D10BE001200BF039FC4EA0F8
:105A900005F0B0FE012251A100200BF05FFB2CE0CD
:105AA0004748808938B900204549C8814DA1012067
:105AB00004F076FC0EE04248C38952A21E2101A8E0
:105AC0000EF0CCFC012201A900200BF047FB01A83D
:105AD00005F090FE3A48C089401C3949C881084603
:105AE000C0898989884202DB00203549C8810122AA
:105AF0004AA100200BF032FB00BF00BF56E001209E
:105B000003F05CFB00202D49088003202C49087419
:105B10002C48807810B1012844D10BE001200BF013
:105B2000EFFB41A005F066FE012244A100200BF02E
:105B300015FB37E02248808948B900202049C881F8
:105B400028A1012004F02CFC10E02DE02DE01C48E1
:105B5000C3892CA21E2101A80EF080FC012201A9FC
:105B600000200BF0FBFA01A805F044FE1448C089A0
:105B7000002805DD1248C089401E1149C8810BE08C
:105B80000F48808918B900200D49C88104E00C48ED
:105B90008089401E0A49C88101222AA100200BF0F9
:105BA000DDFA00BF00BF01E000E000BF00BF002041
:105BB0000149087009B000BD48000020B000002075
:105BC0005C080020DE1B002041542B504F433D3128
:105BD000303030303030370D0A0000005B472B2B5F
:105BE0005D0000003243434544454336453443425B
:105BF00046434233433944344231443444414346BA
:105C00004446000041542B504F433D31303030303A
:105C1000303231253034780D0A0000005B55736551
:105C2000722B2B5D0000000041542B504F433D313F
:105C3000303030303030380D0A0000005B472D2DF9
:105C40005D0000005B557365722D5D00F0B5024686
:105C500018A419A50223002011E0C61700EB9676C0
:105C6000B610A0EB8606965D275C7E400146C717FE
:105C700000EB9777BF10A0EB8707D655401C9842E2
:105C8000EBDB0523002011E0C61700EB9676B6107B
:105C9000A0EB8606965D2F5C7E400146C71700EBA1
:105CA0009777BF10A0EB8707D655401C9842EBDBD7
:105CB000F0BD00005A5400005A5432363000000043
:105CC00010B50C24002012490870012011490870F9
:105CD0000BF02CFB0A214FF47A7008F003FE0A2126
:105CE0004FF4FA7008F0FEFD0A214FF47A7008F0C4
:105CF000F9FD01200DF0E4FD012003F0EBFC08208C
:105D000009F0C8FB012204A100200BF027FA10BD06
:105D1000FE020020F00200205B456E74657254782C
:105D20004D6F64655D00000030B5024600200FE055
:105D3000135C841C145D1454841C1355441C135DA3
:105D4000C41C155D441C1555C41C1355041DA0B27C
:105D50008842EDDB30BD000030B5044604254FF429
:105D6000302000F06FF80546042D17D10C4800696B
:105D700040F002000A49086108464461006940F0A9
:105D8000400008614FF4302000F05CF805460448FC
:105D9000006941F6FD71084001490861284630BD9F
:105DA0000020024004200B49C96801F0010109B13B
:105DB00001200EE00749C96801F0040109B1022081
:105DC00007E00449C96801F0100109B1032000E0AF
:105DD00004207047002002400348006940F0800022
:105DE00001490861704700000020024070B5044678
:105DF0000D460426F00200F025F80646042E11D1C7
:105E00000948006940F00100074908612580F00257
:105E100000F018F806460448006941F6FE71084093
:105E200001490861304670BD002002400248034924
:105E300048600348486070472301674500200240DE
:105E4000AB89EFCD00B502460423FFF7ABFF034655
:105E500003E0FFF7A7FF0346521E012B01D1002AE2
:105E6000F7D102B90523184600BD10B500F002F8BD
:105E700010BD00002DE9F0418CB04FF000084FF448
:105E80000A617A48FEF789F90024002642E03022B0
:105E90003146684611F046FB75490B98884232D16D
:105EA00004EB440101EBC4027049083101EB8200AC
:105EB00014226946FEF758F904EB440101EBC402D1
:105EC0006A49083101EB820101F11400102205A991
:105ED000FEF74AF904EB440000EBC40263480830C3
:105EE00000EB82000999416204EB440000EBC4011D
:105EF0005E48083000EB81008662641C0A9808B195
:105F00000A9E07E009E05B490B98884200D104E053
:105F100006F5805658488642B9DB00BF53484460B6
:105F2000012C06DA55A00EF089FA01200CB0BDE86C
:105F3000F08156484D49086004254968491E01EB27
:105F4000410202EBC1024949083101EB820050A134
:105F5000FEF75FF970B945494968491E01EB4102F6
:105F600002EBC1024149083101EB8201886A0FF05E
:105F700013FE054604274FF4FF100FF00DFE0746F1
:105F80002DB943A144A00EF059FA0020CEE7002F0E
:105F900064D1042D05D13EA141A00EF04FFA002698
:105FA00004E03BA143A00EF049FA012630224FF451
:105FB000FF11684611F0B6FA04EB440101EBC4028C
:105FC0002A49083101EB820014226946FEF7CCF819
:105FD00004EB440101EBC4022449083101EB8201C6
:105FE00001F11400102205A9FEF7BEF804EB4400ED
:105FF00000EBC4021D48083000EB820009994162A1
:10600000601E801B00EB400202EBC0021748083004
:1060100000EB8200816A3022684611F083FA04EBBB
:10602000440000EBC4021148083000EB82000A99DA
:106030008162A11B01EB410202EBC1020B49083155
:1060400001EB82000121FFF77DF8042D04D1074800
:106050004068401C05494860002067E73B462A46E7
:106060000BA11AA00EF0EAF902205FE7FC2A00203B
:10607000311B200812EFCDABFFDF1F004E6F2072E7
:1060800065732066696C65730D0A0000F8DEBC8AD2
:106090007379732E696E69002573206F6B0D0A008A
:1060A0002573206C6F73742C207265636F76657234
:1060B0000D0A0000257320696E76616C69642C20DE
:1060C0007265636F7665720D0A00000025732065A6
:1060D00072726F722C207374617475733A25642C1C
:1060E00025640D0A000000002DE9F04F0146C1F3C0
:1060F000074CC1F3072801F0FF09DFF85CA000207E
:10610000002224E09300DFF854B01BF8035003F1A1
:10611000010E1BF80E6003F1020E1BF80E40A9EBF6
:106120000505002D00DA6D42A8EB0606002E00DA08
:106130007642ACEB0404002C00DA644205EB060B5B
:106140000BEB0407574501DABA461046521CFF2AEA
:10615000D8DDBDE8F08F00003F420F00FC26002094
:106160002DE9F04705460E46174698464FF00009C0
:10617000C246002410E0285DB04203D109F10100BD
:1061800000F0FF09B94505D1601C05EB000A504637
:10619000BDE8F087601CC4B22846FEF733F8A04281
:1061A000E9D800BFF4E72DE9F04704460E4617464C
:1061B0001D46DDF820A04FF00008C14615E02A4634
:1061C00039462046FEF733F850B909F1010000F0D6
:1061D000FF09D14504D108EB050000B2BDE8F08706
:1061E000641C08F101001FFA80F82078B042E6D163
:1061F0004FF0FF30F2E7000010B502F071F92A48C5
:10620000007800B110BD2948007818B128480078FE
:10621000002800DDF6E727484078F0B125480078EF
:10622000A8B925480078C0EB0010840021484089B7
:10623000401C80B21F494881A0421EDD00204881D9
:1062400001221EA10AF08AFF08F04EF815E0002096
:1062500018494881204908700FE016484089401CC1
:1062600080B214494881B0F5616F06DD0020488195
:106270001AA00EF0E3F808F037F80E4880790128EC
:1062800010D10C48007A401CC0B20A490872282874
:1062900008DD01200872012218A100200AF05EFF2B
:1062A00008F022F800BFADE7F0020020FE02002057
:1062B000350100205C080020D8020020506F634C9C
:1062C0006F737454696D656F75742152657365746D
:1062D000204D6F64656D2100F402002054696D65E6
:1062E0006F757420204C6F67696E74696D656F758A
:1062F000742D2D2D2D0D0A20000000004D6F6465BA
:106300006D5265637654696D656F7574215265735E
:106310006574204D6F64656D21000000F0B585B097
:1063200054239F222C21002001F0B0FC01204223A5
:106330008022322100901D2001F01DFD0025204803
:10634000D0F8067001AE00242CE010223946304609
:1063500011F0E8F89DF80400012807D100208DF81D
:10636000040001223946304611F052F9049F0A20F8
:1063700094FBF0F100FB114008B902F0B1F80A20DB
:1063800094FBF0F100FB114050B9012005F11D0212
:10639000034640210090342001F019FD681CC5B26D
:1063A000601C84B2B4F57A7FCFDB002004494880BA
:1063B00088800846007820F00100087005B0F0BD24
:1063C000A821002010B504462078302821D031289B
:1063D00002D0322828D10EE02046FDF713FF022814
:1063E00005D9A01CFDF780FF1049086002E010A04D
:1063F00000F036F818E011A000F032F80120124940
:1064000081F86202114908709621114811F092FC3E
:106410000AE010A000F024F801200C490870962131
:106420000B4811F087FC00BF00BF10BD38010020F1
:10643000D5FDD4DAC9FDBCB62E2E2E00D5FDD4DA9A
:10644000D6D8C6F42E2E2E005C0800203C01002079
:1064500040010020CAA7B0DCCDCBB3F6000000009D
:10646000F8B505460122294600200AF077FE2846A5
:10647000FDF7C8FE8021A1EBC0004608402421465C
:1064800010238022002001F0BDFB00202146009057
:10649000B0B201232A4601F091FEF8BD30B50022CA
:1064A0008B071C0F0F2303FA04F20B4B8C1053F8CD
:1064B00024309343084C8D1044F8253023468C102B
:1064C00053F824308C07240F00FA04F42343024CC1
:1064D0008D1044F8253030BD080001402DE9F04111
:1064E000024600250026002000230024002791F802
:1064F00003C00CF00F0591F803C00CF0100CBCF1B8
:10650000000F03D091F802C04CEA050591F800C0D5
:10651000BCF1000F31D0146800202BE04FF0010CCB
:106520000CFA00F3B1F800C00CEA03069E4220D139
:1065300083004FF00F0C0CFA03F7BC4305FA03FC81
:106540004CEA040491F803C0BCF1280F06D14FF0C7
:10655000010C0CFA00FCC2F814C00AE091F803C068
:10656000BCF1480F05D14FF0010C0CFA00FCC2F849
:1065700010C0401C0828D1D31460B1F800C0BCF191
:10658000FF0F34DD546800202EE000F1080C4FF0BE
:10659000010808FA0CF3B1F800C00CEA03069E42A9
:1065A00021D183004FF00F0C0CFA03F7BC4305FA1E
:1065B00003FC4CEA040491F803C0BCF1280F05D198
:1065C00000F1080C08FA0CF8C2F8148091F803C026
:1065D000BCF1480F07D100F1080C4FF0010808FA90
:1065E0000CF8C2F81080401C0828CED35460BDE8D7
:1065F000F0810000F0B50A460023002400210025A8
:1066000000F00046B6F1004F02D11D4EF16901E0E5
:106610001B4E7168C0F3034583B200F44016B6F513
:10662000401F08D121F07061154E766826F0706623
:10663000134F7E6012E000F48016B6F5801F06D17D
:10664000032606FA05F4A14341F0706106E0460D09
:10665000360103FA06F6B14341F0706122B1460DEE
:10666000360103FA06F6314300F00046B6F1004F5A
:1066700002D1034EF16101E0014E7160F0BD0000F6
:10668000000001400246002093680B400BB101203E
:1066900000E00020704741617047016170470000D1
:1066A0000120014908707047D001002010B515483D
:1066B0000078022800D110BD13480068B0F5802F83
:1066C00017D11048007840B90020104908700D48D3
:1066D0000078401C0B49087012E00C480078032831
:1066E0000EDBFFF7EDFA07480078401C05490870FB
:1066F00006E004480078012802D100200149087012
:1067000000BFD8E7F502002040000020470000202D
:106710002DE9F04395B00446607931287ED1A07907
:1067200044287BD16A48007818B9012015B0BDE82B
:10673000F08304F11D00FDF765FD801EC6B2482EF2
:1067400000DB4826324604F11D0102A8FDF70CFDCE
:10675000002002A988556077102201A904F11900D0
:10676000FDF78AFD1FFA80F800206076102201A94B
:1067700004F11100FDF780FD0746564991F86612B5
:1067800001EB410202EBC102534941F8227051482A
:1067900090F8660200EB400101EBC0014E4800EBAF
:1067A0008100A0F804809DF80800C0B92021494864
:1067B00090F8660200EB400202EBC002464800EB94
:1067C000820081710021434890F8660200EB40028C
:1067D00002EBC002404800EB8200C1710DE03D4871
:1067E00090F8660200EB400202EBC0023A4800EB70
:1067F0008200811D02A80AF0D9FD364890F8660291
:10680000401C344981F86602084690F8660291F807
:106810006512884205D101202E4900E003E081F88D
:106820006E02012082E72DA1204605F069F90028BB
:106830004BD104222C21204601F06CFE0546601944
:10684000FDF752FD234991F8661201EB410202EB7C
:10685000C102214941F8220005222C21204601F0E5
:1068600059FE05466019FDF7CDFC801E1FFA80F920
:1068700060194946FFF758FA6019FDF7C3FC801EFE
:106880001FFA80F96219134991F8661201EB41036E
:1068900003EBC103104901EB8301881D49460AF04F
:1068A0000AFE0C4890F86602401C0A4981F866020C
:1068B000084690F8660291F86512884203D10120DB
:1068C000044981F86E02012030E700202EE7000025
:1068D000530200205C080020D80900202B504F43B1
:1068E0003A67726F7570732C000000002DE9F0415B
:1068F00094B004466079312870D1A07945286DD1D3
:106900006848007818B9012014B0BDE8F08104F19E
:106910001900FDF777FC801EC6B2482E00DB482622
:10692000324604F1190101A8FDF71EFC002001A95F
:10693000885560761022694604F11100FDF79CFC31
:106940000746594991F8661201EB410202EBC10278
:106950005549A03141F822709DF80400D0B920219A
:10696000514890F8660200EB400202EBC0024E482C
:10697000A03000EB8200417100214B4890F8660284
:1069800000EB400202EBC0024748A03000EB82005F
:1069900081710EE0444890F8660200EB400202EB81
:1069A000C0024148A03000EB8200411D01A80AF05E
:1069B000FDFC3D4890F86602401C3B4981F86602A8
:1069C000084690F8660291F86512884203D10120CA
:1069D000354981F86E02012096E7FFE733A1204692
:1069E00005F08EF800285AD103222C21204601F010
:1069F00091FD05466019FDF777FC032801D00120C1
:106A000082E704222C21204601F084FD054660190E
:106A1000FDF76AFC244991F8661201EB410202EB92
:106A2000C1022149A03141F8220005222C21204633
:106A300001F070FD05466019FDF7E4FB801E1FFAAA
:106A400080F860194146FFF76FF96019FDF7DAFB2E
:106A5000801E1FFA80F86219134991F8661201EB43
:106A6000410303EBC1031049A03101EB8301481D31
:106A700041460AF020FD0C4890F86602401C0A4985
:106A800081F86602084690F8660291F8651288421D
:106A900003D10120044981F86E02012034E700206F
:106AA00032E70000530200205C0800202B504F43C7
:106AB0003A6D656D626572732C0000002DE9F14F2F
:106AC000A2B0002017909A488069000E8DF81C0033
:106AD00097488069000C8DF81D009548008B000ACE
:106AE0008DF81E009248007E8DF81F009048406986
:106AF000000E8DF818008E484069000C8DF81900C2
:106B00008B48808A000A8DF81A008948007D8DF82C
:106B10001B0018A906A8FEF72CF8002016900024E8
:106B200004E018A8005D16A90855641C032CF8DBC6
:106B300016A8FDF7D9FB824600201390149000247C
:106B400005E018A9E01C085C13A90855641C062C74
:106B5000F7DB13A8FDF7C8FB83464FF47A709BFB65
:106B6000F0F00590FDF762FDCDE90E010022714BBA
:106B7000DDE90E01FDF7EBFCCDE90E014FF47A7073
:106B80009BFBF0F100FB11B0C0EB00108000059002
:106B9000FDF74CFDCDE90C010022674BDDE90C014E
:106BA000FDF7D5FCCDE90C01DDE90C23DDE90E0193
:106BB000FDF7B4FB05460E460022604B28463146E1
:106BC000FDF753FCCDE902015D490AFB01F0FDF739
:106BD0002DFDCDE90001DDE90223FDF79FFBCDE9A5
:106BE0000401FDF734FD5249486617A907A8FDF7CF
:106BF000C0FF002404E017A8005D15A90855641C17
:106C0000032CF8DB15A8FDF76FFB8146002405E097
:106C100017A9E01C085C11A90855641C062CF7DBB9
:106C200011A8FDF761FB10904FF47A71109890FB5A
:106C3000F1F00590FDF7FAFCCDE90A0100223D4B89
:106C4000DDE90A01FDF783FCCDE90A014FF47A7111
:106C5000109890FBF1F201FB1200C0EB00108000D5
:106C60000590FDF7E3FCCDE908010022324BDDE998
:106C70000801FDF76CFCCDE90801DDE90823DDE939
:106C80000A01FDF74BFB0746884600222B4B38468E
:106C90004146FDF7EAFBCDE90201294909FB01F074
:106CA000FDF7C4FCCDE90001DDE90223FDF736FB69
:106CB000CDE90401FDF7CBFC1D4988662298002828
:106CC00033D100221F4B38464146FDF7CEFBCDE9BC
:106CD0000201FDF7BCFC05901BA31CA21E21CDE9FF
:106CE00000901AA80DF0BAFB002001231AAA1B215C
:106CF000009001F063FA0022124B28463146FDF75E
:106D0000B4FBCDE90201FDF7A2FC059014A315A286
:106D10001E21CDE900A01AA80DF0A0FB0020012340
:106D20001AAA2B21009001F049FA23B0BDE8F08F98
:106D3000281F002000004E4040774B4180842E41A8
:106D400040420F00006AF8405300000020CEB3B666
:106D5000C82025733A20252E33642E253035640053
:106D60005700000020BEADB6C82025733A20256428
:106D70002E2530356400000070B5054600240DE076
:106D800004EB440101EBC402084901EB82002946EF
:106D9000FDF73FFA08B9204670BD641C0348083867
:106DA0004068A042ECD84FF0FF30F5E7042B0020FC
:106DB0000246002A01DA0020704702EB420000EB95
:106DC000C203064800EB8300416A002902DB044845
:106DD000814201DD0020EFE70846EDE7042B0020AB
:106DE000FFCF1F002DE9F04704460D4691469A4615
:106DF000A02C01DBA02D02DA0020BDE8F087A4F171
:106E0000A000C6B2A5F1A000C7B2BAF1000F10D120
:106E1000781E711E5E2202FB010000EB40004FEA6B
:106E2000C0080B494B4618224868414607F048F90C
:106E3000E3E7781E711E5E2202FB01004FEA401854
:106E400004494B4620224868414607F039F9D4E707
:106E5000F0260020E426002010B543480078401CAE
:106E6000C0B241490870022801DD002008703E4888
:106E7000007820B902F092F93C49086003E002F082
:106E80008DF93B49086039480068394909688842EA
:106E900001D0002010BD3748006834490968884295
:106EA00014D0324800683349086008460068B0F5DD
:106EB000C42F08D00120304908702E4801682FA047
:106EC0000DF0BCFA02E000202B4908702A48007837
:106ED00000283BD02C480078C8B12C4800782649BF
:106EE0000978884211D02448007828490870214840
:106EF00000682749086008460068B0F5083F02D1DD
:106F00000120244908700120C4E70020C2E71A4884
:106F100000781E4908702048007880B9134800683E
:106F20001B49086008460068B0F5083F02D10120FF
:106F3000184908706420184908700120AAE716480B
:106F40000078401E144908700020A3E70020124971
:106F500008700E48007820B100200C490870401ECF
:106F600098E7002096E700004D0000205400002024
:106F700058000020500000204E0000204B45593D95
:106F8000256C780D0A000000450000204F0000200D
:106F900040000020490000204C00002010B554485B
:106FA0000078401CC0B252490870022801DD002060
:106FB00008704F48007820B900F0BEF84D490860CD
:106FC00003E000F0B9F84C4908604A4800684A49B3
:106FD0000968884201D0002010BD48480068454932
:106FE0000968884213D0434800684449086008464D
:106FF0000068BE2808D20120414908703F48016856
:1070000040A00DF01BFA02E000203D4908703C480A
:10701000007800285FD04048007858B33F48007897
:1070200037490978884223D0354800783B490870B1
:107030003248006818B93A483A49086016E02F48C3
:1070400000684B2803D23848364908600EE02B48C8
:107050000068642803D235483249086006E02748B2
:107060000068BE2802D232482E4908600120B3E7EA
:107070000020B1E722480078284908702D480078A0
:1070800010BB1E48006818B925482649086016E05C
:107090001A4800684B2803D22348224908600EE0B2
:1070A00016480068642803D220481E49086006E09C
:1070B00012480068BE2802D21D481A4908606420A0
:1070C0001C490870012087E71A480078401E1949BA
:1070D0000870002080E70020164908700F480078EB
:1070E00020B100200D490870401E75E7002073E7AD
:1070F0005D00002064000020680000206000002087
:107100005E0000204B45593D25642E2B2B2B2B2B4D
:107110002B2B2B2B0D0A0000450000205F000020C8
:107120002A04EC00400000202A04AC002A00FC00E5
:107130002A04BC005C00002070B500230122114627
:107140001348FDF777FC01211148FDF7CFFC00BF84
:1071500002210F48FDF73DFC0028F9D00C48FDF74F
:1071600034FC0446642C08DAB4F5805F05DB09A022
:107170000DF064F94FF0FF3070BD4FF4967104FBD1
:1071800001F0C11700EB11510D132846F4E7000080
:107190000028014056444143204F5645520000000C
:1071A0002DE9F74F90B00546BB484088052802DB23
:1071B0004FF0050902E0B84890F802904FF0000B3C
:1071C000002009904FF47A780DF1280A11980128CF
:1071D00012D1B148D0F80600AF49C1F812000846F4
:1071E000D0F806101022504610F09CF9AA490C98CD
:1071F000C1F80E00002011900024129864287CD160
:1072000076E0A548D0F8127010223946504610F0AA
:1072100089F9082207F110010EA810F083F99DF8F2
:10722000280001284DD1BBF1000F07D10BF101005F
:1072300000F0FF0B98490C98C1F80E00DDF82A0009
:10724000C0F344400090DDF82A10C1F383534FF09F
:107250003F0C0CEA916204EBC40C05F1DE0101EB7A
:107260004C008EA10DF00EF904EBC40205F1DE0115
:1072700001EB42000EA9FCF79BFF9DF829000128B5
:1072800008D1002104EBC40205F1DE0000EB42004E
:10729000417407E0012104EBC40205F1DE0000EBBC
:1072A000420041747C490D98C1F8120001F11600AA
:1072B00000EB84000760601CC4B24C4508DB264626
:1072C00017E07548D0F806007349C1F812000FE0C6
:1072D000A8F101001FFA80F8B8F1000F07D10122D0
:1072E00072A1002009F03AFF264602E005E000BF47
:1072F00087E700BF0020E880BEE072E06648D0F873
:107300000E7010223946504610F00CF9082207F191
:1073100010010EA810F006F99DF8280001284CD1A4
:10732000099838B90998401CC0B209905A490D987B
:10733000C1F81200DDF82A00C0F344400090DDF8E7
:107340002A10C1F383534FF03F0C0CEA916204EB17
:10735000C40C05F1DE0101EB4C0057A10DF092F8D1
:1073600004EBC40205F1DE0101EB42000EA9FCF7BB
:107370001FFF9DF82900012808D1002104EBC40259
:1073800005F1DE0000EB4200417407E0012104EB4F
:10739000C40205F1DE0000EB420041743E490C9846
:1073A000C1F80E0001F1160000EB84000760601CBC
:1073B000C4B24C4506DB264614E037490C98C1F8A8
:1073C0000E000EE0A8F101001FFA80F8B8F1000FDE
:1073D00006D101223BA1002009F0C0FE264601E0B3
:1073E00000BF8BE700BF0DF1100A304606EBD071ED
:1073F000C1F347010391002438E004EBC40105F117
:10740000DE0000EB41000290701E001B00EBC0018B
:1074100005F1DE0000EB4100019012225046029976
:10742000FCF7A2FE1222DDE90110FCF79DFE1222FC
:1074300051460198FCF798FE1748163000EB84007F
:107440000768701E011B1448163000EB81000168AC
:107450001148163000EB84000160701E011B0E48BD
:10746000163000EB81000760601CC4B203988442B0
:10747000C3DBA9F10100E880AE80002085F83E0161
:10748000B5F83A11B5F83C0102F092FA284602F03C
:107490009FFD13B0BDE8F08FA82100202530326495
:1074A0002F253032642F2530326420005B534D533A
:1074B0005D6572723100000025642F25642F2564FC
:1074C000200000005B534D535D6572723200000076
:1074D0002DE9F04F87B082460E4617464FF000095F
:1074E0000024A3469AF8000008B1307818B90020AB
:1074F00007B0BDE8F08F0FE058460BF1010B01A972
:1075000001F80080B8F13D0F02D0B8F13B0F01D176
:107510000020EDE7761C641C96F80080B8F1000F9F
:1075200001D0142CE8DB3D222046641C01A90A543A
:10753000002008555046FCF747FE0546254405E067
:10754000287838706D1C7F1C09F1010928782028E3
:1075500005DD28783B2802D0B9F1500FF0DD00207E
:1075600038704846C4E7000070B5002301220821A6
:107570000F48FDF75FFA01210D48FDF7B7FA00BF8C
:1075800002210B48FDF725FA0028F9D00848FDF73D
:107590001CFA0446642C08DAB4F5805F05DB05A00C
:1075A0000CF04CFF4FF0FF3070BD25462846FBE73E
:1075B0000024014056444143204F564552000000EC
:1075C0002DE9F0410546022737E0E85D2C2832D14D
:1075D000A81CFCF789FE0646E919481CFCF784FE46
:1075E0000446052E06D1192C04D11C4890F82F030F
:1075F00000B129E0052E07D1372C05D1174890F8A6
:107600002F03012800D01FE0052E07D1052C05D13E
:10761000124890F82F03022800D015E0192C0AD048
:10762000372C08D0052C06D00526052402200B494E
:1076300081F82F0308E0781C07B22846FCF7E2FD2A
:10764000B842C2D8BDE8F081044991F82F0304F094
:1076500029FA002004F068FA00BFF3E7DE1B0020DF
:107660000021064A00BF05E013780370401C521C3D
:107670004B1CD9B20C29F7DB70470000E8F7FF1F5D
:10768000024602B97047002008E0131823B1054BE9
:1076900053F821301B5C1354431CD8B20C28F4DB84
:1076A00000BFEFE7780200200346002227E04D29C3
:1076B00003D102F10C0082B221E0412905DB5A29F5
:1076C00003DC02F1080082B219E0612905DB7A29A6
:1076D00003DC02F1080082B211E0302905DB392910
:1076E00003DC02F1080082B209E0202905DB6029F1
:1076F00003DC02F1080082B201E0901D82B213F8AF
:10770000011B0029D3D1D0B270470000F0B589B079
:10771000074617B9002009B0F0BD06A8FFF7A0FF83
:107720001BA00CF08BFE002406E006A8015D1BA048
:107730000CF084FE601C04B20C2CF6DB19A00CF0DB
:107740007DFE052408E0300240EA15662D0206A8F9
:10775000005D0543601E04B2002CF4DAB6B22A467E
:10776000334611A00CF06AFE13A2102102A8CDE945
:1077700000560CF073FE002404E002A8005D3855AA
:10778000601C04B20F2CF8DB0020F8730120C2E764
:1077900053544D33322049443D3D0000253032786A
:1077A000000000000D0A000074656D703D25303149
:1077B000356C6C750D0A0000253031356C6C750028
:1077C0002DE9F0438FB00023012219463548FDF71B
:1077D00031F901213348FDF789F900BF0221314811
:1077E000FDF7F7F80028F9D02E48FDF7EEF8064629
:1077F000642E0ADAB6F5805F07DB2BA00CF01EFEC4
:107800004FF0FF300FB0BDE8F0832A482A490968DD
:1078100040F8216028480068401C27490860092872
:1078200001DD00200860002406E0224850F8240012
:1078300005A941F82400641C0A2CF6DB002419E099
:1078400000204DF8240000250DE005A850F8250083
:107850005DF82410884205DD05A850F825004DF894
:1078600024002F466D1C0A2DEFDB002005A941F8EE
:107870002700641C042CE3DBDDE9010100EB0108B7
:107880000298C82802DA4FF0FF30BBE74FF49A7134
:1078900008FB01F0C11700EB11514FEA21394846AE
:1078A000B0E700000024014056444143204F5645B4
:1078B0005200000080210020F001002010B51D487A
:1078C00000781D490968884206D000201B490870CD
:1078D00019480078174908701848007810B1012835
:1078E00025D116E01448006848B115A003F082FFC6
:1078F00017A003F07FFF1DA00CF0A0FD05E021A064
:1079000003F078FF23A003F075FF01200B490870F6
:107910000DE00948006818B125A003F06BFF02E0F4
:1079200027A003F067FF02200449087000BF00BFD2
:1079300010BD0000DF010020B4000020DE010020A7
:1079400041542B4750533D224F4E220D0A00000058
:1079500041542B5649424354524C3D22504F5745B7
:1079600052222C224F4E220D0A0000004750532075
:107970006F70656E2D2D6368616E67652D2D720ABF
:107980000000000041542B4750533D224F464622F1
:107990000D0A000041542B5649424354524C3D229B
:1079A000504F574552222C224F4646220D0A0000C6
:1079B00041542B475053414E543D310D0A000000B5
:1079C00041542B475053414E543D300D0A000000A6
:1079D00010B500200F4981F8F802084690F8F80227
:1079E0000D4931F8100018B101200C49086008E079
:1079F00000200A4908600A48007820F00100084980
:107A00000870044890F8F8120448026805A00CF0C9
:107A100015FD10BDDE1B00204A7D0108B4000020CA
:107A2000281F00206E6577506172612E6770735455
:107A3000696D65496E6465783D3D3D25642C25641E
:107A40000D0A000010B58EB049480078002841D1D9
:107A50004848C08858B9484800684849884206D113
:107A600001200CF0F3F901204149087011E0414870
:107A7000C088401C3F49898888420AD13E48006836
:107A80003F49884205D102200CF0E0F90220384934
:107A90000870384801F0D8FF044637480068394973
:107AA000884210D1002038490870012037490871F8
:107AB0000846807918B101200AF08AFD54E00220BE
:107AC0000AF086FD50E0324884424DD13148D0F86A
:107AD000680200B949E001200CF0AAF92E480078AC
:107AE00001280ED12348C08800EB400101EBC00102
:107AF0002A4850F821302AA2322101A80CF0AEFC0D
:107B00000DE01C48C08800EB400101EBC001234898
:107B100050F8213028A2322101A80CF09FFC01A8C6
:107B200003F068FE012201A9002009F017FB1148AB
:107B3000C08800EB400101EBC001184800EB810058
:107B4000831D22A2322101A80CF088FC01202149CA
:107B50000870012201A9002009F000FB01200AF0B1
:107B600037FD00200249087000BF00BF0EB010BDF5
:107B700060030020C0240020400000202A04DC0014
:107B80002A04BC002A00FC00530200204A03002003
:107B90002A04EC005C0800209C000020D80900208A
:107BA00041542B504F433D656E74657267726F751B
:107BB000702C25640D0A000041542B504F433D307A
:107BC0003930303030253038780D0A00BDF8C8EB38
:107BD0003A257300D902002008B502201A239F22FB
:107BE0000D210090002000F00DF905480078802359
:107BF0001A461B210090002004F0F2FA08BD000094
:107C0000120400202DE9F05F04460D4616461F467B
:107C1000802C01DA802D01DBBDE8F09FA0198028BF
:107C200002DBC4F17F0086B2E819802802DBC5F1CF
:107C30007F0087B2E819401E83B2A019401E82B2AD
:107C40002946204601F012FB4FF0000818E005EB32
:107C500008001FFA80FA4FF000090BE004EB09005E
:107C60001FFA80FB084800780CF0F4F909F10100D4
:107C70001FFA80F9B145F1DB08F101001FFA80F825
:107C8000B845E4DB00BFC7E7120400202DE9FC5F24
:107C900004460D4616461F46B44201DCBD4201DDD6
:107CA000BDE8FC9F802E00DB7F26802F00DB7F2736
:107CB000301B401C80B20090781B401C1FFA80FBD8
:107CC00005EB0B00401E83B200982044401E82B298
:107CD0002946204601F0CAFA4FF0000829E005EBDA
:107CE00008001FFA80F94FF0000A1BE004EB0A00BD
:107CF00080B20190B9F10D0F04DA104800780CF051
:107D0000A9F90BE0B9F11B0F04DA0D4800780CF06B
:107D1000A1F903E00B4800780CF09CF90AF101008E
:107D20001FFA80FA00988245E0DB08F101001FFA93
:107D300080F8D845D3DB00BFB2E700001104002073
:107D40001004002012040020F8B507460D46164620
:107D50001C4604B9F8BDBD4200DAFBE7601EC4B2A0
:107D600000200090301983B22A463146384600F090
:107D700049F800BFEEE72DE9F84306460C461746E2
:107D80001D46DDF82080BE4201DCAC4201DDBDE8CD
:107D9000F8834346224639463046FFF7D5FF43462F
:107DA0002A4639463046FFF7CFFF01204346324688
:107DB00029460090204600F00AF8012043463A4642
:107DC00029460090204600F002F800BFDFE72DE9C9
:107DD000F84305460E4617461C46DDF820800CB9D0
:107DE000BDE8F883AE4200DAFAE7601EC4B2381983
:107DF00082B2334629463846CDF8008000F002F8BA
:107E000000BFEDE72DE9FC5F04460D4616461F4610
:107E1000B44201DCBD4201DDBDE8FC9F802C01DAEB
:107E2000802D00DBF8E7802E00DB7F26802F00DB33
:107E30007F27301B401C1FFA80FB781B401C1FFA59
:107E400080FA05EB0A00401E83B204EB0B00401ED3
:107E500082B22946204601F009FA4FF000083DE0C1
:107E600005EB080080B2009000987F2801DD7F209C
:107E700000904FF000092BE004EB090080B2019064
:107E800001987F2801DD7F2001900C98012815D0F2
:107E9000022808D003280BD004280ED111480078FE
:107EA0000CF0D8F80FE0104800780CF0D3F80AE096
:107EB0000E4908780CF0CEF805E000BF0C480078B9
:107EC0000CF0C8F800BF00BF09F101001FFA80F9EB
:107ED000D945D1DB08F101001FFA80F8D045BFDB9E
:107EE00000BF99E7130400201004002018040020AC
:107EF0001104002010B510A000F064FA18B90EA10A
:107F00000FA00CF09BFA16A000F05CFA18B914A1AF
:107F100015A00CF093FA1CA007F0EAFC1D4BFF2201
:107F20006FF07F414FF40B0000F03CF81AA20021E3
:107F3000084600F0E2F810BD485A4B313600000008
:107F400043616E27742066696E64207468652048FA
:107F50007A6B313646696C6528257329210D0A0034
:107F6000485A4B313200000043616E277420666925
:107F70006E642074686520487A6B313246696C659E
:107F800028257329210D0A00616C6C7069632E62CB
:107F90006D7000006464FF0077656C636F6D652E23
:107FA000626D7000F0B507460C4615461E46384611
:107FB000FEF79AF8094908702046FEF795F8084937
:107FC00008702846FEF790F8064908703046FEF71C
:107FD0008BF8054908700BF0CBFFF0BD11040020B1
:107FE0001204002010040020130400202DE9F84F93
:107FF00005460E461746984608F00F0908F0F00AA5
:10800000B9F1010F09D0B9F1020F21D0B9F1030F75
:1080100039D0B9F1040F6CD150E0002415E00120F3
:1080200006EB040C1FFA8CF305EB040C1FFA8CF220
:10803000A6EB040C1FFA8CF105EB040C00901FFA60
:108040008CF0FFF798FE601C84B2BC42E7DB51E085
:10805000002415E0012006EB040C1FFA8CF3A5EBBD
:10806000040C1FFA8CF2A6EB040C1FFA8CF1A5EBA2
:10807000040C00901FFA8CF0FFF77DFE601C84B2A8
:10808000BC42E7DB36E0002415E0012006EB040CDF
:108090001FFA8CF305EB040C1FFA8CF206EB040CB0
:1080A0001FFA8CF1A5EB040C00901FFA8CF0FFF77F
:1080B00062FE601C84B2BC42E7DB1BE0002415E0DA
:1080C0000120A6EB040C1FFA8CF305EB040C1FFA3D
:1080D0008CF2A6EB040C1FFA8CF1A5EB040C0090BB
:1080E0001FFA8CF0FFF747FE601C84B2BC42E7DB4E
:1080F00000E000BF00BFBDE8F88F2DE9F04FFDB0F4
:1081000080460D4691464846FEF736FE8346584661
:10811000FEF74EFE8246BAF1000F02D17DB0BDE8F7
:10812000F08F7CAB02221C21584605F0C9FF7BABC7
:1081300004221221584605F0C3FF7AAB042216210F
:10814000584605F0BDFF7B98802802D87A98802891
:1081500000D9E3E779AB04220A21584605F0B0FFC5
:1081600018207B990CF012F906467A98471E7A98E7
:108170002844401E83B27B984044401E82B2294668
:10818000404601F073F8002413E0799806FB0701DC
:1081900001AB3246584605F093FF01A800907B984A
:1081A00082B2281981B20123404604F091F97F1E62
:1081B000641C7A988442E8D300BFAFE72DE9FF4FF3
:1081C00085B0804692461F46DDF848B007F0F000C3
:1081D0000390039828B94FF00C0901250C20049056
:1081E00004E04FF0100901251020049054460026A9
:1081F00025E020789F280EDDCDE9007B637822788A
:1082000008EB060188B2069904F03CF806EB090079
:1082100086B2A41C13E0CDE9007B237808EB0601AD
:1082200088B20022069904F02DF8039818B906EBDD
:10823000C50086B202E006EBC50086B2641C207859
:108240000028D6D109B0BDE8F08F00000948C088E9
:108250000849898808430749498808430549098826
:108260000843054908800846018804A00CF0E6F898
:1082700000BFFEE738030020400300200D0A5B48E2
:1082800046483D253034785D0D0A000010B504469F
:108290004FF480612B48FEF7F5F9012803D1FF2048
:1082A0002949087002E0012027490870274890F901
:1082B0000000254991F90010884201D1002C1ED000
:1082C0002148007801280AD121A00CF0B7F824A099
:1082D00003F090FA0120264981F86F0209E025A0F9
:1082E0000CF0ACF827A003F085FA0020204981F8B3
:1082F0006F02154890F900001449087008E02548FD
:108300000078002804DD23480078401E21490870C9
:1083100021480078A8B1164890F86F0288B11F482C
:108320000FF0F0FC68B11E480078012803D11DA0B1
:1083300003F060FA02E01FA003F05CFA0020164987
:10834000087010BD000C01405C0200205D0200209E
:10835000B6FABBFABDD3C8EB2D2D2D0D0A000000D7
:1083600041542B41554443483D312C330D0A000004
:108370005C080020B6FABBFAB0CEB3F62D2D2D0D59
:108380000A00000041542B41554443483D302C30F5
:108390000D0A00005E020020E7020020E802002033
:1083A0009C00002041542B504F433D7074742C317D
:1083B0000D0A000041542B504F433D3042303030C5
:1083C000300D0A0070B505462C48406808B90020F9
:1083D00070BD2BA12846FBF71CFF58BB2A48002183
:1083E0000160416081602846FEF7C6FC0446002C0F
:1083F00001DA0020ECE71020234908704870097862
:10840000214A527801FB02F0C11700EB5171C1F310
:10841000C7011D4A91701046446004EB440000EB14
:10842000C4011648083000EB8100406A114688609C
:108430000120CDE715A12846FBF7EBFED8B915487A
:1084400000210160416081602846FEF795FC0446EA
:10845000002C01DA0020BBE70E48446004EB440026
:1084600000EBC4010548083000EB8100406A09496F
:1084700088600120ACE700BFAAE70000FC2A0020CA
:10848000485A4B3136000000E4260020485A4B3150
:1084900032000000F026002010B504460121C80279
:1084A00005F0F2FB7D2005F083FC08B105F00CFC23
:1084B00045F2555000F028F8062000F019F8A0B257
:1084C00000F01CF800F00CF800F002F810BD0000FD
:1084D0004CF6CC4001490860704700000030004075
:1084E0004AF6AA20014908607047000000300040A9
:1084F0000149486070470000003000400149886031
:1085000070470000003000400149086070470000DB
:108510000030004030B50346002500240BE01878F9
:10852000884201D1681CC5B25B1C601CC4B2AA425F
:1085300001D1204630BD18780028F0D100BFF9E7FE
:10854000002101600171FF2141710021817170479B
:1085500000B587B00121880205F0A6FB01210420A7
:1085600005F0A2FB0220ADF8040048208DF80700BA
:1085700001A91648FDF7B2FF6420FDF72EF8002090
:108580008DF8070001A91148FDF7A8FFC820FDF7E5
:1085900024F8002002908DF80C008DF80D004FF4A7
:1085A000602004900020059001208DF8180002A999
:1085B0000748FCF717FA01210548FCF7FBF90121F0
:1085C0000348FCF793FA07B000BD00000008014023
:1085D0000028014004480078FF2804DA02480078A7
:1085E000401C0149087070474700002010B5A7489B
:1085F0000078A7490978884207D0A5480078A349A0
:1086000008700020A349087010BDA3480078012815
:108610001ED19F48007801281AD1A0480068B0F503
:10862000842F0ED09D4800689D49884209D09B4800
:108630000068B0F5C02F04D0984800689949884276
:1086400006D1002093490870012097490870DBE7A4
:1086500092480068954A811A904270D018DCB0F5B3
:10866000C02F7ED009DCB0F5083F38D0B0F5802FA0
:1086700067D0B0F5842F3FD14EE0B0F5E02F6FD03A
:10868000B0F5601F1ED08A4908440028F3D1A7E046
:10869000884A881A91426ED009DCB1F5001F6BD070
:1086A000B1F5401F70D0B1F5601FE4D174E001282E
:1086B00070D08149084400286DD0804908440028C2
:1086C000D9D15BE07E480FF01DFB10B900207D4939
:1086D000087001227CA1002008F040FD00BF0122AB
:1086E0007FA1002008F03AFD0020854908708549E7
:1086F00008708548007800B1BDE084480078012802
:1087000003D183A003F076F802E085A003F072F8AD
:10871000002087490870AEE0012286A1002008F001
:108720001DFD0020884908748848807850B10020D9
:108730008649887086A1012001F032FE09E037E009
:108740000FE03EE08BA1012001F02AFE01207F49CD
:108750008870002003F0E8F90020754908708AE06D
:1087600055E00020724908708B49087001228BA1E6
:1087700008F0F4FC7FE03CE014E005E001228CA16D
:10878000002008F0EBFC76E001228EA1002008F02A
:10879000E5FC70E033E01DE0012291A1002008F02B
:1087A000DDFC68E0012295A1002008F0D7FC62E022
:1087B000012298A1002008F0D1FC00203549087062
:1087C00059E001229AA1002008F0C8FC002033499A
:1087D000086050E001229DA1002008F0BFFC4AE0A3
:1087E0000122A1A1002008F0B9FC00202B4908605B
:1087F00041E00122A3A1002008F0B0FC3BE00020F2
:10880000244908700122A4A108F0A8FC33E0012249
:10881000A6A1002008F0A2FC1F48007801280BD177
:10882000002000F0CBFC494890F89A10903000EB03
:1088300041000088A349088017480078202816D0F6
:10884000154800780E2812D01348007808280ED05A
:108850001148007801280AD00F4800780D2806D06A
:108860000D480078052802D0012009F0B1FE002053
:108870009549087000BF00BF0848006893498842C6
:1088800002D000202A49087000BFBDE6F102002096
:10889000E4020020E2020020460300204000002005
:1088A0002A04EC002A00FC00E50200202A04BC0097
:1088B000D6FB53FF01003800FDFBFBFF0408FCFF63
:1088C000E8020020E70200205B484541445345543C
:1088D0005F4D49432052656C656173655D00000022
:1088E0005B4B45595F5050542F4B45595F50505486
:1088F0005F4D49432052656C656173655D00000002
:108900004600002049000020DA0200209C000020E0
:1089100041542B504F433D7074742C300D0A0000AD
:1089200041542B504F433D3043303030300D0A001E
:10893000450000205B4B45595F55502052656C65E2
:108940006173655D000000005C080020DE1B0020F4
:108950003243443244314339453844364333423359
:1089600043394246454342444444433842414437F4
:1089700045390000324344324431433945384436A6
:1089800043334233433942464543424444444235EB
:108990004135424146340000E30200205B4B45591B
:1089A0005F444F574E2052656C656173655D0000F2
:1089B0005B4B45595F4F4B2052656C656173655D3C
:1089C000000000005B4B45595F50414E454C5F4DE8
:1089D000454E552052656C656173655D0000000071
:1089E0005B4B45595F50414E454C5F4558495420BB
:1089F00052656C656173655D000000005B4B455915
:108A00005F50414E454C5F55502052656C65617317
:108A1000655D00005B4B45595F50414E454C5F44DE
:108A20004F574E2052656C656173655D0000000014
:108A30005B4B45595F455849545F444F574E5F471C
:108A4000542052656C656173655D00005B4B455950
:108A50005F50315F50335F5550444154452052655B
:108A60006C656173655D00005B4B45595F55505FF8
:108A7000444F574E5F49502052656C656173655D88
:108A8000000000005B4B45595F50312052656C651A
:108A90006173655D000000005B4B45595F503220FB
:108AA00052656C656173655D000000005B4B455964
:108AB0005F4F5054494F4E2052656C656173655D40
:108AC00000000000B0000020DE0200202A04FC00AC
:108AD00070B500240025FEF7BFF944B2FEF75EFA38
:108AE00045B20121204600F0D3FA0021284600F0CB
:108AF000CFFA70BD08B50121192005F0D5F8012184
:108B00002248FDF777FD48208DF8030003208DF8FB
:108B100002000420ADF8000069461D48FDF7DEFCA8
:108B20000420ADF8000069461948FDF7D7FC4FF462
:108B30000050ADF8000069461648FDF7CFFC022052
:108B4000ADF8000069461248FDF7C8FC48208DF8D2
:108B5000030003208DF802004FF40060ADF8000020
:108B600069460B48FDF7BAFC48208DF80300032046
:108B70008DF802004FF48060ADF8000069460448AB
:108B8000FDF7ACFC00200449087008BD000230006D
:108B9000000C0140001001404500002000B589B0E4
:108BA000AE480078012819D1AD480078012815D1C8
:108BB000AC480068B0F5842F0ED0AA480068AA49D6
:108BC000884209D0A7480068B0F5C02F04D0A54856
:108BD0000068A649884201D109B000BDA1480068DB
:108BE000A34A811A904271D018DCB0F5C02F6ED024
:108BF00009DCB0F5083F3DD0B0F5802F68D0B0F566
:108C0000842F36D17CE0B0F5E02F76D0B0F5601F30
:108C10001ED0984908440028F3D10AE1964A881AE0
:108C200091426BD009DCB1F5001F68D0B1F5401F4F
:108C30007ED0B1F5601FE4D1ABE0012879D08F4937
:108C40000844002876D08E4908440028D9D17AE01B
:108C50008C4890F86F0200B9BEE701208A4908707D
:108C600014218A480FF066F8012289A1002008F03B
:108C700075FAEFE001208B4908708248007C0028DB
:108C800027DD8948807870B901208849087008F08C
:108C900037FB874B87A21E2101A80BF0DFFB01A841
:108CA00002F0A8FD23E07748808920B986A1012041
:108CB00001F076FB1BE07E4B093B8BA21E2101A835
:108CC0000BF0CCFB01A802F095FD10E079E01FE06D
:108CD000A3E08A48007850B989480078012803D178
:108CE00088A002F087FD02E08AA002F083FD012245
:108CF0008CA1002008F032FAACE0A0E04FE05AE08E
:108D000000206849087001228DA108F027FAA1E02F
:108D10000020644908708E480078401CC0B28C491D
:108D20000870022809DD01208A4988711E2002E0AE
:108D30000FE03AE077E009F04BFC012286A1002029
:108D400008F00CFA86E0012288A1002008F006FA5B
:108D500080E0012289A1002008F000FA8D48007807
:108D6000B0B100208B490870514B213B51A21E210C
:108D700001A80BF073FB01A802F03CFD86A26B2159
:108D8000012007F0FDFB002201A9104608F0E6F9DA
:108D900060E0012282A1002008F0E0F95AE00122FF
:108DA00085A1002008F0DAF954E0012286A1002014
:108DB00008F0D4F94EE0012287A1002008F0CEF996
:108DC00048E001228AA1002008F0C8F98E48007806
:108DD000401CC0B28C49087002281DD12048007880
:108DE00080B100201E49087088A00BF027FB1B48AB
:108DF0000078012810D10C23682200215C20FEF7A6
:108E000045FF09E001201649087009F0E1FB83A243
:108E100000215C20FFF771F91CE0012282A10020F3
:108E200008F09CF916E0012286A1002008F096F9CE
:108E300010E001228AA1002008F090F90AE08E4893
:108E40000078401C8C49087001228CA1002008F099
:108E500085F900BF00BF00BFBEE60000460300204A
:108E6000E4020020400000202A04EC002A00FC005C
:108E70002A04BC00D6FB53FF01003800FDFBFBFFBA
:108E80000408FCFF5C080020E7020020E802002044
:108E90005B484541445345545F4D494320507265FA
:108EA00073735D0045000020DE1B0020D902002006
:108EB000D50A002041542B504F433D3039303030DB
:108EC0003025730D0A0000003243434544454336C4
:108ED00045344342464342334339443442314434B7
:108EE000444143464446000041542B504F433D30DB
:108EF000413030303025730D0A000000DA020020C6
:108F00009C00002041542B504F433D7074742C3111
:108F10000D0A000041542B504F433D304230303059
:108F2000300D0A005B4B45595F5050542F4B45594B
:108F30005F5050545F4D49432050726573735D001C
:108F40005B4B45595F55502050726573735D00004F
:108F5000E30200204A0300205B4B45595F444F5712
:108F60004E2050726573735D000000005B4B4559E5
:108F70005F4F4B2050726573735D00005B4B45592A
:108F80005F50414E454C5F4D454E552050726573C4
:108F9000735D0000DC020020B2CBB5A5000000002C
:108FA0005B4B45595F50414E454C5F4558495420F5
:108FB00050726573735D00005B4B45595F50312003
:108FC00050726573735D00005B4B45595F503220F2
:108FD00050726573735D00005B4B45595F50414EA5
:108FE000454C5F55502050726573735D0000000062
:108FF0005B4B45595F50414E454C5F444F574E20A7
:1090000050726573735D0000E2020020636C65615D
:1090100072206C6F636B2D2D2D0D0A006C6F636BCE
:109020002E626D70000000005B4B45595F4558494A
:10903000545F444F574E5F47542050726573735DC1
:10904000000000005B4B45595F50315F50335F5566
:1090500050444154452050726573735D0000000018
:109060005B4B45595F55505F444F574E5F49502009
:1090700050726573735D0000DE0200205B4B455942
:109080005F4F5054494F4E2050726573735D00001E
:1090900070B504460D46012C41D100F08FF8002038
:1090A0003149088031480078401C30490870304808
:1090B0000068B0F5083F19D02E4890F8F702012853
:1090C00014D108460078022810DA0EF0BFFD2A49B4
:1090D000096888420AD90A214FF47A7005F0F2FB38
:1090E00008F024F90F2100200EF0F8FD2348007845
:1090F00050B91F480068B0F5601F05D01C480068D3
:10910000B0F5083F00D070BD1D480068401C1C49E8
:109110000860FFF743FD0A201A49087022E0601C2E
:1091200000BB00201149087017480078012806D1BB
:109130002DB116A002F05EFB0020134908700F4805
:10914000007850B90A480068B0F5601F05D008489B
:109150000068B0F5083F00D0D5E7FFF747FA0A20CE
:109160000849087000BFCEE7B0000020F2020020DE
:1091700040000020DE1B0020080300200D0400201A
:10918000EC020020E60200204900002041542B5050
:109190004F433D3043303030300D0A000548016800
:1091A0000548826801F00601090402F4005241EA10
:1091B00002007047080C01400010014010B5044641
:1091C0001C4800781C4908702CBB1A4804704FF4E6
:1091D00080501A490860282000F028FA184890F8B2
:1091E000F802184931F810001E2805DA144890F8E2
:1091F000F80231F8100018B93C201349087017E044
:109200000F4890F8F8020F4911F810004006000EC0
:109210000D4908700CE00A200B49087005480470DD
:109220004FF480500549091F0860292000F0FEF91D
:1092300010BD00000E0400200D04002014080140A1
:10924000DE1B00204A7D01085102002010B50446B3
:109250002146054805F090F900BF8021024805F03D
:109260007FF90128F9D010BD003800402DE9F05FEA
:1092700004460D4616461F46A046B146AA46BB46C2
:109280002A2000F0D3F94FEA282000F0E3F908F093
:10929000FF0000F0DFF94FEA292000F0DBF909F0C8
:1092A000FF0000F0D7F92B2000F0C0F94FEA2A2088
:1092B00000F0D0F90AF0FF0000F0CCF94FEA2B20C3
:1092C00000F0C8F90BF0FF0000F0C4F92C2000F00A
:1092D000ADF9BDE8F09F00002DE9F0410E4800888F
:1092E00006120D4807787F231A4600210846FFF72B
:1092F000BDFF00240BE0002506E0304600F0AAF98F
:10930000384600F0A7F96D1C802DF6DB641C802C1C
:10931000F1DBBDE8F08100000804002010B500F08A
:109320000DF94FF48050844908604010091F08600F
:109330000120FCF752F94FF400607F4908600120DA
:10934000FCF74BF94FF400607B49091F0860782057
:10935000FCF743F9FE2000F069F9EF2000F066F910
:10936000362000F063F9682000F074F93A2000F02C
:109370005DF9052000F06EF9B62000F057F91120D4
:1093800000F068F9AC2000F051F90B2000F062F910
:10939000B42000F04BF9212000F05CF9B12000F07E
:1093A00045F9C02000F056F9B22000F03FF908203E
:1093B00000F050F9B32000F039F9232000F04AF909
:1093C000EB2000F033F9112000F044F9662000F0A2
:1093D00041F92A2000F02AF9002000F03BF9002092
:1093E00000F038F9002000F035F97F2000F032F964
:1093F0002B2000F01BF9002000F02CF9102000F0C9
:1094000029F9002000F026F9A02000F023F9F5202A
:1094100000F00CF9092000F01DF9842000F01AF981
:10942000E62000F003F9282000F014F9002000F0F5
:1094300011F9E72000F0FAF8702000F00BF9002095
:1094400000F008F9F02000F0F1F8042000F002F933
:10945000322000F0FFF8252000F0FCF8412000F059
:10946000F9F8BA2000F0F6F80E2000F0F3F80F201B
:1094700000F0F0F8002000F0EDF8012000F0EAF82C
:109480000B2000F0E7F80E2000F0E4F8192000F0BF
:10949000E1F8182000F0DEF80F2000F0DBF8F120F2
:1094A00000F0C4F8072000F0D5F83C2000F0D2F816
:1094B0002D2000F0CFF8502000F0CCF8AC2000F0C8
:1094C000C9F8252000F0C6F8252000F0C3F80020D8
:1094D00000F0C0F8012000F0BDF80C2000F0BAF850
:1094E0000E2000F0B7F8152000F0B4F8142000F0BA
:1094F000B1F80F2000F0AEF8FE2000F097F8FF2042
:1095000000F094F8212000F091F8112000F08EF87E
:109510007820FCF762F8292000F088F84FF6FF71F8
:10952000002000F0ABF8FFF7D7FE4FF4805002495F
:10953000091F086010BD00001408014000B587B085
:1095400001210C2004F0B0FB03208DF81A0010203C
:109550008DF81B000121800204F096FB4FF480403F
:10956000ADF8180006A92E48FCF7B8FF4FF480406C
:109570002B49103108608010ADF8180006A9284862
:10958000FCF7ACFF4FF40050ADF8180018208DF830
:109590001B0006A92248FCF7A1FF4FF40040ADF8DC
:1095A000180006A91E48FCF799FF4FF480501C498B
:1095B000103108604FF44040ADF804004FF4827061
:1095C000ADF806000020ADF80800ADF80A00ADF8CF
:1095D0000C004815ADF80E000020ADF81000ADF8F5
:1095E00012000720ADF8140001A90E4804F0C6FFD0
:1095F00001210C4804F0A8FF10208DF81B004FF447
:10960000C050ADF8180006A90748FCF767FF4FF4F3
:1096100000600549103108604000086007B000BDD7
:10962000000C0140003800400008014010B504461D
:109630004FF4804006490860801008602046FFF71C
:1096400005FE4FF480500249091F086010BD00005C
:10965000140C014010B504464FF4804006490860E0
:109660008010091D08602046FFF7F0FD4FF4805080
:109670000149086010BD0000100C0140024A108032
:10968000024A1180704700000A04002008040020EC
:1096900008B501210C2004F007FB10208DF8030011
:1096A00003208DF802004020ADF80000694608480C
:1096B000FCF714FF8020ADF8000069460448FCF771
:1096C0000DFF40200249143108608020086008BD69
:1096D000000C0140F8B10021604A1160604A11702D
:1096E000604A1170604A1170FF21604A1170604A2F
:1096F000117000215F4A11705F4A11705F4A11704A
:10970000FF215F4A11705F4A117040215E4A11606B
:109710008021116070475D49097819B940215A4A82
:10972000116048E05A49097821B94021564A121F70
:10973000116040E04D490978544A1278914205D1B0
:109740004B490978524A1278914219D00021444A73
:109750001170484A11704D490978444A11704C49BA
:109760000978434A1170494909784906090E3E4A69
:1097700011703F490978127802EB4101394A1170A2
:1097800037490978491CC9B2354A1170354A1278EF
:10979000914202DD0021324A117031490978324A82
:1097A0001278914204DA4021374A121F116002E018
:1097B0004021354A11603749097819B98021324A68
:1097C000116048E03449097821B980212E4A121FDE
:1097D000116040E02A4909782E4A1278914205D159
:1097E000284909782C4A1278914219D000211C4A44
:1097F0001170204A117027490978214A11702649B1
:109800000978204A1170234909784906090E1B4A34
:1098100011701C490978127802EB4101164A117047
:1098200014490978491CC9B2124A1170124A1278B7
:10983000914202DD00210F4A11700E4909780F4A4A
:109840001278914204DA80210F4A121F116002E05F
:1098500080210D4A116000BF5CE700007800002005
:109860007C0000207D0000207E0000207F00002082
:109870008000002081000020820000208300002062
:109880008400002085000020140C01406C000020A2
:109890006D0000206E0000206F0000202DE9F047D1
:1098A0000446884691461E46DDF820A0C4F8008094
:1098B000002507E0206850F82500077807B903E085
:1098C000681CC5B2C82DF5DB00BF681EC5B2681C98
:1098D000A080052095FBF0F060816089052190FB58
:1098E000F1F201FB120010B16089401C608100257B
:1098F000C4F8D8600AE006B90AE0D4F8D80050F8F5
:109900002500077807B903E0681CC5B2C82DF2DB53
:1099100000BFA4F8DC5000250EE0A088A84205DDB9
:109920001AF8051004F10D00415503E0002104F17F
:109930000D004155681CC5B2C82DEEDB84F80C90B3
:1099400000202081E080204600F0D2F9BDE8F087B9
:109950002DE9F04704460F4616469846A4F83A719A
:109960000120A4F83C010020E08084F80C80002550
:10997000C4F8D8600DE006B90DE0D4F8D80050F86E
:10998000250090F80090B9F1000F00D103E0681CA9
:10999000C5B2C82DEFDB00BFA4F8DC50642084F80A
:1099A0003801642201212046FDF7FAFBBDE8F0876B
:1099B0002DE9FF4106460F460A2E01DA012409E08F
:1099C000642E01DA022405E0B6F57A7F01DA032479
:1099D00000E004240A2F01DA012509E0642F01DAEE
:1099E000022505E0B7F57A7F01DA032500E00425BA
:1099F000334612A20B2101A800970AF02FFD60192F
:109A00001049098888420AD060190E49088002204E
:109A10001923A0220D2100905020FEF7F3F9002019
:109A20006119891CC900C1F1A001009088B201230D
:109A300001AA0D21FEF7C2FBBDE8FF8125647C254C
:109A400064000000200400207FB50446A08818B9F7
:109A50004D48006804B070BD4B4800684B4908444D
:109A6000002842D0B0F5001F7ED10021204600F032
:109A70006EF9E08818B9A088401EE08002E0E08816
:109A8000401EE080257AE088052190FBF1F02081DE
:109A90002089A84203D0204600F02AF903E00121E2
:109AA000204600F054F93A480078042803D038489A
:109AB0000078032818D13748B0F86C00401C00EB40
:109AC0008000E188401A0090324833A20A21D0F881
:109AD000683201A80AF0C2FC0020012301AA0D216E
:109AE00000904420FEF76AFB4BE00021204600F086
:109AF0002EF9E088401CE080E088A188884201DBE4
:109B00000020E080257AE088052190FBF1F020819B
:109B10002089A84203D0204600F0EAF803E00121A2
:109B2000204600F014F91A480078042803D0184899
:109B30000078032821D11748B0F86C0000EB8000B2
:109B4000E1880844401C0090124813A20A21D0F872
:109B5000683201A80AF082FCE2880E48B0F86C1066
:109B600010A00AF06BFC00E008E00020012301AA2D
:109B70000D2100904420FEF721FB02E0024800681E
:109B800068E700BF002065E740000020D6FB43FFE8
:109B9000460300205C080020253033642F25303335
:109BA0006400000068616E646C65496E6465783DB0
:109BB0003D25642C702D3E68616E646C653D3D3DB5
:109BC00025640D0A0000000010B50446A08810B9F5
:109BD0004548006810BD44480068444908440028CE
:109BE0003ED0B0F5001F03D0B0F5601F76D172E013
:109BF0000021204600F0EAF8B4F83C01401EA4F829
:109C00003C01B4F83C0118B9B4F83A01A4F83C019D
:109C1000E08880B9B4F83A01052808DD75220021F2
:109C20002046FDF7BDFA012084F83E0106E0A08839
:109C3000401EE08002E0E088401EE08094F83E0193
:109C400018B1002084F83E0103E00121204600F015
:109C5000BDF8B4F83A11B4F83C01FFF7A9FE40E0B2
:109C60000021204600F0B2F8E088401CE080B4F803
:109C70003C01401CA4F83C01B4F83C01B4F83A1192
:109C8000884202DD0120A4F83C01E088A1888842D6
:109C90000EDBB4F83A01052808DD642200212046D5
:109CA000FDF77EFA012084F83E0101E00020E0800B
:109CB00094F83E0118B1002084F83E0103E0012130
:109CC000204600F083F8B4F83A11B4F83C01FFF7ED
:109CD0006FFE06E002E0044800687BE70248006887
:109CE00078E700BF002075E740000020D6FB43FF67
:109CF0002DE9F0410546A88808B9BDE8F081287A29
:109D000000EB8000C6B2344618E0A888A0420FDC01
:109D1000052094FBF0F100FB11401D2101EB001028
:109D200087B21023902239460020FDF76BFF03E035
:109D30002146284600F086F8601CC4B2701D84429B
:109D4000E3DB0121284600F002F800BFD5E72DE94A
:109D5000F04186B004460E464FF00008D4F8D80013
:109D600018B108F1100000F0FF08E088052190FB11
:109D7000F1F201FB1200C7B21D2000EB0710C5B2C3
:109D8000E288206850F82210112201A807F060FB39
:109D90004EB1042005F10E038C2229460090404666
:109DA000FEF730F808E0032005F10E038C22294667
:109DB00000904046FEF726F8012301AA29464046B6
:109DC0000096FEF7FBF906B0BDE8F0812DE9F04101
:109DD00086B004460E464FF00008D4F8D80018B1FB
:109DE00008F1100000F0FF08A7791D2000EB071014
:109DF000C5B24EB1042005F10E036C222946009035
:109E00004046FDF7FFFF08E0032005F10E036C223A
:109E1000294600904046FDF7F5FFE08800EBC002C0
:109E200004F1DE0000EB4201112201A807F010FB53
:109E3000012301AA294640460096FEF7BFF906B065
:109E4000BDE8F0812DE9F0438BB004460D460520B6
:109E500095FBF0F100FB115087B200261D2000EBAE
:109E600007101FFA80F910238E2249463046FDF76D
:109E7000C9FE142106A8FAF790F9207B18B100203A
:109E80008DF82B0009E0206850F82510142206A850
:109E9000FAF7ACF900208DF82B00112206A901A8D1
:109EA00007F0D6FAD4F8D800B0B104F10D0010F8DC
:109EB0000580D4F8D80050F8282049463046FEF7EF
:109EC0001CF9002006F11001009088B2012301AABC
:109ED0004946FEF773F907E00020012301AA49462D
:109EE00000903046FEF76AF90BB0BDE8F083000041
:109EF0002DE9F0438BB004460D46052095FBF0F1AB
:109F000000FB11501FFA80F800271D2000EB0810FD
:109F10001FFA80F910238E2249463846FDF772FE5B
:109F2000142106A8FAF739F9207B18B100208DF822
:109F30002B000CE005EBC50204F1DE0000EB420152
:109F4000142206A8FAF752F900208DF82B001122EE
:109F500006A901A807F07CFAD4F8D80058B305EB9D
:109F6000C50104F1DE0000EB4100407CB4F8DC10D8
:109F7000884206DB012215A1002007F0EFF8002639
:109F800006E005EBC50104F1DE0000EB4100467C74
:109F9000D4F8D80050F8262049463846FEF7ADF8E8
:109FA000002007F11001009088B2012301AA494660
:109FB000FEF704F907E00020012301AA49460090BA
:109FC0003846FEF7FBF80BB0BDE8F0834C42310099
:109FD0002DE9F0410446A08808B9BDE8F0810025CC
:109FE00012E0A088A84209DC1D2000EB0517102311
:109FF000902239460020FDF705FE03E02946204661
:10A00000FFF776FF681CC5B2052DEADB94F838012E
:10A01000752802D1A088401EE08001212046FFF76C
:10A02000D5FE6F26B4F83A01052808DD06F10801CF
:10A0300088B2032308221D21FDF7D8FF05E008237D
:10A0400010221D213046FDF7DDFD6D27B4F83A01E1
:10A05000052808DD06F1080188B2042308223946E4
:10A06000FDF7C4FF07E0A7F1080081B20823102222
:10A070003046FDF7C7FD00BFAFE70000F0B58FB079
:10A0800004460126012704EB840000EB4411174825
:10A090000D18687910B900200FB0F0BD1448007891
:10A0A00010B1052817D106E0631C12A2322102A8C4
:10A0B0000AF0D4F912E0A87858B9B5F80300691D80
:10A0C000631C11A2CDE90010322102A80AF0C6F9E2
:10A0D00000E0002702E00026002700BF00BF17B104
:10A0E00002A801F087FB3046D6E7000033210020AC
:10A0F0005202002041542B54435053544154555361
:10A100003D25640D0A00000041542B5443504F502C
:10A11000454E3D25642C25733A25640D0A00000048
:10A120002DE9F04190B0044620680E9060680F90D1
:10A130002088C0F3C507382F02DAC7F1380001E0E4
:10A14000C7F17800804642462849204600F062F870
:10A150000026002518E004F11800E91C405C020606
:10A1600004F11800A91C405C42EA004204F1180006
:10A17000691C405C42EA002004F11801495D084373
:10A180004DF82600761C2D1D0E2EE4D3694604F1F1
:10A19000080007F0C1FC0026002521E004F10800BA
:10A1A00010F8261050304155503830F82600C0F3D2
:10A1B000072204F15800691C4254503850F8260018
:10A1C000C0F3074204F15800A91C4254503850F81B
:10A1D0002600000E04F15801EA1C8854761C2D1D3F
:10A1E000042EDBD310B0BDE8F0810000A88F010879
:10A1F00000214160016005498160054AC260CA438F
:10A200000261034AD243426170470000012345675F
:10A2100089ABCDEF2DE9F04391B004460F461546CA
:10A220002088C0F3C509206800EBC500216888427A
:10A2300002D26068401C6060206800EBC5002060AE
:10A24000606800EB5570606033E017F8012B4846FA
:10A2500009F1010904F118010A54B9F1400F28D19C
:10A260004FF0000800261AE004F11800F11C405CD1
:10A27000020604F11800B11C405C42EA004204F1FD
:10A280001800711C405C42EA002004F11801895D4D
:10A29000084301A941F8280008F10108361DB8F16A
:10A2A000100FE1D301A904F1080007F035FC4FF0CD
:10A2B0000009281EA5F10105C7D111B0BDE8F08342
:10A2C00008B54FF4A06001F0C9FD25208DF800000D
:10A2D00001208DF801008DF802008DF8030068461A
:10A2E00001F084FD26208DF8000001208DF801008A
:10A2F0008DF802008DF80300684601F077FD092013
:10A300008DF8000001208DF801008DF802008DF815
:10A310000300684601F06AFD0A208DF80000022063
:10A320008DF8010001208DF802008DF803006846C9
:10A3300001F05CFD17208DF8000002208DF801006F
:10A3400001208DF802008DF80300684601F04EFDF3
:10A350004FF4C06001F082FD03208DF80000012061
:10A360008DF8010000208DF8020001208DF8030017
:10A37000684601F03BFD08BD70B50546002407E0C6
:10A38000285D0D2802D10020285570BD601C84B2C4
:10A390002846F9F737FFA042F2D800BFF5E70000E2
:10A3A00030B585B004460D46012006F0A9FF2346CE
:10A3B00009A2142168460AF051F8684601F01AFA19
:10A3C000284601F017FA08A001F014FA0120074905
:10A3D000087105B030BD000041542B4C5348545413
:10A3E000533D25642C220000220D0A005C08002049
:10A3F00000BFFEE72DE9F04104460F462760002527
:10A4000000BF206850F8250090F80080B8F1000FD8
:10A4100000D102E0681CC5B2F3E700BF681EC5B2F8
:10A42000681C2071052095FBF0F0E071E0790521B2
:10A4300090FBF1F201FB120010B1E079401CE071D9
:10A440000E4800680E49884202D00E48007960B17B
:10A450000C4803F0E3FBC6B2052096FBF0F0A071B8
:10A46000667100200749087102E00020A071607148
:10A47000204600F05BF8BDE8F081000040000020BD
:10A480002A00FC004A03002070B5044625480068F5
:10A490002549084408B3B0F5001F3DD100212046EE
:10A4A00000F09DF8607918B92079401E607102E0D3
:10A4B0006079401E6071A5796079052190FBF1F00B
:10A4C000A071A079A84203D0204600F02FF803E045
:10A4D0000121204600F083F821E00021204600F011
:10A4E0007EF86079401C607160792179884201DBD7
:10A4F00000206071A5796079052190FBF1F0A071D1
:10A50000A079A84203D0204600F010F803E0012112
:10A51000204600F064F802E00248006870BD00BF09
:10A520000020FBE740000020D6FB43FF2DE9F0416F
:10A530000446A07900EB800000F0FF08454619E0D2
:10A540002079A84210DC052095FBF0F100FB1150AA
:10A550001D2101EB001087B2781E81B210237822F2
:10A560000020FDF74FFB03E02946204600F06FF87E
:10A57000681CC5B208F105008542E1DB01212046D7
:10A5800000F02DF87C26A079002808DD06F10A01EC
:10A5900088B2032308221D21FDF728FD05E01223C0
:10A5A0001A461D213046FDF72DFB6D27A179E07974
:10A5B000401E814209DABA1E91B206F10A0290B237
:10A5C00004230822FDF712FD07E0A7F10A0081B27B
:10A5D000082313223046FDF715FBBDE8F0812DE975
:10A5E000F84F04460D464FF000096079052190FBB5
:10A5F000F1F201FB120000F0FF081D2000EB081033
:10A60000C6B26179206850F821703846FDF74CF8E1
:10A610000FFA80FA4DB1042006F10E038C22314668
:10A6200000904846FDF7EEFB08E0032006F10E031C
:10A630008C22314600904846FDF7E4FB01233A4660
:10A64000314648460095FDF7B9FDBDE8F88FF8B5ED
:10A6500005460C46052094FBF0F100FB1140C6B204
:10A660001D2000EB0610C7B2781E81B2122378229B
:10A670000420FDF7C7FA00200090286850F8242035
:10A68000012339460020FDF799FDF8BD10B50B48B0
:10A6900000680B49884208D10A484088012801DB3C
:10A6A000FAF7D2FF052007F093FF04480068064937
:10A6B000884202D1052007F08BFF10BD400000202A
:10A6C0002A04EC00A82100202A04F40038B504462E
:10A6D000ACB1FDF781FA012109A005F0CDFF0BA077
:10A6E00006F09AF801236E229F210020FDF72CFB33
:10A6F0000020012308A272210090FDF75FFD38BD04
:10A70000CFFBCFA2C9BEB3FD00000000C8B7B6A8FA
:10A71000C9BEB3FD3F0000005B4D5DC8B7B6A820C1
:10A72000205B455849545DC8A1CFFB002DE9F0419D
:10A7300004460F4615461E462780A5703046F9F799
:10A7400061FD84F87500102084F87700002084F8FB
:10A750007400BDE8F0812DE9F84F044689464FF0BA
:10A76000000A4E4694F802C094F877E00CEB0E0312
:10A77000B4F800C094F876E0F4441FFA8CF2A178A3
:10A780002088FDF73FFA142104F16000F9F705FD78
:10A790002088C0F17F0087B23846F91707EB517166
:10A7A000C1F3C70184F87410D0460025AB4646E0DB
:10A7B00030789F2810DD94F87400401B022808DBD5
:10A7C00004F16000284431880180A81CC5B2B61C81
:10A7D00011E04FF0010B0EE094F87400401B0128CB
:10A7E00007DB317804F160004155681CC5B2761C66
:10A7F00001E04FF0010BBBF1000F20D04FF0000B38
:10A80000002104F1600041550020009094F802C03E
:10A810004246531C03F0FF080CEB02112088102362
:10A8200004F16002FDF7CAFC0AEB05001FFA80FA8A
:10A830000025B8F1050F02DB5046BDE8F88F3078EF
:10A840000028B5D1002104F160004155002000909E
:10A8500094F802C04246531C03F0FF080CEB0211AF
:10A860002088102304F16002FDF7A8FC0020E4E733
:10A8700010B5094800680949884204D1FBF74EFD2C
:10A88000052007F0A5FE044800680549884202D16A
:10A89000052007F09DFE10BD400000202A04EC00BA
:10A8A0002A04F40038B50446ACB1FDF795F901214E
:10A8B00009A005F0E1FE0BA005F0AEFF01236E221A
:10A8C0009F210020FDF740FA0020012309A27221F8
:10A8D0000090FDF773FC38BDCFFBCFA2B8F1CABD25
:10A8E000BBAF0000C8B7B6A8C9BEB3FDCBF9D3D083
:10A8F000A3BF00005B4D5DC8B7B6A820205B4558DC
:10A9000049545DC8A1CFFB0010B51048FFF7BCFD4E
:10A9100004460F4884420ED10C48407910B10128FA
:10A9200008D103E00A2007F053FE03E00B2007F0F4
:10A930004FFE00BF08E0074800680749884203D17E
:10A940000649487807F044FE10BD0000B80000201A
:10A950002A04EC00400000202A04F40046030020F2
:10A9600038B50446E4B1FDF737F901210DA005F033
:10A9700083FE01236E229F210020FDF7E5F90C499B
:10A980000C48FFF737FD01236E229F210020FDF7C1
:10A99000DBF90020012308A272210090FDF70EFCD4
:10A9A00038BD0000CEC4B1BED1A1CFEE0000000082
:10A9B0000C020020B80000205B4D5DC8B7B6A8208F
:10A9C0002020205B455849545DCDCBB3F6000000F4
:10A9D00010B51C4800681C49884203D1052007F0C7
:10A9E000F7FD2EE0174800681849884229D015481D
:10A9F00000681749884224D11648F9F703FC164924
:10AA0000098888421DD96A237F2218210020FDF77A
:10AA10003DF9104B1B2208211048FFF787FE0D4817
:10AA20000D4A128881180D48FFF795FE04462CB197
:10AA30000948008820440849088002E000200649AF
:10AA4000088010BD400000202A04F4002A04EC0015
:10AA50002A04BC004A22002008020020D221002043
:10AA600038B50446002C2DD00020174908804FF43B
:10AA7000C8711648F9F791FBFDF7AEF8012114A053
:10AA800005F0FAFD114803F0DFFB104B1B220821F3
:10AA90001248FFF74BFE0D480B4A128881180F48E9
:10AAA000FFF759FE0849088001236E229F210020EC
:10AAB000FDF74AF90020012309A272210090FDF759
:10AAC0007DFB38BD00BFFCE7080200204A220020C1
:10AAD000CFFBCFA2D4C4B6C100000000D221002019
:10AAE0005BCFC25DB7ADD2B3205B455849545DB76B
:10AAF000B5BBD80010B51148408810B11048FFF719
:10AB000063F8104800681049084420B1012806D0B5
:10AB100002280FD10AE0022007F05AFD0BE0074897
:10AB2000408810B1092007F053FD04E0082007F029
:10AB30004FFD00E000BF00BF10BD0000A8210020B5
:10AB4000C024002040000020D6FB0BFF10B5294C8C
:10AB50002948007800B910BD48E040F21E21A01C31
:10AB600001F068F820802088002835DD234800782F
:10AB700018B923480078012800DD37E00022A11C25
:10AB8000104606F0EBFA00201E490872A0782B2828
:10AB900002D0A0785E2809D1A01C02F0D5F90128C6
:10ABA00000D123E0A01CFAF779F814E0A07824285B
:10ABB00011D1607952280ED1E07943280BD1218838
:10ABC00004F109000BF0B2FD0F48007820F00100FD
:10ABD000401C0D49087009E02088002805DA012290
:10ABE0000AA1002006F0BAFA00E000E0B5E700BFD5
:10ABF00000BFB0E76A0E0020FF020020F002002034
:10AC0000350100205C080020281F00205175657563
:10AC1000654631002DE9F041B0B0002600274348D9
:10AC200090F8DD01C0EB4011414800EB41043F4882
:10AC300090F8DD01C0EB40113D4800EB410000F110
:10AC40001F05DFF8F0803CA2642117A809F006FC7C
:10AC5000207808B1287820B93AA117A8F9F7A8FAFE
:10AC600019E0334B1F3B3BA2502103A8CDE900451F
:10AC700009F0F4FB03A800F0BDFD2D4B1F3B3CA2E7
:10AC8000502103A8CDE9004509F0E8FB03A917A866
:10AC9000F9F78EFA0126012217A9002006F05EFAC4
:10ACA000002E40D035A2642117A809F0D7FB1F4819
:10ACB00090F89B0000B3012802D0022821D104E0C3
:10ACC00031A117A8F9F774FA00BF30A117A8F9F756
:10ACD0006FFA1648CDE9004590F89B302DA250211F
:10ACE00003A809F0BBFB03A800F084FD002203A920
:10ACF000104606F033FA09E02CA117A8F9F758FA24
:10AD000004E02CA117A8F9F753FA00BF00BF0122F5
:10AD100017A9002006F022FA00BF00BF012228A1D7
:10AD2000002006F01BFA30B0BDE8F081DE1B0020E9
:10AD3000DC1D00206A0E0020416363657373703A66
:10AD400000000000756E737570706F72742D456D24
:10AD50007074790041542B435354543D222573227F
:10AD60002C222573222C222573220D0A00000000BC
:10AD700025732C25732C2573000000004155544881
:10AD80002D4C4F47494E3A005041500043484150E6
:10AD90000000000041542B4347415554483D312C9D
:10ADA00025642C25732C25730D0A00004E4F4E454B
:10ADB0000000000020446F206E6F7468696E6700A9
:10ADC000417574684C6F67696E20446F6E65000052
:10ADD00010B586B004461522E11D2748F9F7C4F9DD
:10ADE000002025490875084600798DF814000846AA
:10ADF00040798DF8150000208DF8160005A8F9F7A8
:10AE000073FA0C2829D2DFE800F01106121D13286E
:10AE100007141E08281F00BF00BF02201749087032
:10AE200017A21421684609F019FB1CE000BF00BFFF
:10AE300000BF01201149087015A21421684609F0CD
:10AE40000DFB10E000BF00BF00200C49087014A2E9
:10AE50001421684609F002FB05E015A2142168469A
:10AE600009F0FCFA00BF00BF6A46034914A009F0CC
:10AE7000E5FA06B010BD0000AB100020FD02002076
:10AE80004348494E415F554E49434F4D5D000000D8
:10AE90004348494E415F4D4F42494C455D000000DB
:10AEA0004348494E415F54454C45434F4D5D00007A
:10AEB000554E4B4E4F572D49434349445D000000CA
:10AEC00049434349443A25732025730D0A00000085
:10AED00010B586B00446204603F0F6F904F10800E8
:10AEE000F9F702FA80B2ADF8100004F10B00F9F79F
:10AEF000FBF9C0B28DF8120004F10E00F9F7F4F975
:10AF0000C0B28DF8130004F11100F9F7EDF9C0B2E9
:10AF10008DF8140004F11400F9F7E6F9C0B28DF8C9
:10AF2000150004F11700F9F7DFF9C0B28DF816002B
:10AF3000DDE9040102F0AAFF9DF816009DF8151046
:10AF40009DF81420CDE9002102909DF813309DF862
:10AF50001220BDF8101002A009F070FA06B010BD62
:10AF60000D0A4E657754696D653A253032642D259A
:10AF70003032642D2530326420253032643A253059
:10AF800032643A253032640D0A000000F0B585B015
:10AF90000446FE4EB51C0027FD480078102819D243
:10AFA000DFE800F008A827F4F318CBF2F9F0DA7222
:10AFB00061EF8319012C0BD10122F6A1002006F0CC
:10AFC000CDF8F8A000F016FC0F200AF065FE01E0B5
:10AFD0004FF0FF377EE3012C07D10122F3A10020BF
:10AFE00006F0BCF8E81D01F05DFF02200AF054FEF7
:10AFF00070E3012C18D0F1480078401CEF4908702C
:10B0000008460078012803D102200AF045FE61E3DA
:10B01000EA48007802281FD1E94908700122E9A115
:10B02000002006F09BF817E0E448007830B90020D3
:10B03000E3490870E7A000F0DDFB08E0DF48007896
:10B04000012804D1DE490870E6A000F0D3FBDC48FB
:10B05000017828460AF060FD0020D84908700C20CD
:10B060000AF01AFE36E3012C05D00122E0A10020EF
:10B0700006F074F804E00122E2A1002006F06EF868
:10B0800001200AF009FE25E3012C05D00122E1A1EF
:10B09000002006F063F804E00122E2A1002006F09F
:10B0A0005DF80E200AF0F8FD14E3012C05D0012212
:10B0B000E0A1002006F052F818E00122E2A10020F1
:10B0C00006F04CF8687A302807D10120E34981F86E
:10B0D0006F02E3A009F0B2F908E0687A312805D1DF
:10B0E000E3A000F087FBE6A009F0A8F901200AF030
:10B0F000D3FDEFE2012C05D00122E6A1002006F0ED
:10B100002DF802E028460AF0A7FC64200CF005FEAA
:10B110000120FDF7BBF832200CF0FFFDE24800688B
:10B1200000F068FB32200CF0F8FDE048006800F009
:10B1300061FB06200AF0B0FDCCE2012C05D0012213
:10B14000DBA1002006F00AF802E02846FFF740FEE7
:10B150000A200AF0A1FDBDE2012C05D00122D8A1F0
:10B16000002005F0FBFF05E005F10A00F9F7BCF847
:10B17000D84908709248007848B908200AF08CFD38
:10B1800008E089E018E006E091E2D5E0C5E009209A
:10B190000AF082FD9EE2012C05D00122CEA1002002
:10B1A00005F0DCFF04E00122CFA1002005F0D6FF6E
:10B1B00009200AF071FD8DE2012C05D00122CDA1FC
:10B1C000002005F0CBFF26E0022004F015FDA81DAD
:10B1D000F9F78AF80A2190FBF1F0CA4991F8321385
:10B1E000884213D0C74890F8320300EB8000430038
:10B1F000C5A21421684609F031F9C24890F832130B
:10B20000C5A009F01BF9684600F0F4FA0122C6A1B6
:10B21000002005F0A3FF0CF019FD00F5FA70C549F8
:10B2200008606748007801282AD10020C2490860D8
:10B23000B44981F8F802084690F83233BFA21421CD
:10B24000684609F00BF9684600F0D4FA012006F0D0
:10B2500057F8AC4890F8F70218B9BDA000F0CAFA48
:10B260000AE0A84890F83233BEA21421684609F0DB
:10B27000F5F8684600F0BEFA04200AF00DFD02E081
:10B280000D200AF009FDBC48007820B905F0CAFF7E
:10B290000120B94908701DE2012C05D00122B7A197
:10B2A000002005F05BFF24E0A8794E280ED1A248CB
:10B2B0000068C8B9B6A000F09DFAB9A000F09AFAEB
:10B2C0009D480168BDA009F0B9F80DE09A480068F2
:10B2D00050B1BEA000F08EFAC0A000F08BFA9648E4
:10B2E0000168C5A009F0AAF80122C7A1002005F055
:10B2F00035FF9148006810B1C6A000F07BFA3048D5
:10B30000007818B903200AF0C7FC02E004200AF014
:10B31000C3FC1120C3490870DCE1012C05D00122D7
:10B32000C1A1002005F01AFF02E028460AF0D4FB74
:10B3300004200AF0B1FCCDE1BF48007810B101282B
:10B3400022D18CE1012C06D0B648007800F0100024
:10B35000B449087000E091E15E48007808B9012026
:10B3600000E000205B49087008460378B3A214216E
:10B37000684609F073F8684600F03CFA64200CF067
:10B38000CCFC6FF0020763E18FE100006A0E002041
:10B390000C0300204D6F64656D53746172742E2E22
:10B3A0002E000000415445300D0A0000504F432D3F
:10B3B000417574684F6B2D2D0000000010030020B4
:10B3C0009C000020476574506F635665722066616B
:10B3D000696C000041542B504F433D3035303030C4
:10B3E000300D0A0041542B4C5350413D310D0A00A1
:10B3F000536574545453504152414D206661696CF9
:10B4000000000000536574545453504152414D2084
:10B410004F4B00005345545F4D49434C56206661E5
:10B42000696C00005345545F4D49434C56204F4BC7
:10B4300000000000434845414B5F484541445345A7
:10B4400054206661696C0000434845414B5F4845A4
:10B450004144534554204F4B000000005C0800203D
:10B46000B6FABBFABDD3C8EB2D2D2D2D2D0D0A003C
:10B4700041542B41554443483D302C300D0A0000C7
:10B48000B6FABBFACEB4BDD3C8EB2D2D2D2D0D0AC7
:10B49000000000004765744D6F64656D4D6F647505
:10B4A0006C65206661696C0014030020180300209D
:10B4B0004765744943434944206661696C00000054
:10B4C00047657453494D53656C65637420666169C3
:10B4D0006C00000004030020536574546F6E6573A4
:10B4E000206661696C000000536574546F6E65736B
:10B4F0005F4F6B005265616453706B4C76206661E0
:10B50000696C0000DE1B002041542B434C564C3D1F
:10B5100025640D0A00000000566F6C756D4C763D79
:10B5200025640D0A0000000053657453504B6C767F
:10B53000204F4B0008030020B400002041542B5042
:10B540004F433D747473766F6C3D25640D0A0000A3
:10B5500041542B504F433D746F6E65766F6C3D3098
:10B560000D0A000041542B504F433D746F6E6576B9
:10B570006F6C3D25640D0A001C030020476574476D
:10B580005053737461747565206661696C000000C6
:10B5900041542B4750533D224F4646220D0A00008E
:10B5A00041542B5649424354524C3D22504F57452B
:10B5B00052222C224F4646220D0A0000636C6F7304
:10B5C00065204750532D2D25640D0A0041542B470B
:10B5D00050533D224F4E220D0A00000041542B567D
:10B5E00049424354524C3D22504F574552222C223F
:10B5F0004F4E220D0A0000006F70656E20475053B9
:10B600002D2D25640D0A0000536574696E6720476F
:10B610005053000041542B475053414E543D310D7F
:10B620000A00000003030020476574506F63436FF6
:10B630006465206661696C000203002041542B534D
:10B64000494D43524F53533D25640D0A00000000FD
:10B65000012022490870224981F8620225E0002079
:10B660001E490870012C08D01E48007800F0010027
:10B670001C4908706FF0010717E000BF01221AA1F2
:10B68000002005F06BFD01201549887019480078ED
:10B6900030B919A000F0AEF807200AF0FDFA03E077
:10B6A0001AA000F0A7F8012700BF00BF12E0012C8C
:10B6B00005D001221AA1002005F050FD03E03188D9
:10B6C000284600F0ABF8FFF7A5FA19A000F092F8B1
:10B6D000012700BF00BF384605B0F0BD02030020BF
:10B6E0005C080020030300204361726420526561FE
:10B6F000647900009C00002041542B504F433D31A1
:10B70000303030303032300D0A00000041542B50C0
:10B710004F433D6F70656E2C312C310D0A000000D7
:10B72000476574506F6350617261206661696C0097
:10B7300041542B504F433D3033303030300D0A00F0
:10B7400010B51148007810B11048007800B110BD54
:10B750000F48007818B9012003F06CFE12E00C4885
:10B76000C078002803DD032003F064FE0AE00848E7
:10B770004079002803DD042003F05CFE02E0022093
:10B7800003F058FE00BFE2E7FE020020F0020020B6
:10B790005C08002008B501211C2002F085FA102069
:10B7A0008DF8030002208DF802008003ADF8000040
:10B7B00069460E48FAF792FE4FF48040ADF800005B
:10B7C00069460A48FAF78AFE4FF48070ADF8000027
:10B7D00069460748FAF782FE4FF480700449143135
:10B7E0000860C0010149486108BD00000010014027
:10B7F0000008014070B504462046F8F703FD85B205
:10B800002946204608F0FEFA70BD70B504460D4684
:10B810002946204608F0F6FA70BD00002DE9F04FE9
:10B82000A3B004460D460026B046B146B2460127F5
:10B830000021E81E2154214604F10D00F9F7CBF94F
:10B8400005460020605519AA74A12046FBF740FE6A
:10B8500005467348D0F81D3072A26421684608F08E
:10B86000FDFD19A96846F8F7D4FC00B1012619AA14
:10B870006DA12046FBF72CFE05466C4B6CA26421A3
:10B88000684608F0EBFD19A96846F8F7C2FC08B154
:10B890004FF00109674890F89C0005282FD2DFE897
:10B8A00000F003040607050000BF00BF27E000BF4B
:10B8B000604890F89C00022806D15F4B5CA264218E
:10B8C000684608F0CBFD0BE05A4890F89C0003282E
:10B8D00006D1594B283356A26421684608F0BEFDB4
:10B8E00019AA56A12046FBF7F3FD054619A968469B
:10B8F000F8F78FFC08B14FF0010A002700BF00BF26
:10B90000AFB119AA4FA12046FBF7E2FD05460AF0A8
:10B91000B7F883465B4646A26421684608F09EFD60
:10B9200019A96846F8F775FC08B14FF0010886B907
:10B93000B8F1000F0DD1B9F1000F0AD1BAF1000F23
:10B9400007D1012240A1002005F008FC23B0BDE88A
:10B95000F08F40A0FFF74EFF76B13148D0F81D3090
:10B9600040A2282119A808F079FD694619A8F9F71D
:10B97000C8F86846FFF73EFF7FB10AF081F88346BA
:10B980005B463AA2282119A808F068FD694619A863
:10B99000F9F7B7F86846FFF72DFF244B35A22821A9
:10B9A00019A808F05BFD694619A8F9F7AAF86846D6
:10B9B000FFF720FF1F4890F89C00022806D11E4B7D
:10B9C0002EA2282119A808F049FD15E0194890F881
:10B9D0009C00032807D1184B283328A2282119A836
:10B9E00008F03CFD08E028A2282119A808F036FD3F
:10B9F000694619A8F9F785F8694619A8F9F781F891
:10BA00006846FFF7F7FE23A0FFF7F4FE012222A10C
:10BA1000002005F0A3FB00BF98E700006964000068
:10BA20009C1B0020256C750070776400CE1B0020E5
:10BA300025730000DE1B00206B1D0020646F6D610C
:10BA4000696E000069700000504F43207374696C88
:10BA50006C00000041542B504F433D3031303030AA
:10BA60003000000069643D256C753B0069703D2520
:10BA7000733B00007077643D25733B00646F6D611C
:10BA8000696E3D25733B0000646F6D61696E3D3BDF
:10BA9000000000000D0A00005273745F504F4350C5
:10BAA0006172610070B58AB0064626B1012E05D0DC
:10BAB000022E09D105E00524192507E005243725C4
:10BAC00004E00524052501E00AB070BD00BF23464F
:10BAD00007A21E2102A8009508F0C0FC02A8FFF7EB
:10BAE00089FE002202A9104605F038FB00BFEBE7F3
:10BAF00041542B5544503D25642C25640D0A00000B
:10BB000030B502460B461946144607E008782578FA
:10BB1000A84201D0012030BD491C641C08780028CF
:10BB2000F4D100BFF7E700002DE9F04705460027F4
:10BB300033480468002640F23338DFF8C8904FF4E9
:10BB4000807031490860002C00DA55E02F484068C9
:10BB5000A04200D850E015B100200BF013FE06EB18
:10BB6000080104EB440000EBC4022848083000EB55
:10BB70008200406A81420AD904EB440000EBC40110
:10BB80002248083000EB8100406A871B00E04746EE
:10BB9000FCF7A6FC04EB440101EBC4021B4908318D
:10BBA00001EB82000021F9F7CDFA04EB440101EB2F
:10BBB000C4021649083101EB82004B463A46314631
:10BBC00000F026F804EB440101EBC4020F490831F0
:10BBD00001EB820008F074F904EB440101EBC402AC
:10BBE0000A49083101EB82000121F9F7ABFA15B1DE
:10BBF00001200BF0C7FD00BF3846BDE8F08700000C
:10BC0000A8000020DE1B0020100C0140FC2A0020B0
:10BC10002DE9F04180460C4615461E46044827187B
:10BC2000AAB2394630460BF0F3FCBDE8F0810000C3
:10BC300000F01F00F8B505460B462B49888808B967
:10BC40000020F8BD4F88881D30F82700ADF80000AF
:10BC50004F88881D00EB87004088ADF80200002463
:10BC6000002220E0B1F8D00000B920E0CE31D1F8B8
:10BC70000A00CF88C65DC888401CC880C88831F8D3
:10BC8000CE79B84202DB0020A1F8D400B1F8D00090
:10BC9000401EA1F8D0009C4203DA2046671CBCB2CB
:10BCA0002E54501C82B2BDF800009042DADC00BF76
:10BCB0004888401C48804888322801DB00204880A2
:10BCC0008888401E8880BDF80000904202D06FF046
:10BCD0000100B6E7BDF80000984202DD4FF0FF30EA
:10BCE000AFE7BDF80000ACE7C01A002030B503464E
:10BCF0000A4612480024048084804480002108E021
:10BD00000025841D04EB81046580841D24F82150E6
:10BD1000491C3229F4DBC0F8D830002104E00024AB
:10BD2000D0F8D8506C54491C9142F8DB20F8CE2F43
:10BD300000248480C4804480CE3830BDC01A0020E6
:10BD400070B504460A4622498888322802DB4FF043
:10BD5000FF3070BDB1F8D0001044B1F8CE50A84209
:10BD600002DD6FF00100F4E7B1F8D2500E88881DB3
:10BD700000EB860045800D88881D20F825200023D3
:10BD800017E0E05CD231D1F806500E88A85508883B
:10BD9000401C088031F8D209B0F5206F02DB00208A
:10BDA000A1F8D200B1F8D000401CA1F8D000581C76
:10BDB00083B29342E5DB0888401C0880088832285B
:10BDC00001DB002008808888401C88800020C0E7B4
:10BDD000C01A002000B54FF420610248FFF786FF2B
:10BDE00000BD0000C01000207047000070B50021A9
:10BDF00000230F22C47804B3154C246804F4E064D3
:10BE0000C4F5E064210AC1F10403CA40447804FA8D
:10BE100003F184781440214309010E4C0678A155A2
:10BE2000047804F01F050124AC4005786D11AD00C5
:10BE300005F1E025C5F8004109E0047804F01F058C
:10BE40000124AC40044D0678761145F8264070BDBB
:10BE50000CED00E000E400E080E100E00249014375
:10BE6000024A1160704700000000FA050CED00E086
:10BE70002DE9F04104460D4616461F462580A67062
:10BE800014223946E01CF8F7B1F9E01CF8F7BAF9CA
:10BE90006076607EC006000EA0761020E07600205E
:10BEA0002076BDE8F081000070B50446217EE01CDC
:10BEB000455C164800681649084490B1B0F5601F0B
:10BEC0001ED014490844E8B9392D02DA681CC5B2FD
:10BED00000E03025217EE01C4554204600F01CF88F
:10BEE00010E0217E607E401E814203DA207E401CED
:10BEF000207601E000202076204600F00DF801E0D9
:10BF0000022070BD00BF0020FBE7000040000020C1
:10BF1000D6FB43FF0004C0FF2DE9FC410446A7788F
:10BF200094F81BC06744103FBBB2278894F81AC02E
:10BF30006744BAB2A1782088FBF7A8FE207EC5002E
:10BF400000200090A17820880123E21CFCF736F93C
:10BF50002088284485B22188681AC11700EB5171E6
:10BF6000C1F3C706E01C805D8DF8040000208DF849
:10BF7000050001200090A178034601AA2846FCF79D
:10BF80001DF9BDE8FC8100000EB50121092001F07A
:10BF90008BFE04208DF8030003208DF8020008209A
:10BFA000ADF8000069460B48FAF798FA0321012022
:10BFB000FAF774FA0820019000208DF80800082094
:10BFC0008DF8090001208DF80A0001A8F9F7D0FCCE
:10BFD0000EBD0000000C014010B51048FFF764FFD3
:10BFE0000F4800680F49884216D106220E490B48B7
:10BFF000C01CF8F71CF918B9122006F0E9FA0BE09A
:10C000000AA004F009FC32200BF087FE01200A4947
:10C010000871062006F0DCFA10BD0000DA230020CB
:10C02000400000202A04EC00A1000020C3DCC2EB89
:10C03000B4EDCEF3000000004A030020F0B5A7B035
:10C0400000272D48FDF700FD06462C48864203D107
:10C05000062006F0BDFA4DE0294886424AD126481E
:10C0600084792848007818B1022C01DBA01CC4B2E6
:10C07000254890F89C00A04239D0234880F89C4085
:10C0800022A004F0C9FB0020FFF74EFD09F0B6FC2A
:10C0900009F0F6FC054609F097FC074619480078B8
:10C0A00038B92B461CA232211AA8009708F0D6F9FD
:10C0B00008E01E480095D0F81D301DA232211AA8B4
:10C0C00008F0CCF901A91AA8F8F71BFD1CA0FFF78E
:10C0D00091FB01A8FFF78EFB1DA0FFF78BFBFCF780
:10C0E000FFF914200BF019FE1AA0FFF783FB0120C3
:10C0F00006F06EFA27B0F0BDC02400202A00FC0034
:10C100002A04EC009C000020DE1B0020C5E4D6C3FE
:10C11000CDEAB3C90000000069703D25733B646F30
:10C120006D61696E3D25733B000000009C1B002083
:10C1300069643D256C643B69703D25733B000000DC
:10C1400041542B504F433D303130303030000000EF
:10C150000D0A000041542B504F433D3034303030F5
:10C16000300D0A007047000001460868034A126853
:10C17000904201D8012070470020FCE71C040020F9
:10C18000024B1B6813440B60704700001C04002026
:10C1900002490968491C014A116070471C040020CB
:10C1A00010B5024600200C4B186820F00300104325
:10C1B00018600A4B1B6843F00403084C23600129F4
:10C1C00001D130BF00E020BF044B1B6823F0040303
:10C1D000024C236010BD00000070004010ED00E034
:10C1E0002DE9F84F05460C4616461F46802D01DA0C
:10C1F000802C01DBBDE8F88FA819802802DDC5F18D
:10C200007F0086B2E019802802DDC4F17F0087B28A
:10C21000FCF766F90A984FEA8009194B13F80920D0
:10C220009C4609F101031CF803105B1C1CF8030079
:10C2300001F0DCFD8246E019401E83B2A819401EC1
:10C2400082B221462846FDF711F84FF0000813E0AE
:10C2500004EB080000904FF0000B09E04FEA2A20A1
:10C26000FDF7F8F90AF0FF00FDF7F4F90BF1010B07
:10C27000B345F3DB08F10108B845E9DB00BFB9E7D6
:10C28000FC2600202DE9FF4F95B0239C229800F05A
:10C29000F0001090229800F00F000F904FF0000B6C
:10C2A000179848BB109840B94FF008090C254FF07B
:10C2B000010A7E4FDFF8F88107E04FF008091025EA
:10C2C0004FF0010A7B4FDFF8F0810BE098F8001087
:10C2D0001898814200D109E008F101080BF1010032
:10C2E0001FFA80FB98F800000028EFD100BF0BFB7D
:10C2F0000AF000FB057728E0109898B94FF0100974
:10C300000C254FF0020A01AF4FF000084FF0000B70
:10C3100001AA109BDDE91701FAF764FD182814D073
:10C32000664F12E04FF0100910254FF0020A07AFD8
:10C330004FF000084FF0000B07AA109BDDE9170132
:10C34000FAF750FD202800D05C4F1698284480282A
:10C3500002DD19B0BDE8F08F15984844802800DD53
:10C36000F7E716982844401E83B215984844401EAB
:10C3700082B2DDE91501FCF779FF002013908EE011
:10C3800013991698084486B2002014907FE0DDE9E6
:10C39000140101EBC00080B2129017F8010B11904C
:10C3A0004FF0000B6CE0802040FA0BF01199084030
:10C3B00080B30D2E0ADA24B94148007807F04AFE0E
:10C3C0005AE04048007807F045FE55E01B2E0ADA97
:10C3D00024B93B48007807F03DFE4DE03A4800782C
:10C3E00007F038FE48E06E2E09DA1CB9002007F08D
:10C3F00031FE41E03248007807F02CFE3CE024B9E1
:10C400003148007807F026FE36E02D48007807F026
:10C4100021FE31E0FFE70D2E0ADA24B92948007821
:10C4200007F018FE28E02648007807F013FE23E006
:10C430001B2E0ADA24B92448007807F00BFE1BE013
:10C440002048007807F006FE16E06E2E0ADA24B9BE
:10C450001B48007807F0FEFD0EE01C48007807F04E
:10C46000F9FD09E024B91648007807F0F3FD03E070
:10C470001548007807F0EEFD0BF101001FFA80FB74
:10C48000BBF1080F8FDB1498401C80B214901498F5
:10C490005045FFF67CAF1398401C80B21390139860
:10C4A000A842FFF66DAF00BF53E70000648B0108A0
:10C4B000088B0108947F0108347F010884850108F6
:10C4C0001204002011040020100400201304002096
:10C4D0002DE9F04F87B0894616469A46109F0025F1
:10C4E00033E009EB0500059005FB06F006900024FB
:10C4F00028E004EB4400385C039004EB4400401C4B
:10C50000385C049004EB4400801C17F800B04FEA3C
:10C51000EB0002900498801001900398C0100090E6
:10C520000298C102019801EB4011009808441FFADB
:10C5300080F84FEA2820FDF78DF808F0FF00FDF79E
:10C5400089F8641CB442D4DB6D1C5545C9DB07B0C7
:10C55000BDE8F08F2DE9F04FDFB082464FF00008C4
:10C560000020189017905022FB4903A8F7F7FCFD14
:10C5700000BF4046411C0FFA81F803A951F8200082
:10C5800000780028F5D1A8F101000FFA80F8002604
:10C5900023E003A850F826900AF1030B00205D90D9
:10C5A0005E9010E099F800009BF80010884202D0DD
:10C5B00001205D900BE009F101090BF1010B5E9880
:10C5C000401C00B25E9099F800000028EAD100BF3C
:10C5D0005D9800B903E0701C06B24645D9DB00BF88
:10C5E000464502D15FB0BDE8F08F132E7DD2DFE863
:10C5F00006F00A192797ABFEFDFCFBFAF9F8F7F6EF
:10C60000F5F4F3F2F1000122D4A1002004F0A6FD1C
:10C61000092002F03FFF0220F8F7E4FE0120D24992
:10C620000870A5E30122D1A1002004F097FD0920A4
:10C6300002F030FFFAF734F80120F8F7D3FE97E361
:10C6400037AACDA15046FAF743FF0446012C01DB7F
:10C65000282C05DB0122C9A1002004F07FFD87E31F
:10C6600037A92DA8F7F7F0FD37AACAA15046FAF767
:10C670002FFF04460CB900270BE0052C05DD012235
:10C68000C6A1002004F06AFD72E337A8F7F72CFE7C
:10C6900087B237AAC8A15046FAF71AFF0446012C00
:10C6A00001DB0A2C05DD0122C4A1002004F056FDA7
:10C6B0005EE337A8F7F725FE0546C748D0F81D000A
:10C6C000A84204D0C448C0F81D5001201890C348A7
:10C6D00090F89C00042805D00420C04981F89C00F3
:10C6E000012017902DA9BE4800E040E3F7F791FD27
:10C6F00028B12DA9BA48F7F7A7FD01201790B64831
:10C70000D0F81D00B64BB7A29621CDE9007037A82E
:10C7100007F0A4FE012237A9002004F01FFD27E343
:10C7200009F0AEF9B7490290CDE90010AA48D0F857
:10C730001D30B5A2962137A807F090FE012237A937
:10C74000002004F00BFD13E337AA8BA15046FAF743
:10C75000BFFE0446012C01DB282C05DB0122BAA117
:10C76000002004F0FBFC03E337A92DA8F7F76CFDCC
:10C7700037AA88A15046FAF7ABFE04460CB9002749
:10C780000BE0052C05DD0122B5A1002004F0E6FC3C
:10C79000EEE237A8F7F7A8FD87B2904890F89C0022
:10C7A000042805D004208D4981F89C0001201790B1
:10C7B0002DA98B482830F7F72CFD20B98748B0F811
:10C7C0002D03B84218D02DA985482830F7F73CFD35
:10C7D00082480DE09EE28FE23BE22AE211E202E2B1
:10C7E000F4E1E2E1D5E1C7E15FE051E026E014E0E9
:10C7F000A0F82D73012017907848B0F82D03784BDE
:10C8000028339EA29621009037A807F027FE012228
:10C8100037A9002004F0A2FCAAE27048B0F82D036A
:10C820006F4B28339BA29621009037A807F016FE85
:10C83000012237A9002004F091FC99E237AA9BA1BC
:10C840005046FAF745FE0446002C01DB1E2C05DDA0
:10C85000012298A1002004F081FCC3E624B9002144
:10C860005E4880F8DF1104E037A95D48A230F7F791
:10C87000EBFC5B4BA23397A2962137A807F0EEFDA5
:10C88000012237A9002004F069FC012017906FE213
:10C89000534BA23394A2962137A807F0DFFD012263
:10C8A00037A9002004F05AFC62E237AA93A150464F
:10C8B000FAF70EFE0446012C01DB1E2C05DD0122D9
:10C8C00090A1002004F04AFC8CE637A923A8F7F7D2
:10C8D000BBFC37AA93A15046FAF7FAFD0446012C97
:10C8E00001DB1E2C05DD012291A1002004F036FCA5
:10C8F00078E637A919A8F7F7A7FC19A823AB94A2E3
:10C900009621009037A807F0A9FD012237A9002041
:10C9100004F024FC96480068002800DA28E29549D3
:10C9200023A8F7F776FC30B992491F3119A8F7F719
:10C9300070FC00B91CE223A98E48F7F785FC19A901
:10C940008C481F30F7F780FC0320244981F8DD0173
:10C95000012017900CE20000947E010847542B54EC
:10C960004D3A4F4B00000000DA02002047542B5490
:10C97000473A4F4B000000004950000047542B53EA
:10C980004D503A4641494C5B495020496E76616CA6
:10C9900069645D00506F72740000000047542B53AF
:10C9A0004D503A4641494C5B506F727420496E7647
:10C9B000616C69645D00000050534E0047542B5376
:10C9C0004D503A4641494C5B50534E20496E76617A
:10C9D0006C69645D000000009C1B0020DE1B0020D1
:10C9E0001B1D002047542B534D503A49503D257391
:10C9F0003B506F72743D25753B50534E3D256C7511
:10CA00003B000000CE1B002047542B524D503A50A3
:10CA1000534E3D256C753B4D4549443D25733B4385
:10CA20004E554D3D303030303030303030303B5569
:10CA3000494D49443D303030303030303030303B7B
:10CA400049503D25733B000047542B5347503A460D
:10CA500041494C5B495020496E76616C69645D00C8
:10CA600047542B5347503A4641494C5B506F7274C0
:10CA700020496E76616C69645D00000047542B5359
:10CA800047503A49503D25733B506F72743D2575B0
:10CA90003B00000047542B5247503A49503D257304
:10CAA0003B504F52543D25643B0000004163636599
:10CAB0007373700047542B534143433A4641494CEA
:10CAC0005B4163636573737020496E76616C696462
:10CAD0005D00000047542B534143433A4163636573
:10CAE0007373703D25733B0047542B524143433AC7
:10CAF000416363657373703D25733B004163636FEE
:10CB0000756E740047542B41504E3A4641494C5B78
:10CB10004163636F756E7420496E76616C69645D04
:10CB20000000000050617373776F726400000000B2
:10CB300047542B41504E3A4641494C5B5061737308
:10CB4000776F726420496E76616C69645D000000E5
:10CB500047542B41504E3A4163636F756E743D25C7
:10CB6000733B50617373776F72643D25733B0000B4
:10CB7000A8000020961E0020834BA3F11F0283A172
:10CB800037A807F07FFC012237A9002004F0E6FA5D
:10CB9000EEE064224FF4601137A80AF0C3FC0122D2
:10CBA00037A9002004F0DAFAE2E08048B0F82F005C
:10CBB0007E4B21337EA29621009037A807F04EFCD1
:10CBC000012237A9002004F0C9FAD1E07C487DA2F7
:10CBD0009621036837A807F041FC012237A90020FD
:10CBE00004F0BCFA00BF01227AA1002004F0B6FADA
:10CBF0004FF480707C49086001207C4981F8620212
:10CC0000B6E07B48007850B901207949087004F0FB
:10CC10008DFB012277A1002004F0A0FA08E004F0C7
:10CC200079FB002072490870012275A104F096FA80
:10CC30009EE05E48D0F81D00754B76A296210090CC
:10CC400037A807F00BFC012237A9002004F086FA70
:10CC50008EE037AA75A15046FAF73AFC0446282C14
:10CC600005DD012273A1002004F078FABAE47548CA
:10CC700090F89C00022805D00220724981F89C009F
:10CC80000120179028216248F7F787FA37A96048F2
:10CC9000F7F7DAFA37AAAFF2E0215046FAF718FCB4
:10CCA0000446012C01DB0A2C06DD0122AFF2F4213F
:10CCB000002004F053FA5BE037A8F7F722FB0546A3
:10CCC0003A48D0F81D00A84204D03848C0F81D509A
:10CCD000012018903548D0F81D004D4B5AA29621DE
:10CCE000009037A807F0BAFB01201790012237A95E
:10CCF000002004F033FA3BE02C48D0F81D3058A255
:10CD0000962137A807F0AAFB012237A9002004F0DA
:10CD100025FA2DE037AAAFF260315046FAF7D8FB7A
:10CD20000446012C01DB0A2C05DD012251A1002063
:10CD300004F014FA1CE037A8F7F7E3FA05461B489D
:10CD4000D0F81D00A84204D01848C0F81D5001209A
:10CD500018901648D0F81D304DA2962137A807F03C
:10CD60007DFB012237A9002004F0F8F900E000BFA4
:10CD700000BF189808B101F065FC179810B10020A9
:10CD8000FEF7D2FE00BF2DE4B51E002047542B5203
:10CD900041504E3A4163636F756E743D25733B504D
:10CDA000617373776F72643D25733B009C1B002099
:10CDB00047542B5645523A25735F562564000000B0
:10CDC000EC01002047542B4241543A202564205660
:10CDD00000000000676F746F204D6F64656D5570C3
:10CDE0006461746500000000100801405C080020C8
:10CDF000F3020020656E61626C652073706B000049
:10CE0000646973656E61626C652073706B0000000D
:10CE10006B1D002047542B52444F4D41494E3A253B
:10CE2000733B50534E3D256C753B000053444F4DB2
:10CE300041494E004D41494E4950204C454E2045F8
:10CE400052520000DE1B002047542B53444F4D41EB
:10CE5000494E3D25733B50534E3D256C753B0000BC
:10CE600047542B525049443A50534E3D256C753B24
:10CE70000000000047542B535049443A4641494C66
:10CE80005B50534E20496E76616C69645D00000012
:10CE900047542B535049443A50534E3D256C753BF3
:10CEA00000000000F0B5C1B00546002778216846B3
:10CEB000F7F773F978211EA8F7F76FF914213CA84A
:10CEC000F7F76BF9284607F0B9FA3CA9284604F0B1
:10CED0006DFA184801680091416801910089ADF828
:10CEE00008000A243CA8F7F78DF9461E23466A4637
:10CEF00031463CA808F0D8FC22461EA96846F7F740
:10CF000019FE1EA807F09AFA78216846F7F745F946
:10CF10001EAB09A27821684607F0A0FA684607F020
:10CF20008DFA0C2000EB44016846FEF76EFC41B020
:10CF3000F0BD0000887D010841542B5341555448F1
:10CF40003D25730D0A0000002DE9F043BBB00446F7
:10CF500048210CA8F7F721F9002560784C2817D153
:10CF6000A078532814D1E078482811D1207954288A
:10CF70000ED1607A45280BD10020F9490871084686
:10CF8000C07808B904F0C6F901203BB0BDE8F083D1
:10CF90006079302804D1A079422801D10120F4E73A
:10CFA0006079542810D1A0794F280DD1E0794E280E
:10CFB00008D1207A452805D104F0B8F914210020C1
:10CFC0000AF08CFE0120E0E76079382857D1A0797B
:10CFD000422854D1E07930280CD1207A312809D167
:10CFE00008F0ACFB0120DE4948710020C870012028
:10CFF000087031E0607A302805D1A07A322802D159
:10D0000004F094F928E0607A302813D1A07A31280E
:10D0100010D104F08BF908F091FB0120FCF7CEF859
:10D020000020D04908800120CD490870C870002038
:10D03000487111E0E07930280ED1207A30280BD1E8
:10D04000607A302808D1A07A302805D10020C44960
:10D05000C870487104F05EF9607A31280DD1A07A69
:10D0600033280AD10120BE4981F8610204F05EF93B
:10D070000A214FF47A7001F025FC012085E76079E0
:10D08000382874D1A0793228FBD1E0798DF87C0062
:10D09000207A8DF87D0000208DF87E001FA8F7F71C
:10D0A00023F900F0FF08B8F1000F09D0B8F1010F23
:10D0B00078D0B8F1020F76D0B8F1030F74D1B2E096
:10D0C0000020A74981F860020870A748007820F086
:10D0D0001000A5490870A5A266211FA807F0BEF997
:10D0E000607C422814D1A07C352811D1607E432871
:10D0F0000ED1A07E41280BD105209E490870012049
:10D10000974981F863029CA11FA8F7F751F850E0F6
:10D11000607C432816D1A07C452813D1607E43282B
:10D1200010D1A07E32280DD18D4890F863020128DD
:10D1300003D002208A4981F8630293A11FA8F7F760
:10D1400037F836E0607C432812D1A07C45280FD107
:10D15000607E43280CD1A07E312809D1052080496A
:10D1600081F863028BA11FA8F7F722F821E063E0A2
:10D17000607C432819D1A07C332816D1607E4228D8
:10D1800013D1A07E372810D1754890F86302042887
:10D1900003D00620724981F8630281A11FA8F7F726
:10D1A00007F806E00BE010E043E080A11FA8F6F7C7
:10D1B000FFFF01221FA9002003F0D0FF39E0012268
:10D1C0007DA1002003F0CAFF33E004F11100F7F75E
:10D1D00019F8801EC7B2242F00DB24273A4604F139
:10D1E00011017848F6F7C0FF00207649C8555C4920
:10D1F0001931744804F0DAF80020607410221EA976
:10D2000004F10900F7F738F85549486101226EA189
:10D21000002003F0A3FF01206E490870032050494D
:10D2200081F8630205E001226BA1002003F096FF64
:10D2300000BF00BF0120A8E6607933281AD1A07989
:10D24000442802D0A079452814D110221EA904F147
:10D250000D00F7F711F84249C1F86802A079452896
:10D2600003D10846B0F86802888101203C4981F862
:10D270006C028AE62046F9F74BFA08B1012084E6F1
:10D280002046F9F733FB08B101207EE660793828A3
:10D2900065D1A079362862D10120314908701E205D
:10D2A00034490870207A302850D104F11100F6F783
:10D2B000A9FF801EC7B2242F00DB24273A4604F1C1
:10D2C000110102A8F6F750FF002002A9C8556074AA
:10D2D00010221EA904F10900F6F7CEFF20490864C8
:10D2E000463102A804F062F81D484078E0B9394898
:10D2F000007838B91A4B46333AA266211FA807F0C6
:10D30000ADF80CE000203349087015484630A0F114
:10D310002D0335A2662100901FA807F09FF81FA9D2
:10D320000320FDF73DF811E03348007801280DD1C6
:10D330000020314908700A4B463330A266211FA8ED
:10D3400007F08CF81FA90320FDF72AF800200549F3
:10D350000880034981F860020120487015E651E019
:10D360005C080020B0000020281F00205B6D736760
:10D370005D000000D8020020D5CBBAC5D0C5CFA231
:10D38000B4EDCEF300000000CEDECDF8C2E7C1ACB4
:10D39000BDD30000CEDEB7A8C1ACBDD300000000F5
:10D3A000C3BBD3D0B7FECEF1000000004E6F206C9F
:10D3B0006F67696E000000006C6F67696E20696EB0
:10D3C00067000000240C00206C6F67696E206F6B93
:10D3D00000000000900000206C6F676F757420697A
:10D3E0006E6700002573000025732CD2D1B5C7C22B
:10D3F000BC2C257300000000D9020020BDF8C8EB4A
:10D400002C257300607938282BD1A079332828D1B6
:10D41000E079302825D1207A302822D104F111007A
:10D4200000F052FF04F11100F6F7ECFE0646242E40
:10D4300001DB242600E0761CFE4904F1110003F014
:10D44000B5FF0020607410221EA904F10900F6F750
:10D4500013FFF8497839C1F89C000020607401205E
:10D4600093E5607938280AD1A079332807D1E0798B
:10D47000302804D1207A312801D1012085E5607956
:10D48000392804D1A079312801D101207DE56079C6
:10D49000302825D1A079452822D1002060743AA9EE
:10D4A00004F10D0003F082FF9DF8E9008DF8E4001F
:10D4B0009DF8EA008DF8E500BDF8E400DD49783913
:10D4C0008881012081F8700008468389DAA26621EC
:10D4D0001FA806F0C3FF01221FA9002003F03EFE93
:10D4E0006079382836D1A079342833D12046FCF72A
:10D4F00043FFD44904F1090003F058FFD149032048
:10D50000FCF74EFF0822D0A104F10900F6F78FFEC8
:10D5100028B90120C749783981F8600218E008224B
:10D52000CCA104F10900F6F782FE28B90020C14918
:10D53000783981F860020BE01022C9A104F10900DA
:10D54000F6F775FE20B90120BA49783981F86002F2
:10D5500001201AE56079312831D1E07930282ED1C7
:10D56000A07B372802D0A07B382828D1C1480021D1
:10D57000016041600172A0F2792054F8131FC0F8D5
:10D5800079126168C0F87D1200F50070216881652C
:10D590006168133CC16504F11F00FCF7EDFE01203A
:10D5A000B549087003F0ACFEB24BB4A266211FA8C7
:10D5B00006F054FF1FA8FEF71DF90120E5E460798D
:10D5C000322815D1A079312812D12046FCF7D4FE9B
:10D5D00004F115010120FCF7E3FE0020607509222B
:10D5E00004F10D01A3480938F6F700FE0120CCE450
:10D5F000A7A12046FEF784FAF0B9E07931280ED1D0
:10D60000A5A0FEF7F7F803F091FEA7A0FEF7F2F849
:10D610000120FBF7D3FD0020A74908800AE0E0794C
:10D62000302807D1A5A0FEF7E5F803F073FEA7A008
:10D63000FEF7E0F80120A8E4A8A12046FEF760FA72
:10D64000F0BB02222C212046FAF764FF0546601940
:10D65000F6F74AFE77497839486103222C212046A3
:10D66000FAF758FF05466019F6F73EFE714978391A
:10D6700048616019F6F7C6FDA0F1020949469CA071
:10D6800006F0DCFE25219D48F6F787FD6019F6F7C8
:10D69000B9FD801E1FFA80F960194946F8F744FB6E
:10D6A0006019F6F7AFFD801E1FFA80F9621949462E
:10D6B000924803F000FF914991A006F0BFFE00E000
:10D6C00006E08E495B485F38F6F7BEFD01205CE45A
:10D6D0008EA12046FEF714FA28B900205549783962
:10D6E0000870012051E48EA12046FEF709FA00BB24
:10D6F00002222C212046FAF70DFF05466019F6F7A5
:10D70000F3FD4C497839C1F86802012081F86C02B8
:10D7100081F87000084648A26621D0F868321FA838
:10D7200006F09CFE01221FA9002003F017FD012036
:10D730002BE47FA12046FEF7E3F900BB04222C2155
:10D740002046FAF7E7FE05466019F6F7CDFD3949A0
:10D750007839C1F86802012081F86C0281F8700004
:10D76000084635A26621D0F868321FA806F076FE7A
:10D7700001221FA9002003F0F1FC012005E470A1A3
:10D780002046FEF7BDF9E8BB01202A497839087028
:10D790004870002081F8600202222C212046FAF70E
:10D7A000B9FE05466019F6F79FFD224978390864ED
:10D7B00003222C212046FAF7ADFE05466019F6F744
:10D7C00021FDA0F10209494649A006F037FE611982
:10D7D00060A006F033FE282102A8F6F7DEFC6019EF
:10D7E000F6F710FD801E1FFA80F960194946F8F718
:10D7F0009BFA6019F6F706FD801E1FFA80F9621980
:10D80000494600E0B6E002A803F055FE002605E018
:10D8100002A8815D53A006F011FE761C02A8F6F75F
:10D82000F1FCB042F4D838A006F008FE02A9014885
:10D8300032389BE0D40800206F6E654C696E653A03
:10D8400025640000E00A002043314439434142315D
:10D8500000000000434443424233463600000000CB
:10D8600042414634424444304233433942394136DE
:10D8700000000000D50A0020D902002041542B509E
:10D880004F433D30393030303025730D0A000000F1
:10D890002B4C5350413A000041542B4C5350413DC6
:10D8A000312C310D0A00000041542B4C5350413DA6
:10D8B000312C320D0A000000B000002041542B4CE6
:10D8C0005350413D312C330D0A00000041542B4C84
:10D8D0005350413D312C340D0A0000002B504F4372
:10D8E0003A6E6C6F67696E737461742C322C000031
:10D8F0006C656E3D3D3D3D25640D0A00240C002005
:10D900002D2D2D2D2D2D25730D0A00002B504F434D
:10D910003A6E6C6F67696E737461742C310000002D
:10D920002B504F433A67726F75706E756D2C000007
:10D930002B504F433A6D656D6265726E756D2C00AC
:10D940002B504F433A6E6375727267726F75702C0D
:10D9500030000000636F6E74656E743D3D3D3D2583
:10D96000730D0A002530327800000000F6F76CFCD9
:10D97000012060E42EA12046FEF7C2F818B901206C
:10D98000304981F8600230A12046FEF7B9F850B95D
:10D9900002222C212046FAF7BDFD05466019F6F754
:10D9A000A3FC284948712BA12046FEF7A9F880BBAB
:10D9B00002222C212046FAF7ADFD05466019F6F744
:10D9C00093FC08B9012036E46019F6F78DFC1D4977
:10D9D000C1F89C0003222C212046FAF79BFD054646
:10D9E0006019F6F70FFC801E1FFA80F9601949468E
:10D9F000F8F79AF96019F6F705FC801E1FFA80F90E
:10DA0000621949460F48783003F055FD01200D4951
:10DA1000C87013A12046FEF773F810B90020094919
:10DA2000C87012A12046FEF76BF8002021E4000028
:10DA30002B504F433A6E6375727267726F75702C1C
:10DA4000320000005C0800202B504F433A70747481
:10DA50002C3100002B504F433A6E73706B2C30000A
:10DA60002B504F433A6E73706B2C31002B504F4349
:10DA70003A6E757365726368616E67656400000075
:10DA800008B501211C2000F00FF910208DF80300CB
:10DA900003208DF802004FF48070ADF80000694655
:10DAA0000448F8F71BFD4FF48070024914310860F8
:10DAB00008BD0000000C014010B51348007800B903
:10DAC00010BD4FF48070114908600120FBF776FB10
:10DAD0004FF400700E4908610EA0FDF78BFE11A2F5
:10DAE00000210846FAF709FB03F014FC32200AF083
:10DAF00014F94FF480700549091D0860800104493C
:10DB0000086100BFFEE70000DB020020100C0140AE
:10DB1000001001404154244D59504F5745524F4633
:10DB2000460D0A004259454259452E626D7000006B
:10DB300010B5114800681149084418B1B0F5002F1C
:10DB400017D112E00EA200210846FAF7D6FA3220C9
:10DB50000AF0E3F84FF480400C49486180110C4909
:10DB600008604020086000BFFEE7012004F030FD9F
:10DB700000BF00BF10BD000040000020D6FB13FF17
:10DB80004259454259452E626D7000000010014017
:10DB9000140C014038B50446012C0BD1FAF71CF8DF
:10DBA00005A002F039FE0020012306A27221009098
:10DBB000FAF704FB38BD0000C8B7C8CFB9D8BBFA24
:10DBC000A3BF00005B455849545DCDCBB3F65B4D18
:10DBD0005DC8B7C8CF00000070B505460E46314697
:10DBE00008A006F02BFC002405E0295D08A006F043
:10DBF00025FC601C84B2B442F7DB07A006F01EFCD3
:10DC000070BD0000446174615B25645D3A0D0A00DB
:10DC100025303278000000000D0A000070B504467F
:10DC20006079002805DA06A006F008FC4FF0FF3006
:10DC300070BD6079255C6079401E60712846F7E709
:10DC4000737461636B20697320656D7074790D0A5C
:10DC50000000000070B504460D466079042804D128
:10DC600005A006F0EBFB012070BD6079401C6071DF
:10DC7000617965540020F7E7737461636B20667502
:10DC80006C6C0D0A0000000029B1064AD2690243FB
:10DC9000044BDA6104E0034AD2698243014BDA6142
:10DCA000704700000010024029B1064A9269024301
:10DCB000044B9A6104E0034A92698243014B9A61E2
:10DCC00070470000001002400348406A40F0807036
:10DCD00001494862704700000010024030B5002141
:10DCE0000022002400232D4D6D6805F00C0121B1A8
:10DCF000042905D0082923D105E0294D056022E03B
:10DD0000274D05601FE0254D6D6805F47012234D09
:10DD10006D6805F48034022505EB92421CB9214D53
:10DD2000554305600BE01D4D6D6805F400351DB1D0
:10DD30001C4D5543056002E0194D5543056002E056
:10DD4000174D056000BF00BF144D6D6805F0F00170
:10DD50000909154D6B5C0568DD4045600F4D6D6828
:10DD600005F4E061090A104D6B5C4568DD40856093
:10DD70000A4D6D6805F46051C90A0B4D6B5C45682E
:10DD8000DD40C560054D6D6805F44041890B074DC8
:10DD90006B5CC568B5FBF3F5056130BD0010024052
:10DDA000001BB700808D5B000000002010000020E9
:10DDB00010B501460022002300204A11012A02D199
:10DDC000094C236806E0022A02D1074C236A01E0CD
:10DDD000054C636A01F01F02012494401C400CB101
:10DDE000012000E0002010BD0010024070B5034685
:10DDF000DC108D10D610E00200EB4510304480B2EC
:10DE000070BD00004FF4FA6004490880012088705A
:10DE1000C870002008714871887170472002002086
:10DE20000E488079401CC0B20C4988713C2813DB35
:10DE30000020887108464079401CC0B248713C28D7
:10DE40000ADB0020487108460079401CC0B2087106
:10DE5000182801DB00200871704700002002002014
:10DE60000949098801800849897881700649C9787B
:10DE7000C170054909790171034949794171024924
:10DE800089798171704700002002002003B5BDF838
:10DE90000000094908809DF8020088709DF8030081
:10DEA000C8709DF8040008719DF8050048719DF840
:10DEB000060088710CBD0000200200201FB5002460
:10DEC00007E03248324941F8240000203149085522
:10DED000641C052CF5DD00241DE001202D490855AA
:10DEE00004EB440000EBC4012B4850F821002A4900
:10DEF000A039096C884202D100202649085504EB5C
:10DF0000440000EBC401244800EB8100401D20497F
:10DF100041F82400641C2048A03890F86602A04212
:10DF2000DBDC1D48A038D0F8680228B91BA01849CE
:10DF300008600020174908550020012318A20D2170
:10DF400000900220FAF73AF91348A038B0F86C00B4
:10DF500000EB8000401C00900F48A03813A20A215B
:10DF6000D0F8683201A806F079FA0020012301AA4E
:10DF70000D2100904420FAF721F906480E4B0022AB
:10DF8000034900900D48FBF789FC1FBDDC0300200E
:10DF9000CC260020DD030020FC080020BFD50000B7
:10DFA000B3C9D4B1D1A1D4F100000000253033644D
:10DFB0002F25303364000000D0030020C02400204F
:10DFC0001FB5002407E03048304941F82400002004
:10DFD0002F490855641C052CF5DD00241CE00120A8
:10DFE0002B49085504EB440000EBC401294850F8C4
:10DFF00021002949096C884202D100202449085592
:10E0000004EB440000EBC401224800EB8100801DBA
:10E010001E4941F82400641C1F4890F86602A04283
:10E02000DDDC1D48D0F8680228B91CA0174908603B
:10E030000020174908550020012319A20D21009046
:10E040000220FAF7BBF81448B0F86C0000EB80002F
:10E05000401C0090104815A20A21D0F8683201A88F
:10E0600006F0FCF90020012301AA0D2100904420B4
:10E07000FAF7A4F80648104B0022044900900F4814
:10E08000FBF70CFC1FBD0000C0030020B4260020DD
:10E09000C1030020D80900205C080020BFD5000083
:10E0A000C8BAD7E9D1A1D4F100000000253033640B
:10E0B0002F25303364000000B4030020C02400206A
:10E0C0002DE9F04704460D4617469846002C02DA23
:10E0D0000020BDE8F08719484068A04201D8002020
:10E0E000F7E7E91904EB440000EBC40213480830D9
:10E0F00000EB8200406A81420AD904EB440000EB45
:10E10000C4010E48083000EB8100406A461B00E065
:10E110003E4604EB440000EBC4010848083000EB25
:10E120008100806A00EB050909F58059B2B24946C1
:10E13000404609F0F7F93046CBE70000FC2A002002
:10E14000F0B505460B461646002700240DE02819B9
:10E1500000F073FA024638467F1C1A544FEA122C1C
:10E1600038467F1C03F800C0A41CB442EFDBF0BDAE
:10E1700070B500240025322226492748FFF7E0FF2A
:10E180002448D0F81D002549884208D32148D0F8FA
:10E190001D100022224B591A72EB020009DA1D48A9
:10E1A000D0F81D101FA006F049F923481949C1F8FD
:10E1B0001D001848B0F82F00672804D067201549C3
:10E1C000A1F82F0001241DA112482130F6F721F8F3
:10E1D00028B11AA10F482130F6F736F80124194862
:10E1E0008078012803DD0020164988700124094841
:10E1F00090F83100012805D10124012500200549AE
:10E2000081F831000CB100F01DFA0DB102F094FF5D
:10E2100070BD00009C1B002000F8010840420F0068
:10E2200000EA56FA50534E20696E76616C69643A82
:10E2300025780D0A00000000BF11A6765A54323628
:10E2400030000000DE1B00207FB504466D461C48F0
:10E25000C2881C4800EB8200006800F110014FF4F6
:10E26000C872204609F05EF91548C288154800EBCF
:10E27000820001680222284609F054F900208DF836
:10E2800001000F48C2880F4800EB8200016802229B
:10E29000284609F0BDF90B481638808870B1094846
:10E2A00016388088401E07491639888008468088BD
:10E2B00020B90846007820F0010008707FBD0000FA
:10E2C000C0240020BE2100200246114607E00D2890
:10E2D00001D00A2802D100230B7003E0491C087802
:10E2E0000028F4D100BF704710B505F03DFB0120B8
:10E2F000014981F8620210BD5C0800202DE9F0415F
:10E3000086B004460F462760002500BF206850F8FD
:10E31000250090F80080B8F1000F00D102E0681CE1
:10E32000C5B2F3E700BF681EC5B2681C20710520A6
:10E3300095FBF0F0E071E079052190FBF1F201FB33
:10E34000120010B1E079401CE071254800682549B1
:10E35000884202D02448007990B12348FFF75EFC40
:10E36000C6B2314621A006F069F8052096FBF0F10F
:10E3700000FB1160A071667100201B49087102E06A
:10E380000020A071607102201A237F220D210090CD
:10E390000020F9F737FD1948007880231A461B2121
:10E3A00000900020FDF71CFF6279216851F82200DF
:10E3B0000D2102F061F9637911A213A102A806F000
:10E3C00061F802AA1B211820F9F797FE002001230B
:10E3D00010A272210090F9F7F1FE06B0BDE8F081BD
:10E3E000400000202A00FC004A03002070756C6C7D
:10E3F0002D2D2D2D25640D0A000000001204002093
:10E4000050616C6163650000257325642E626D7038
:10E41000000000003CCDCBB3F62020C8B7B6A82042
:10E4200020CFC2B7AD3E000070B504461948006861
:10E4300019490844A8B1B0F5001F25D1607918B971
:10E440002079401E607102E06079401E6071A579FC
:10E450006079052190FBF1F0A071204600F01EF8D4
:10E4600015E06079401C607160792179884201DB98
:10E4700000206071A5796079052190FBF1F0A07111
:10E48000204600F00BF802E00248006870BD00BFB3
:10E490000020FBE740000020D6FB43FF10B586B00C
:10E4A000044602201A237F220D2100900020F9F754
:10E4B000A9FC6279216851F822000D2102F0DCF8F4
:10E4C000637906A207A102A805F0DCFF02AA1B21BE
:10E4D0001820F9F712FE06B010BD000050616C6103
:10E4E00063650000257325642E626D7000000000D6
:10E4F00010B50F480078C0F3400000B110BD0D48C2
:10E500000078012803D00B48007802280ED1094872
:10E51000B0F8961108A005F091FF064C083421468A
:10E520000320FBF73DFF00200249087000BFE5E72C
:10E53000A8210020981F00205454535F4C454E3AA8
:10E5400025640D0A0000000021B1028842F040025B
:10E55000028004E002884FF6BF731A4002807047C1
:10E560000246002013890B400BB1012000E000207F
:10E5700070470146888970478181704710B5002235
:10E58000028802F441520B884C8823438C88234331
:10E59000CC8823430C8923434C8923438C89234310
:10E5A000CC8923431A430280838B4FF2FF742340AC
:10E5B00083830B8A038210BD10B5044600BF02217D
:10E5C0000A48FFF7CDFF0028F9D021460748FFF79A
:10E5D000D3FF00BF01210548FFF7C2FF0028F9D093
:10E5E0000248FFF7C6FFC0B210BD00000030014076
:10E5F00001461CE000BF00BF00BF00BF00BF00BF5E
:10E6000000BF00BF00BF00BF00BF00BF00BF00BF12
:10E6100000BF00BF00BF00BF00BF00BF00BF00BF02
:10E6200000BF00BF00BF00BF00BF00BF00BF0A1E89
:10E63000A1F1010399B2DDD1704701460888704706
:10E640007047000010B54FF4807004490860322212
:10E650000349044805F0C0FE10BD0000100C014045
:10E660009C1B002000F8010810B51948FBF7ECF9D5
:10E670000446184884421CD117A002F0CDF81A486D
:10E6800090F8DD011249C98888420ED0104880797F
:10E69000154981F8DD010020FDF746FA01201349F4
:10E6A00081F8620203F094FF10E0062003F090FF6F
:10E6B0000CE0B4F5E02F03D10E2003F089FF05E054
:10E6C0000B48844202D1062003F082FF10BD0000F7
:10E6D000C02400202A00FC00BCB4BDABD6D8C6F4D0
:10E6E000B8FCD0C22E2E2E00DE1B00205C080020BD
:10E6F0002A04EC0038B50446002C3FD020480078AE
:10E70000012809D01FA002F087F8C82009F005FBF6
:10E71000062003F05DFF38BD1D480078012809D1AF
:10E720001CA002F079F8C82009F0F7FA062003F0DF
:10E730004FFFF0E71B4800210160F9F74DFA022175
:10E7400019A001F099FF0120194991F8DD11154A2E
:10E7500050541046174B0022174900901748FBF7FA
:10E760009DF801236E229F210020F9F7EDFA002089
:10E77000012313A272210090F9F720FD00BFCAE720
:10E780000C040020BDFBD6B9D0DEB8C400000000E8
:10E79000D4000020C5E4D6C3CEC4BCFECEDE4150BA
:10E7A0004E00000045010020C9E8D6C341504E008C
:10E7B000DE1B0020EC000020D8000020C024002038
:10E7C0005B4F4B5DC7D0BBBB20202020205B535D3F
:10E7D000CFEAC7E90000000010B51D4800681D49D8
:10E7E000884212D11C480078401C1B49087008461A
:10E7F00000781A490978884202DB0020164908701F
:10E800001548007801F042FD21E0114800681449E4
:10E81000884214D11048007818B9104800780E4981
:10E8200008700D480078002804DD0B480078401E71
:10E83000094908700848007801F028FD07E00448FD
:10E8400000680849884202D10D2003F0C1FE10BDC6
:10E85000400000202A04BC0010010020D400002049
:10E860002A04DC002A00FC0038B50446CCB1F9F7D4
:10E87000B3F902210BA001F0FFFE00200B49087044
:10E880000846007801F002FD01236E229F2100203E
:10E89000F9F75AFA0020012305A272210090F9F736
:10E8A0008DFC38BD41504ECFEAC7E9001001002071
:10E8B0002020202020202020205B455849545DB78F
:10E8C000B5BBD80070B505460C46284607F0DAFD02
:10E8D0002146002009F002FA04F10801012009F0A4
:10E8E000FDF970BD70B505460C460A4890F8F70270
:10E8F00000B970BD284607F0C5FD0121064802F0A9
:10E900002AFF20B209F009FA0021034802F023FF90
:10E9100000BFEEE7DE1B00200008004043185A004D
:10E92000FF2A00DD7047034B1870034B197000BFBE
:10E93000F8E700006E0000206F00002010B586B0E0
:10E940001748FBF781F804461648844214D114484E
:10E95000C38815A2142101A805F080FD01A8FCF7C9
:10E9600049FF0F488079154908700120144981F842
:10E97000620203F02DFE10E0124884420DD11248CD
:10E980008079012806D100200F498871012003F009
:10E990001FFE02E0062003F01BFE06B010BD0000C3
:10E9A000C02400202A04EC0041542B53494D43520B
:10E9B0004F53533D25640D0A00000000040300205E
:10E9C0005C0800202A00FC004A0300207CB50446B5
:10E9D00000250CB3F9F700F901211CA001F04CFE51
:10E9E00000200190012001A91B4A1278885401A837
:10E9F0001A4B00221A4900901A48FAF74FFF0020DC
:10EA0000012319A272210090F9F7D8FB01236E228D
:10EA10007F210020F9F798F918480088142807D1B9
:10EA20000020012310A272210090F9F7C7FB00E03B
:10EA300000BF12480088401C80B210490880B0F521
:10EA4000C87F01DB002008807CBD000053494DBF1A
:10EA5000A8D1A1D4F100000004030020EC000020A4
:10EA600028010020C02400203CCDCBB3F62020C8D4
:10EA7000B7B6A82020CFC2B7AD3E00005801002095
:10EA800000B589B02948006829490844C0B1B0F5EB
:10EA9000001F06D0B0F5401F22D0B0F5601F41D155
:10EAA0003CE02448007818B901202249087004E0AD
:10EAB00020480078401E1F490870F6F75DFC31E0E1
:10EAC0001C480078012803D100201A49087004E08E
:10EAD00018480078401C17490870F6F74DFC21E0F3
:10EAE000154890F8640213490978884212D01148F9
:10EAF0000078114981F864020E4802780FA101A83C
:10EB000005F0C0FC01A8FCF775FE012211A1002050
:10EB100002F024FB012003F05BFD03E0062003F07C
:10EB200057FD00BF00BF09B000BD0000400000203D
:10EB3000D6FB43FF110100205C08002041542B50FC
:10EB40004F433D3430303030303031253032780D65
:10EB50000A00000055706461746520636F64657419
:10EB60007970650038B504460425012C22D10020B7
:10EB700021490880F9F730F8012120A001F07CFD3F
:10EB800001236E229F210020F9F7DEF81E4800784D
:10EB900048B91EA001F040FE322009F0BEF8062060
:10EBA00003F016FD06E01D4890F864021C49087049
:10EBB000F6F7E2FB1048008838B90020012319A2BB
:10EBC00072210090F9F7FAFA0AE00B480088C82889
:10EBD00006D10020012318A272210090F9F7EEFA65
:10EBE00005480088401C80B203490880B0F5C87F02
:10EBF00001DB0020088038BD4E010020B1E0C2EBEF
:10EC0000C6F7C9E8D6C3000001030020C4A3BFE9CA
:10EC1000D4DDCEB4C6F4B6AF000000005C0800201E
:10EC2000110100205BC9CF5DD1A1D4F1205BCFC21F
:10EC30005DD1A1D4F10000005B4D5DB1A3B4E65BF2
:10EC4000455849545DCDCBB3F600000010B52D48B2
:10EC500000682D49084458B1B0F5001F07D0B0F541
:10EC6000401F49D029490844002849D128E000BF65
:10EC70002748007800B143E02248006825498842CF
:10EC80000DD12548807A072805DA2348807A401C70
:10EC9000214988720FE000201F4988720BE01E484E
:10ECA000807A18B907201C49887204E01A48807AD3
:10ECB000401E194988721849887A00F0A3F81FE0AD
:10ECC0001348007800B11BE01348807A134991F88B
:10ECD000F812884209D01048807A104981F8F80269
:10ECE000F8F776FE0120FCF71FFF01200C490871A0
:10ECF000022003F06DFC03E0022003F069FC00BF7A
:10ED000000BF10BD40000020D6FB43FF0004C0FF41
:10ED10009C0000202A04DC00281F0020DE1B0020AD
:10ED20004A03002038B5044604B3F8F755FF012123
:10ED30001FA001F0A1FC0020012320A23B21009094
:10ED4000F9F73CFA0020F7F7B9FE214890F8F802ED
:10ED500020498872887A00F055F801236E229F219D
:10ED60000020F8F7F1FF00201B4908801A480088AE
:10ED700038B90020012319A272210090F9F71EFA78
:10ED80000AE015480088C82806D10020012318A2EF
:10ED900072210090F9F712FA0F480088401C80B2E7
:10EDA0000D490880B0F5C87F01DB0020088038BD20
:10EDB000B6A8CEBBC9E8D6C300000000B6A8CEBB3B
:10EDC000C9CFB4ABC9E8D6C33A202020C3EB0000BA
:10EDD000DE1B0020281F0020500100205BC9CF5DF2
:10EDE000D1A1D4F1205BCFC25DD1A1D4F10000004C
:10EDF0005B4D5DB1A3B4E65B455849545DCDCBB3E3
:10EE0000F60000007FB50546104830F815404B234A
:10EE10007F223B216420F8F739FF44B90020012309
:10EE20000BA23B2100906420F9F7C8F90DE02346BE
:10EE300009A20A2101A805F011FB0020012301AA63
:10EE40003B2100906420F9F7B9F97FBD4A7D0108A4
:10EE500020B9D8B1D5200000202530326420C3EB82
:10EE6000000000002DE9F0413248047945798679A7
:10EE7000C779302C1AD1302D18D1322E16D1302F1F
:10EE800014D1B0F89601001F2A49A1F8960101207B
:10EE9000087088700020C8704870012226A102F016
:10EEA0005DF90220234981F898013BE0012C19D13A
:10EEB000022D17D11F48B0F89601001F1D49A1F877
:10EEC00096010220087081F898011E48007820F011
:10EED0000200801C1B49087001221BA1002002F0C7
:10EEE0003DF91FE0202C1DD1202D1BD1202E19D142
:10EEF000202F17D10F48B0F89601001F0D49A1F837
:10EF0000960100200870012081F898010D480078D2
:10EF100020F00200801C0B49087001220DA1002086
:10EF200002F01CF900200E49487101200870BDE86C
:10EF3000F0810000981F0020416C61726D53746174
:10EF400072740000A821002050757265205454533B
:10EF500000000000507572652054585400000000F5
:10EF60003602002038B504461CB3F8F735FE0121FF
:10EF70001CA001F081FB1E480021016001201D49F9
:10EF800091F8F7121A4A505410461B4B00221B49A5
:10EF900000901B48FAF782FC0020012319A272217D
:10EFA0000090F9F70BF901236E229F210020F8F75A
:10EFB000CBFE19480088142807D10020012311A294
:10EFC00072210090F9F7FAF800E000BF12480088BB
:10EFD000401C80B210490880B0F5C87F01DB0020DA
:10EFE000088038BDCCE1CABED2F4C9E8D6C300005F
:10EFF00054010020DE1B0020EC0000201401002042
:10F00000C02400203CCDCBB3F62020C8B7B6A82042
:10F0100020CFC2B7AD3E00005201002010B586B02F
:10F020002448FAF711FD0446234884423AD1214886
:10F03000C088224991F8F71288422CD01D48807967
:10F040001E4981F8F702084690F8F702B0B11C4853
:10F05000007818B91BA0FCF7CDFB19E01848007820
:10F06000012815D1154890F832331AA2142101A8AD
:10F0700005F0F4F901A8FCF7BDFB09E010480078A1
:10F0800018B919A0FCF7B6FB02E01BA0FCF7B2FB15
:10F090000120FCF749FD01201C490871022003F002
:10F0A00097FA05E01A48844202D1022003F090FA50
:10F0B00006B010BDC02400202A04EC00DE1B002096
:10F0C0009C00002041542B544F4E45533D310D0AB6
:10F0D0000000000041542B504F433D746F6E657625
:10F0E0006F6C3D25640D0A0041542B544F4E45531F
:10F0F0003D300D0A0000000041542B504F433D7439
:10F100006F6E65766F6C3D300D0A00004A0300207B
:10F110002A00FC0010B5042425480068254908444D
:10F12000C0B1B0F5001F07D0B0F5401F23D0224971
:10F130000844002839D134E020480078401CC0B28F
:10F140001E490870052801DB00200870022000F02D
:10F150003BF82AE019480078002805DD17480078B8
:10F16000401E1649087002E004201449087002206D
:10F1700000F02AF819E0124890F89A000F4909782F
:10F18000884207D00D4800780D4981F89A00012087
:10F19000FCF7CAFC01200B490871062003F018FA9D
:10F1A00003E0062003F014FA00BF00BF10BD00000A
:10F1B00040000020D6FB43FF0004C0FF34010020C4
:10F1C000DE1B00204A03002030B587B0054604242A
:10F1D000012D4FD14C4890F89A004C490870F8F72F
:10F1E000FBFC01214AA001F047FA00200090A0B2E8
:10F1F000012349A23821F8F7E1FF444800780428A8
:10F2000005D149A20A2104A805F028F90BE03E48DF
:10F2100090303E49097800EB4100038844A20A215E
:10F2200004A805F01BF9002004F13C01009088B20D
:10F23000012304AA3821F8F7C1FF344803783EA21D
:10F24000062102A805F00AF9012202A9002001F016
:10F2500085FF0020012339A272210090F8F7AEFF4C
:10F2600001236E227F210020F8F76EFD002038492F
:10F2700008802FE0022D2DD104F13C0188B210232B
:10F2800080223821F8F702FD20480078042805D1B3
:10F2900025A20A2104A805F0E1F80BE01A489030F5
:10F2A0001A49097800EB4100038821A20A2104A829
:10F2B00005F0D4F8002004F13C01009088B201234D
:10F2C00004AA3821F8F77AFF01236E227F2100205B
:10F2D000F8F73AFD1E48008838B90020012317A22C
:10F2E00072210090F8F76AFF00E000BF184800881C
:10F2F000401C80B216490880B0F5C87F01DB0020B1
:10F30000088007B030BD0000DE1B00203401002063
:10F310004C4344C9E8D6C30020B1B3B9E2CAB1BC7A
:10F32000E43A202020200000B3A3C1C12020200007
:10F3300025336420C3EB0000253364003CCDCBB300
:10F34000F62020C8B7B6A82020CFC2B7AD3E000037
:10F350005A01002010B51148FAF776FB0446104810
:10F36000844213D10D48C0880E490979884206D0DD
:10F370000A4880790B4908710120FCF7D5FB012070
:10F3800009490871062003F023F905E00748844283
:10F3900002D1062003F01CF910BD0000C02400209B
:10F3A0002A04EC00DE1B00204A0300202A00FC0097
:10F3B00038B504461CB3F8F70FFC022110A001F089
:10F3C0005BF912480021016001710120104909799F
:10F3D0000E4A505410460F4B00220F4900900F4820
:10F3E000FAF75CFA01236E229F210020F8F7ACFCAB
:10F3F000002001230AA272210090F8F7DFFE38BD39
:10F40000B1B3B9E2B5F7BDDA000000004901002050
:10F41000DE1B0020EC000020F8000020C0240020AB
:10F420003CCDCBB3F62020C8B7B6A82020CFC2B7BA
:10F43000AD3E000010B50446052C27D2DFE804F0ED
:10F44000030A11181F00002011490870012000F064
:10F4500021F81BE001200E490870052000F01AF881
:10F4600014E002200A490870062000F013F80DE0AD
:10F47000032007490870042000F00CF806E004207F
:10F4800003490870012000F005F800BF00BF10BD5F
:10F490007100002010B504460A2C60D2DFE804F0A9
:10F4A000050E172029323B444D560021084600F036
:10F4B000B1FA00210846FFF731FA50E0002101209F
:10F4C00000F0A8FA00210846FFF728FA47E00121DA
:10F4D000084600F09FFA00210846FFF71FFA3EE0B9
:10F4E0000A21012000F096FA00210846FFF716FADB
:10F4F00035E00021084600F08DFA00210120FFF7D9
:10F500000DFA2CE00021084600F084FA012108469B
:10F51000FFF704FA23E00021084600F07BFA0A21F5
:10F520000120FFF7FBF91AE00021012000F072FA38
:10F5300000210120FFF7F2F911E00121084600F057
:10F5400069FA01210846FFF7E9F908E00A210120DC
:10F5500000F060FA0A210120FFF7E0F900BF00BFC8
:10F5600010BD000030B589B03B4800683B490844F5
:10F5700008B3B0F5001F06D0B0F5401F33D0B0F58A
:10F58000601F65D160E0364800786E2803D16420A2
:10F590003349087004E032480078401C3049087054
:10F5A0002F4803782FA21E2101A804F057FF01A8BD
:10F5B000F6F756FF4CE02A480078642803D16E2005
:10F5C0002749087004E026480078401E2449087046
:10F5D0002348037823A21E2101A804F03FFF01A8BD
:10F5E000F6F73EFF34E0322008F097FB1C48007825
:10F5F0001E4981F831031A4805780478E01704EBB6
:10F6000010700011A4EB0013E81705EB1070021145
:10F6100017A101A804F036FF01A8FCF7EBF8104889
:10F6200005780478E01704EB10700011A4EB0013C8
:10F63000E81705EB1070021101A915A004F0FEFEF9
:10F640000020FCF771FA03E0062002F0C1FF00BFC2
:10F6500000BF09B030BD000040000020D6FB43FFD2
:10F66000440100202530336400000000DE1B002030
:10F6700041542B43414343503D322C312C362C22F4
:10F68000253032783030253032783030220D0A0083
:10F6900025732D2D2D253032782D2D2D2D25303211
:10F6A000780000001CB50446012C2AD10020264910
:10F6B0000880F8F791FA012124A000F0DDFF012372
:10F6C0006E229F210020F8F73FFB2348007848B9BD
:10F6D00022A001F0A1F8322008F01FFB062002F062
:10F6E00077FF0EE0214890F8310321490870084661
:10F6F000037820A2042101A804F0B0FE01A8F6F7C7
:10F70000AFFE1148008838B9002001231BA27221E6
:10F710000090F8F753FD0AE00B480088C82806D18E
:10F72000002001231BA272210090F8F747FD064834
:10F730000088401C80B204490880B0F5C87F01DB16
:10F74000002008801CBD0000CE010020C2F3BFCB0A
:10F75000B7E7D4F6D2E6000001030020C4A3BFE956
:10F76000D4DDCEB4C6F4B6AF00000000DE1B00202E
:10F770004401002025303364000000005BC9CF5DE8
:10F78000D1A1D4F12020202020205BCFC25DD1A1C7
:10F79000D4F100005B4D5DB1A3B4E6202020205BD6
:10F7A000455849545DCDCBB3F600000010B586B086
:10F7B0001B48FAF749F904461A48844227D11A48E7
:10F7C00090F8F6121648C088B1EB400F18D01448D4
:10F7D00080794006000E144981F8F602084690F838
:10F7E000F6020090114890F9003011A20F2102A8F2
:10F7F00004F034FE02A8FBF7FDFF0120FCF794F9AA
:10F8000001200F490871022002F0E2FE05E00D48D8
:10F81000844202D1022002F0DBFE06B010BD0000DF
:10F82000C02400202A04EC00DE1B0020440300203A
:10F8300041542B435445433D25642C25640D0A0057
:10F840004A0300202A00FC001CB504460020019059
:10F85000E4B1F8F7C1F9022118A000F00DFF012171
:10F86000194A92F8F60200EBD072521001AB99548B
:10F8700001A8164B0022164900901648FAF70EF818
:10F8800001236E227F210020F8F75EFA12480088DB
:10F8900038B90020012311A272210090F8F78EFCE4
:10F8A00000E000BF0C480088401C80B20A49088074
:10F8B000B0F5C87F01DB002008801CBDCDF8C2E791
:10F8C000C9E8D6C300000000DE1B0020EC000020C9
:10F8D00060010020C02400205C0100203CCDCBB39F
:10F8E000F62020C8B7B6A82020CFC2B7AD3E000092
:10F8F000F8B504462046F7F73FFA06463046F7F7D4
:10F9000057FA054605B9F8BD6B4602221C21304660
:10F91000FEF7D6FBBDF80000082800D0F3E7044B43
:10F920004FF4806236213046FEF7CAFB00BFEAE79B
:10F93000FC26002010B51248FAF786F80446114854
:10F94000844215D10E48C0880F4991F82F13884280
:10F9500007D00B4880790C4981F82F030120FCF770
:10F96000E3F8012009490871062002F031FE05E0A4
:10F970000748844202D1062002F02AFE10BD000092
:10F98000C02400202A04EC00DE1B00204A030020D3
:10F990002A00FC001CB504460020019004B3F8F7CF
:10F9A0001BF902210FA000F067FE0120104991F819
:10F9B0002F1301AA505401A80E4B00220E490090AB
:10F9C0000E48F9F76BFF01236E227F210020F8F724
:10F9D000BBF9002001230AA272210090F8F7EEFB88
:10F9E0001CBD0000C4A3CABDC9E8D6C30000000006
:10F9F000DE1B0020EC00002084010020C024002039
:10FA00003CCDCBB3F62020C8B7B6A82020CFC2B7D4
:10FA1000AD3E000043185A00FF2A00DD7047034B3B
:10FA20001870034B197000BFF8E700006C0000204D
:10FA30006D00002010B51D48FAF726FD04461C484D
:10FA400084422CD119484079072821D2DFE800F000
:10FA500004080C1014181C00102002F0B9FD17E067
:10FA60001D2002F0B5FD13E01E2002F0B1FD0FE0F5
:10FA70001C2002F0ADFD0BE0192002F0A9FD07E00B
:10FA8000132002F0A5FD03E01A2002F0A1FD00BF43
:10FA900000BF064841790748FEF7DCF805E0064854
:10FAA000844202D1022002F093FD10BDB800002074
:10FAB0002A04EC004A0300202A00FC0010B5164876
:10FAC000F9F7C2FF0446154884421ED11448C07895
:10FAD0001149C988884211D00F4880791049C870EF
:10FAE0000846C078012803D10EA0FBF783FE02E090
:10FAF00015A0FBF77FFE0120FCF716F801201B493B
:10FB00000871062002F064FD05E01948844202D124
:10FB1000062002F05DFD10BDC02400202A04EC0088
:10FB2000DE1B002061742B737973636D643D737405
:10FB30006172745F70636D20766F6C756D652037D0
:10FB400020370D0A0000000061742B737973636D18
:10FB5000643D73746172745F70636D20766F6C7551
:10FB60006D65203720350D0A000000004A03002093
:10FB70002A04F4001CB50446002001900CB3F8F7E9
:10FB80002BF802210FA000F077FD0020019001204A
:10FB90000F49C97801AA505401A80E4B00220E4902
:10FBA00000900E48F9F77AFE01236E227F21002093
:10FBB000F8F7CAF80020012309A272210090F8F793
:10FBC000FDFA1CBDB3A1BEB0C4A3CABD00000000B5
:10FBD000DE1B0020EC00002094010020C024002047
:10FBE0005B4F4B5DC7D0BBBB2020205B45584954C1
:10FBF0005DCDCBB3F600000070B590B00546002493
:10FC0000002618228C4902A8F4F7AEFAF7F7ACFCEC
:10FC100004B28A4800788A49087000BF49E08848E1
:10FC2000007888B986480078002840D102A8844925
:10FC3000097830F811000A30A04238DA804800789C
:10FC4000401C7F49087032E07D4800780A281CDAA1
:10FC500002A87B49097830F811000A30A04205DC7F
:10FC600077480078401C7649087020E07448007896
:10FC7000401E02A931F810000A38A04217DD704872
:10FC80000078401E6E49087011E06D4800780A281F
:10FC90000DD16B480078401E02A931F810000A38D7
:10FCA000A04204DD66480078401E65490870701C5B
:10FCB000C6B20B2EB3DB012D03D16148007810B022
:10FCC00070BD5F4800785D490978884201D1022DF6
:10FCD0007DD15B48007808B101F028FB58480278D4
:10FCE000214658A004F0AAFB022D09D154480078FF
:10FCF0005249087052480078584981F832032DE083
:10FD000057480078012820D14D4800784B490978A0
:10FD100088420BDA4A49097801EB81011B2202EB88
:10FD200041007B2369226F21F7F7B0FF4448037835
:10FD30004CA21E2108A804F091FB0020012308AA70
:10FD40006E2100902C20F8F739FA3D4800783B49A5
:10FD500008703B480078414981F8320337480378FE
:10FD600043A21E2108A804F079FB08A804F066FB52
:10FD70003248007800EB800043003FA21E2108A813
:10FD800004F06CFB08A8FBF735FD3F48007868B924
:10FD90002A48007800EB800043003CA21E2108A8FE
:10FDA00004F05CFB08A8FBF725FD19E02B4890F850
:10FDB000F70248B12148037838A21E2108A804F0B0
:10FDC0004DFB08A8FBF716FD1C48037800E011E086
:10FDD00037A21E2108A804F041FB08A8FBF70AFD82
:10FDE0000120F9F7EBF90020364908804FF49670AE
:10FDF000354908803448B0F90000002818DD324841
:10FE00000088401E00B23049088088B91448007844
:10FE100001280DD17E2364226E212C20F7F736FFB6
:10FE20002A48C07820B92948007908B901F072FA47
:10FE30000348007843E700005C7D0108F6010020DC
:10FE4000F501002074656D706C763D25642D2D2DB7
:10FE50002D6E756D3D3D3D25640D0A00DE1B0020B5
:10FE600046030020D2F4C1BF2530326400000000F8
:10FE7000D2F4C1BF2025640041542B434C564C3D65
:10FE800025640D0A000000009C00002041542B4313
:10FE900052534C3D25640D0A0000000041542B5084
:10FEA0004F433D746F6E65766F6C3D25640D0A009F
:10FEB00041542B504F433D747473766F6C3D2564F1
:10FEC0000D0A0000B0000020F80100205C080020AE
:10FED00010B500F001F810BD0CB5002001900090A5
:10FEE0003348006840F480303149086000BF304832
:10FEF000006800F4003000900198401C01900098C8
:10FF000020B94FF6FF7101988842F0D12848006867
:10FF100000F4003010B10120009001E000200090BA
:10FF20000098012843D12348006840F0100021497F
:10FF300008600846006820F0030008600846006872
:10FF400040F0010008601A484068194948600846B6
:10FF5000406848600846406840F480604860084651
:10FF6000406820F47C1048600846406840F4102047
:10FF700048600846006840F08070086000BF0C4888
:10FF8000006800F000700028F9D00948406820F0AF
:10FF90000300074948600846406840F00200486096
:10FFA00000BF0348406800F00C000828F9D10CBDE0
:10FFB000001002400020024010B51E48F9F744FD31
:10FFC00004461D4884422DD11A48C0881B4909782F
:10FFD000884220D017488079184908700846007870
:10FFE00020B1012807D0022814D109E04FF4807015
:10FFF000134908600EE04FF480701149086009E071
:020000040801F1
:100000004FF480700E49091F086001200D4981F8E6
:10001000620200BF00BF01200B490871062002F0F8
:10002000D7FA05E00948844202D1062002F0D0FA4E
:1000300010BD0000C02400202A04EC00350100207F
:10004000140801405C0800204A0300202A00FC003C
:100050001CB5044600200190C4B1F7F7BDFD022194
:1000600016A000F009FB012001A9174A1278885454
:1000700001A8164B0022164900901648F9F70EFC0D
:1000800001236E229F210020F7F75EFE12480088B0
:1000900038B90020012311A272210090F8F78EF8E0
:1000A00000E000BF0C480088401C80B20A4908806C
:1000B000B0F5C87F01DB002008801CBDB4AEBFDAFC
:1000C000C7D0BBBB0000000035010020EC000020C1
:1000D00074010020C0240020700100203CCDCBB36F
:1000E000F62020C8B7B6A82020CFC2B7AD3E00008A
:1000F00010B50D480078022814D10C4800680C494E
:10010000884206D10320084908700AA0FBF772FB59
:1001100007E0064800680A49884202D1062002F03A
:1001200057FA00BF00BF10BD3C0100204000002076
:100130002A04EC0041542B464F54413D310D0A0036
:100140002A00FC0010B58CB00446002C24D0F7F730
:1001500043FD012130A000F08FFA33A0F6F780F9BB
:1001600001236E227F210020F7F7EEFD00200123FE
:1001700031A272210090F8F721F84FF0FF30334997
:10018000086000203249087032A0FBF733FB4FF4BF
:10019000C871334807F0CEFD2D48007810B1012812
:1001A00037D12EE02E4807F0ADFD002828D0274893
:1001B000006850B90120264908702AA0F6F750F9C6
:1001C0009621274807F0B6FD1AE02048006800286D
:1001D0000CDD1E4827A1026802A804F053F902A80A
:1001E000F6F73EF902201A49087009E00120184983
:1001F000087023A0F6F734F99621194807F09AFD04
:1002000007E0174807F07EFD10B1012002F0E0F989
:1002100000BF00BF0CB010BDC9FDBCB6B6D4BDB2A6
:10022000B0E6B1BE00000000D5FDD4DABCECB2E20D
:10023000B0E6B1BE000000003CCDCBB3F62020C834
:10024000B7B6A82020CFC2B7AD3E000038010020CD
:100250003C01002041542B464F54413F0D0A000001
:1002600040010020C3BBD3D0BFC9B8FCD0C2B0E6A8
:10027000B1BE0000B8FCD0C2B5BD562564203F0019
:10028000BCECB2E2B3ACCAB1000000002DE9F04111
:1002900096B0804600261B250E2467237F22294620
:1002A0000020F7F7F3FC53485349097850F8213000
:1002B00052A228210CA804F0D1F800203246761C66
:1002C0000090102000FB025101230CAA1846F7F7FA
:1002D00075FF49490978C1EB4112494901EB4200D8
:1002E000F3F790FFC7B244480078C0EB401244488F
:1002F00000EB4201224602A8F3F736FF002002A9D4
:10030000085502AB3FA228210CA804F0A7F8002052
:100310003246761C0090102000FB025101230CAAEB
:100320001846F7F74BFFA74217DD33480078C0EBBC
:100330004012334800EB420001190CA8F3F784FF88
:10034000002000903046721CD6B2102202FB0051F1
:1003500001230CAA1846F7F731FF27490978C1EBAA
:100360004112274901EB420101F11F00F3F74AFF57
:10037000C7B221480078C0EB4012214800EB420090
:1003800000F11F01224602A8F3F7EEFE002002A9A9
:10039000085502AB1DA228210CA804F05FF800202C
:1003A00000903046721CD6B2102202FB005101238D
:1003B0000CAA1846F7F702FFA74218DD0E4800788E
:1003C000C0EB40120E4800EB42001F3001190CA890
:1003D000F3F73AFF002000903046721CD6B210228C
:1003E00002FB005101230CAA1846F7F7E7FE16B0EE
:1003F000BDE8F081D80000201001002025733A00EC
:10040000DC1D00204E616D653A25730050617373E9
:100410003A25730038B505466A24B5F5A27F20DC7D
:10042000524807F06FFC00B938BD50214F4807F023
:1004300081FC4F48007840B9A0B24EA20121F7F7E5
:100440005CFE01204A4908708EE00020484908708F
:1004500004F115018AB2A0B20D230021F7F716FCB2
:1004600082E0B5F5B17F0FDCA0B242A20121F7F71F
:1004700044FE0320009004F1100082B203230821FF
:100480001846F7F7A4FC6FE0B5F5BB7F19DCA0B206
:1004900038A20121F7F731FE0320009004F10C008F
:1004A00082B2032308211846F7F791FC032000903D
:1004B00004F1100082B2032308211846F7F787FCE5
:1004C00052E0B5F5C87F23DAA0B22AA20121F7F7DE
:1004D00014FE0320009004F1080082B203230821D7
:1004E0001846F7F774FC0320009004F10C0082B268
:1004F000032308211846F7F76AFC0320009004F153
:10050000100082B2032308211846F7F760FC2BE0A5
:10051000A0B218A20121F7F7F0FD03200090201DE2
:1005200082B2032308211846F7F751FC03200090FC
:1005300004F1080082B2032308211846F7F747FCAC
:100540000320009004F10C0082B203230821184616
:10055000F7F73DFC0320009004F1100082B2032362
:1005600008211846F7F733FC00BF5DE7A803002019
:10057000AC03002056424154312E626D70000000E1
:10058000F8B504460D4616463046F7F78DF807468F
:1005900005F1140083B2E019083082B229462046E2
:1005A000F7F774FB0120AA1C91B2221D009090B2B3
:1005B00001233246F7F702FEF8BD000030B58BB0DC
:1005C00004460D462948007898B128480078142838
:1005D0000FD02648007828280BD0244800783C28E3
:1005E00007D022480078502803D02048007864289B
:1005F0002FD124221E491F48F3F72FFE50B9242281
:100600001B491C48F3F729FE20B91948783890F89F
:10061000610288B104F1200188B212237C222946AC
:10062000F7F7F0FA242212491248F3F79DFD002053
:100630000F49783981F8610224220E4902A800F09E
:1006400007FF002010230A4A294600902046F7F7AA
:10065000B5FD06480078401CC0B204490870642803
:1006600001DD002008700BB030BD0000AE0300209B
:10067000D408002048260020F8B504460D46204640
:10068000F7F712F806460E250020C6F1800707EBA3
:10069000D7710090C1F34F00012322462946F7F796
:1006A0008DFDF8BDF0B58DB006460C4615463CA252
:1006B00007CA01AB07C300273C4890F8600270B935
:1006C0003B493A484630F3F7A4FD00B99DB12422D6
:1006D000364946313648F3F747FD01270BE03449E8
:1006E00001A8F3F796FD00B92DB1092201A9304800
:1006F000F3F73AFD01272F492C481930F3F789FD0C
:1007000000B935B12422294919312A48F3F72CFDC3
:100710000127002F41D004F1140083B27F2221462B
:100720003046F7F7B3FA04F1280083B2143881B2E7
:100730007F223046F7F7AAFA1FA221463046F7F784
:10074000DCFC04F1180081B21EA23046F7F7D5FC9C
:100750002422174904A800F07BFE002006F11001B6
:10076000009088B2102304AA2146F7F727FD24221F
:10077000104904A800F06CFE002004F1180291B2A8
:1007800006F11002009090B2102304AAF7F716FDAC
:100790000120064981F8610200270DB0F0BD00007C
:1007A000B5A5BAF4C4A3CABD000000005C080020CF
:1007B000902600206C26002047726F7570322E62E2
:1007C0006D70000070656F706C65322E626D700028
:1007D00000B587B002A8FDF781FA0398009004A045
:1007E000DDE90423029903F029FE07B000BD0000F3
:1007F000535953434C4B3D25642C50434C4B313D96
:1008000025642C50434C4B323D25642C48434C4BC3
:100810003D25640D0A000000F0B593B00546402464
:1008200004F11403A4F1140081B27F220020F7F731
:100830002DFA012004F112030090A4F1120081B2FC
:100840007E220220F7F797FA1222294601A800F02B
:10085000FFFD01A8F6F728FF86B2C6F1800000EB85
:10086000D071C1F34F0700200090A4F1080081B2BD
:10087000012301AA3846F7F7A1FC13B0F0BD000030
:1008800038B5044642480078012805D141A202212A
:100890000020F7F732FC04E042A202210020F7F723
:1008A0002CFC012C01DB632C06D10B23122203212B
:1008B0000720F7F7EBF969E0082C0EDA0320022392
:1008C00007220A2100900920F7F781FA0B23122250
:1008D00003210920F7F7DAF958E0102C16DA032083
:1008E000022307220A2100900920F7F770FA03205B
:1008F00002230A22114600900720F7F768FA0B231B
:10090000122203210D20F7F7C1F93FE0162C1EDA61
:100910000320022307220A2100900920F7F757FA43
:10092000032002230A22114600900720F7F74FFA0E
:10093000032002230D220A2100900520F7F747FA31
:100940000B23122203211020F7F7A0F91EE0032049
:10095000022307220A2100900920F7F738FA032022
:1009600002230A22114600900720F7F730FA0320ED
:1009700002230D220A2100900520F7F728FA032010
:10098000022310220A210090F7F721FA38BD000057
:10099000E901002053696E676C654F4B2E626D70E4
:1009A0000000000053696E676C652E626D70000078
:1009B00038B504460D466C4890F90000401C90B9CB
:1009C00001200C239F22002100900846F7F71AFA15
:1009D00002201A239F220D2100900020F7F712FA1F
:1009E000012061490870614890F900006049097868
:1009F00088422FD05F48007801282BD102201A238B
:100A00009F220D2100900020F7F7FCF9584800784C
:100A100030B1012809D002280CD0032814D10EE0EF
:100A20000D2155A0FFF728FE0EE00D2155A0FFF780
:100A300023FE09E00D2156A0FFF71EFE04E00D2164
:100A400056A0FFF719FE00BF00BF4948007840B22A
:100A500046490870564890F90000564991F900102F
:100A6000884209D0534890F900005149087008465F
:100A700090F9000000F020F94F488078C8B14F4845
:100A800000784F4991F90010884212D04B48007805
:100A900028B94CA203211420F7F72FFB04E04CA245
:100AA00003211420F7F729FB4448007840B2444959
:100AB00008704A4800684A490968884205D149488F
:100AC00000784949097888420BD047480078454961
:100AD0000870434800684149086041480068FFF7D2
:100AE000CFFE42480078642808DA4FF4B4704049D9
:100AF00008603E480078401C3C4908703D4800684A
:100B00003B49096888420CD139480068B0F5A27F9A
:100B100007DD394890F90000384991F90010884202
:100B200015D03348006833490860344890F9000014
:100B3000314908700846007828B931A201216A209D
:100B4000F7F7DBFA03E02A480068FFF763FC20466A
:100B500000F066F82E480078012804D12DA200216B
:100B60005C20F7F7CAFA38BD780300207A0300202A
:100B7000FD02002046030020D6D0B9FAB5E7D0C563
:100B800000000000D6D0B9FAD2C6B6AF000000000F
:100B9000D6D0B9FAC1AACDA800000000B9ABCDF8F3
:100BA000BCAFC8BAB6D4BDB2CFB5CDB3000000005B
:100BB00077030020440300205C0800200403002089
:100BC0007903002053494D312E626D700000000002
:100BD00053494D322E626D70000000006C030020FE
:100BE000F802002076030020E901002068030020BD
:100BF000EC010020700300207B030020FC02002099
:100C00004348415247454241542E626D70000000F6
:100C1000E40200206C6F636B2E626D7000000000B8
:100C200010B58CB004461C48407808B90CB010BD13
:100C30000AA8FDF715F99DF82E0018490978884291
:100C400000D13CB39DF82E0014490870087800EBE1
:100C5000D0714910A0EB410151B19DF82D000090D9
:100C60009DF82C300EA21E2102A803F0F7FB09E02C
:100C70009DF82D0000909DF82C300CA21E2102A89A
:100C800003F0ECFB0020012302AA01460090302073
:100C9000F7F794FA00BFC9E75C080020AD03002015
:100CA000253032643A253032640000002530326449
:100CB000202530326400000038B50446124890F810
:100CC0006302042800D138BD022C00D044B90020B2
:100CD00001230EA2014600901E20F7F76FFA10E0E4
:100CE000072C08D10020012309A2014600901E20F4
:100CF000F7F764FA05E00A232E2200211E20F6F7FA
:100D0000C5FF00BFDFE700005C080020324700009D
:100D10003447000070B58CB004460D4600265CB127
:100D2000C348007840B10020C249A1F86C00C24914
:100D30000870BF49087000BFBF48007806283FD23E
:100D4000DFE800F0033F5CF8F7F6BC4800780428C1
:100D50000FD1BB480078012805D1BAA2282102A8EA
:100D600003F07CFB16E0BCA2282102A803F076FB6E
:100D700010E0B3480078012807D1AE48BAA2282174
:100D8000036C02A803F06AFB04E0BDA2282102A8BC
:100D900003F064FB02A8FAF72DFD002202A9104619
:100DA00000F0DCF90020A34981F86C0281F86602AA
:100DB0004FF4FA71B64806F0BDFF01209E49087055
:100DC00032E19C4890F86C0218B9B14806F09AFFDD
:100DD00098B19848D0F8680260B90020954981F828
:100DE00066020846D0F8682290F86C12A9A003F0B9
:100DF00025FB0AE102209049087015E1012C65D01D
:100E0000012D2DD18B48B0F86C00401C8949A1F808
:100E10006C000846D0F868020521B0FBF1F0854966
:100E2000B1F86C10884203D200208249A1F86C000E
:100E30008048D0F868020521B0FBF1F201FB1200F6
:100E400090BB7C48D0F86802B0FBF1F07949B1F86A
:100E50006C1088423AD100207649A1F86C0035E048
:100E60007448B0F86C00002807DD7248B0F86C00D8
:100E7000401E7049A1F86C0028E06E48B0F86C0084
:100E800090B96C48D0F868020521B0FBF1F201FB83
:100E9000120050B96748D0F86802B0FBF1F0401E6C
:100EA0006449A1F86C0009E010E06248D0F86802DB
:100EB0000521B0FBF1F05F49A1F86C005D48B0F886
:100EC0006C20D0F86812804803F0B8FA5948B0F89E
:100ED0006C00401C00EB80005649D1F86812884233
:100EE00029D95448B0F86C3078A2282102A803F020
:100EF000B5FA012202A9002000F030F94D48D0F8DF
:100F000068020521B0FBF1F201FB120020B90520B7
:100F1000484981F8650212E04648D0F86802052188
:100F2000B0FBF1F201FB1200424981F8650206E0D4
:100F30006AE05AE00BE005203E4981F86502002096
:100F40003C4981F8660203203B4908706CE00020B0
:100F5000384981F86E0239480078042819D1384898
:100F6000007801280AD10846B0F86C0000EB800335
:100F700058A2282102A803F071FA26E02D48B0F803
:100F80006C0000EB800359A2282102A803F066FA46
:100F90001BE02B48007801280DD12648B0F86C00E2
:100FA00000EB80000090234856A22821036C02A881
:100FB00003F054FA09E01F48B0F86C0000EB80031E
:100FC00057A2282102A803F049FA02A8FAF712FC56
:100FD000002202A9104600F0C1F8C8212C4806F0F2
:100FE000A9FE0420144908701EE0124890F86E0211
:100FF00010B1052010490870254806F083FE10B195
:1010000005200D4908700FE000BF01200849087055
:1010100060237F2228210020F6F738FE00200649B1
:10102000087001200CB070BD00BF3046FAE7000028
:10103000940000205C08002095000020460300205A
:101040009C00002041542B504F433D67726F7570D8
:101050006E756D0D0A00000041542B504F433D3317
:1010600044303030300D0A0041542B504F433D6D19
:10107000656D6265726E756D2C25640D0A00000049
:1010800041542B504F433D3345303030300D0A0032
:1010900098000020737574506F6353746174757396
:1010A0002E4C6973745570646174653D3D25642CE4
:1010B0004C6973744375724F6E6C696E654E756DD5
:1010C0003D3D25640D0A0000709001086F76657241
:1010D0003A25640041542B504F433D67726F757041
:1010E000732C25642B312C350D0A000041542B50F4
:1010F0004F433D314430303030253034783030305B
:10110000350D0A0041542B504F433D6D656D6265AE
:1011100072732C25642C25642B312C350D0A0000AC
:1011200041542B504F433D31453030303025303421
:1011300078303030350D0A0010B5012204A10020AE
:1011400000F00CF801210846FBF72AF810BD00005A
:10115000536C656570696E67000000002DE9F04111
:1011600005460E461746012D01D1BDE8F0810C4819
:10117000007800B1F9E73046F3F744F80446B4F5D7
:10118000807F01DD4FF480742146304602F0D6FBAB
:101190001FB1022103A002F0D1FB00BFE5E7000070
:1011A0002C0000200D0A0000F0B589B005460F465E
:1011B0001646022D01DB09B0F0BD05EB850000EB02
:1011C000451112480C18607800B9F4E7A078D0B146
:1011D0003946601DF3F71DF818B9B4F80300B042A2
:1011E00011D014223946601DF3F700F8A4F803600B
:1011F0006B1C07A21E2101A803F030F901A8FAF721
:10120000F9FA0020A07000BFD5E7000033210020CC
:1012100041542B544350434C4F53453D25640D0AD4
:101220000000000070B594B00426324890F83400F5
:1012300008B914B070BD2F483430F2F7E3FF05460B
:101240002846E91705EB5171C910A5EBC101C1F1A1
:1012500008010D44274890F8840000283ED102265A
:10126000002431E023483430A11C405C0DF8040018
:1012700020483430E11C415C601C0DF800101D4812
:101280003430015DA01C0DF800101A483430611C88
:10129000415CE01C0DF800101DF8041016A003F0CE
:1012A000CDF8601C1DF8001013A003F0C7F8A01CB7
:1012B0001DF8001010A003F0C1F8E01C1DF800108C
:1012C0000DA003F0BBF8241DAC42CBDB0021681E4F
:1012D0000DF8001009A003F0B1F805E0054890F8FA
:1012E0008400012800D1032669463046F9F758F8F2
:1012F00000BF9EE7DE1B0020256300000D0A0000F2
:1013000010B5044614B100F011F801E000F002F845
:1013100010BD00000348007818B94FF4004002499E
:1013200008607047D40200201408014030B510480E
:1013300090F86F0200B130BD0425002410E04FF496
:1013400000400C4908600720FDF752F94FF40040B7
:101350000849091D08600720FDF74AF9601CC4B25E
:10136000AC42ECDB4FF400400249086000BFE2E70A
:101370005C0800201008014008B501211C20FCF782
:1013800093FC4FF40040ADF8000010208DF80300EE
:1013900003208DF8020069460348F5F79FF8002006
:1013A000FFF7AEFF08BD000000080140F8B5064693
:1013B0000D463046F2F726FF00F0010000B1F8BDFF
:1013C00040E0002429E016F8010B0DF804001DF898
:1013D000040030280ADB1DF80400392806DC1DF85B
:1013E00004003038C0B20DF8040014E01DF8040009
:1013F00041280ADB1DF80400462806DC1DF804001D
:101400003738C0B20DF8040005E01DF80400573865
:10141000C0B20DF80400601CC4B2022CD3DB9DF8EE
:1014200000000007000E8DF800009DF8000000F09D
:10143000F0008DF800009DF800009DF801100843B1
:1014400005F8010B30780028BBD1287000BFB6E743
:101450002DE9F0470646884614464046F2F7D2FE8C
:1014600081460021601E3154621E41463046F2F72B
:10147000BDFE601E48451CDC052C1ADD2E21A01E79
:101480003154E01E31543546002707E028789F2864
:1014900002DDAD1CBF1C01E06D1C7F1C201FB8428B
:1014A000F4DCB84205D128789F2802DD2E21201FC8
:1014B0003154BDE8F0872DE9FC47044689461546BE
:1014C00000272846F2F79EFE8046B8F1040F02DAA4
:1014D0000020BDE8FC8749462046F2F75EFE2AE080
:1014E00028788DF8000068788DF80100A8788DF8CC
:1014F0000200E8788DF8030000208DF80400102227
:1015000000216846F2F7B8FE1FFA80FA504602F052
:10151000A7FC0646301220B904F8016B781C87B28C
:1015200006E0301204F8010B04F8016BB81C87B216
:101530002D1DA8F10408781C484502DAB8F1000F07
:10154000CEDC002004F8010B3846C2E710B50D4888
:101550000078B0B10C480078401CC0B20A4908704D
:1015600005280EDB09480078012803D108A26B2169
:10157000FFF706F8002003490870012206A1FFF7D3
:10158000EDFD10BDDC020020DD020020460300203E
:10159000B2CBB5A5000000005175697447726F7534
:1015A0007053656C0000000010B511480078E8B178
:1015B00010480078401CC0B20E490870022815DBA4
:1015C0000D480078012811D17E235A226E211D205A
:1015D000F6F75CFB0020FAF7A7FA00200449087030
:1015E00006490870012206A1FFF7B8FD10BD0000F2
:1015F000DF020020E002002046030020E10200207C
:1016000051756974566F69636553656C000000001D
:1016100010B506F021FB05F08BFE06F025FB10BD92
:1016200010B51248006840F00100104908600846F3
:1016300040680F4908400D494860084600680D4958
:1016400008400A4908600846006820F480200860C5
:101650000846406820F4FE0048604FF41F00886090
:10166000FEF736FC04480549086010BD0010024032
:101670000000FFF8FFFFF6FE0040000808ED00E064
:1016800010B500BF0121880700F080F80128F9D1CA
:101690000121800700F05CF81248007800B910BD05
:1016A0001148407800B9FAE710480078401C0F490B
:1016B00008700F480079097888420BDA4FF480509F
:1016C0000C49086009480078052808D1002007491E
:1016D000087004E04FF480500649091D086000BFFF
:1016E000DDE700000E0400205C080020420300201B
:1016F000DE1B0020100801401FB501210846FCF741
:10170000C3FA1C208DF8000000208DF801008DF830
:10171000020001208DF803006846FAF767FB63209A
:10172000ADF80800ADF804000020ADF80A00ADF8EF
:10173000060001A94FF0804000F078F801218807E9
:1017400000F009F801221146900700F028F81FBDAB
:10175000CA430282704721B1028842F0010202802E
:1017600004E002884FF6FE731A400280704731B1E0
:10177000B0F8442042F40042A0F8442005E0B0F85C
:101780004420C2F30E02A0F8442070470246002015
:10179000138A0B400BB1012000E0002070471AB102
:1017A00083890B43838102E083898B438381704764
:1017B00070B5002200230024058C4EF6FF763540DC
:1017C0000584038C8488828B48F6FF752A404FF687
:1017D000FF452A400D884FF6FF7606EA05252A4385
:1017E0004DF6FF752B400D8906EA05352B434D88D4
:1017F00006EA05352B430B4DA84202D00A4DA842FC
:1018000008D14BF6FF752C408D894FF6FF7606EA1E
:1018100085152C4384808283CD88A0F840500384B2
:1018200070BD0000002C01400034014000220288FD
:101830001D4B98420ED01D4B98420BD0B0F1804FFB
:1018400008D01B4B984205D01A4B984202D01A4B35
:10185000984204D14FF68F731A404B881A43174BA6
:10186000984207D0164B984204D04FF6FF431A40D7
:10187000CB881A4302808B8883850B8803850A4BAB
:1018800098420BD0094B984208D00E4B984205D095
:101890000D4B984202D00D4B984201D10B7A038632
:1018A0000123838270470000002C01400034014076
:1018B0000004004000080040000C00400010004000
:1018C0000014004000400140004401400048014035
:1018D00010B502460B465078012103E04C1C145D04
:1018E0006040491C5C1E8C42F8DC10BD10B57021B4
:1018F0000648F2F752FC064890F8F802054A32F81A
:10190000101005A002F09AFD10BD0000281F002055
:10191000DE1B00204A7D010847707374696D653DC8
:1019200025640D0A000000002DE9F04F8DB0064639
:101930008B4691469A46DDF858803546002008903F
:101940000024012007900020069008F1060080B2D4
:10195000029008F10C0080B201905B4634A20C2189
:1019600003A802F07BFD7E222046641C2A544FEA25
:1019700019222046641C2A542046641C05F8009055
:1019800000208DF82C00CDF830809DF82C202046CA
:10199000641C2A540C98C2B22046641C2A540022AB
:1019A0002046641C2A5400270BE003A8C15D03AA4B
:1019B000781C105C61F31F10C2B22046641C2A54CC
:1019C000BF1C0A2FF1DB1C480088020A2046641C59
:1019D0002A54194802782046641C2A541648008864
:1019E000401C15490880BAF1000F09D0002705E016
:1019F0001AF807202046641C2A547F1C4745F7DB51
:101A000021462846FFF764FF09902146641C099887
:101A10006854611E681C03F009FF0446641C7E22A2
:101A20002046641C2A5420460DB0BDE8F08F00000B
:101A300025303130750000004802002010B5044602
:101A40003448C07AA0753348017BE175417B21762B
:101A5000817B6176C17BA176017CE17600202060EC
:101A60006060606840F080706060606840F00070A6
:101A70006060284890F86C00532803D1606840F0FB
:101A800080606060234890F86D00572803D160683B
:101A900040F000606060606840F0805060601D4809
:101AA000808FC0F307201B4991F83C1040EA0120C9
:101AB00020821848808BC0F307201649097F40EA2E
:101AC000012060821348008CA0820120F4F7F6FF09
:101AD0001048806E000E20720E48806E010C6172FC
:101AE0000C48B0F86800010AA1720A4890F8681022
:101AF000E172406E000E20730648406E010C617367
:101B00000448B0F86400010AA173024890F8641018
:101B1000E17310BD281F0020F0B505460C4628686B
:101B20006968AA68EB6801EA020623EA01073E43F6
:101B300027683E44FE4F3E443044C60146EA5060AA
:101B4000084400EA010622EA00073E4367683E4473
:101B5000F84F3E4433441E0346EA1353034403EA5A
:101B6000000621EA03073E43A7683E44F24F3E4485
:101B70003244560446EAD2321A4402EA030620EA04
:101B800002073E43E7683E44EC4F3E4431448E0535
:101B900046EA9121114401EA020623EA01073E4385
:101BA00027693E44E64F3E443044C60146EA506051
:101BB000084400EA010622EA00073E4367693E4402
:101BC000E04F3E4433441E0346EA1353034403EA02
:101BD000000621EA03073E43A7693E44DA4F3E442C
:101BE0003244560446EAD2321A4402EA030620EA94
:101BF00002073E43E7693E44D44F3E4431448E05DC
:101C000046EA9121114401EA020623EA01073E4314
:101C1000276A3E44CE4F3E443044C60146EA5060F7
:101C2000084400EA010622EA00073E43676A3E4490
:101C3000C84F3E4433441E0346EA1353034403EAA9
:101C4000000621EA03073E43A76A3E44A6F5244660
:101C50004F3E3244560446EAD2321A4402EA0306A0
:101C600020EA02073E43E76A3E44BB4F3E4431440C
:101C70008E0546EA9121114401EA020623EA010792
:101C80003E43276B3E44B54F3E443044C60146EACE
:101C90005060084400EA010622EA00073E43676BF1
:101CA0003E44AF4F3E4433441E0346EA13530344BD
:101CB00003EA000621EA03073E43A76B3E44A94F0F
:101CC0003E443244560446EAD2321A4402EA03063B
:101CD00020EA02073E43E76B3E44A34F3E443144B3
:101CE0008E0546EA9121114401EA030622EA030720
:101CF0003E4367683E449D4F3E443044460146EAB9
:101D0000D060084400EA020621EA02073E43A769C0
:101D10003E44974F3E4433445E0246EAD353034465
:101D200003EA010620EA01073E43E76A3E44914F79
:101D30003E443244960346EA92421A4402EA0006BE
:101D400023EA00073E4327683E448B4F3E4431441C
:101D50000E0546EA1131114401EA030622EA03079F
:101D60003E4367693E44854F3E443044460146EA5F
:101D7000D060084400EA020621EA02073E43A76A4F
:101D80003E447F4F3E4433445E0246EAD35303440D
:101D900003EA010620EA01073E43E76B3E44794F20
:101DA0003E443244960346EA92421A4402EA00064E
:101DB00023EA00073E4327693E44734F3E443144C3
:101DC0000E0546EA1131114401EA030622EA03072F
:101DD0003E43676A3E446D4F3E443044460146EA06
:101DE000D060084400EA020621EA02073E43A76BDE
:101DF0003E44674F3E4433445E0246EAD3530344B5
:101E000003EA010620EA01073E43E7683E44614FCA
:101E10003E443244960346EA92421A4402EA0006DD
:101E200023EA00073E43276A3E445B4F3E44314469
:101E30000E0546EA1131114401EA030622EA0307BE
:101E40003E43676B3E44554F3E443044460146EAAC
:101E5000D060084400EA020621EA02073E43A76870
:101E60003E444F4F3E4433445E0246EAD35303445C
:101E700003EA010620EA01073E43E7693E44494F71
:101E80003E443244960346EA92421A4402EA00066D
:101E900023EA00073E43276B3E44434F3E44314410
:101EA0000E0546EA1131114481EA02065E40676977
:101EB0003E443E4F3E443044060146EA107008441A
:101EC00080EA01065640276A3E44394F3E44334477
:101ED000DE0246EA5353034483EA00064E40E76AB3
:101EE0003E44344F3E443244160446EA12421A44F9
:101EF00082EA03064640A76B3E442F4F3E443144DE
:101F0000CE0546EA5121114481EA02065E40676827
:101F10003E442A4F3E443044060146EA10700844CD
:101F200080EA0106564027693E44254F3E4449E079
:101F300078A46AD756B7C7E8DB702024EECEBDC1BF
:101F4000AF0F7CF52AC68747134630A8019546FD9A
:101F5000D8988069AFF7448BBED75C892211906B0B
:101F6000937198FD8E4379A62108B44962251EF627
:101F700040B340C0515A5E26AAC7B6E95D102FD6BD
:101F80005314440281E6A1D8C8FBD3E7E6CDE12192
:101F9000D60737C3870DD5F4ED145A4505E9E3A9F3
:101FA000F8A3EFFCD9026F678A4C2A8D4239FAFFF9
:101FB00081F6718722619D6D0C38E5FD44EABEA46F
:101FC000A9CFDE4B3344DE0246EA5353034483EA8F
:101FD00000064E40E7693E449F4F3E44324416049B
:101FE00046EA12421A4482EA03064640A76A3E4481
:101FF0009A4F3E443144CE0546EA5121114481EACC
:1020000002065E40676B3E44954F3E4430440601F5
:1020100046EA1070084480EA0106564027683E44AC
:10202000904F3E443344DE0246EA5353034483EA6E
:1020300000064E40E7683E448B4F3E44324416044F
:1020400046EA12421A4482EA03064640A7693E4421
:10205000864F3E443144CE0546EA5121114481EA7F
:1020600002065E40676A3E44814F3E4430440601AA
:1020700046EA1070084480EA01065640276B3E4449
:102080007C4F3E443344DE0246EA5353034483EA22
:1020900000064E40E76B3E44774F3E443244160400
:1020A00046EA12421A4482EA03064640A7683E44C2
:1020B000724F3E443144CE0546EA5121114461EA53
:1020C0000306564027683E446D4F3E443044860127
:1020D00046EA9060084460EA02064E40E7693E44E2
:1020E000684F3E4433449E0246EA9353034463EAF6
:1020F00001064640A76B3E44634F3E443244D6033C
:1021000046EA52421A4462EA00065E4067693E446B
:102110005E4F3E4431444E0546EAD121114461EA06
:1021200003065640276B3E44594F3E4430448601D7
:1021300046EA9060084460EA02064E40E7683E4482
:10214000544F3E4433449E0246EA9353034463EAA9
:1021500001064640A76A3E444F4F3E443244D603F0
:1021600046EA52421A4462EA00065E4067683E440C
:102170004A4F3E4431444E0546EAD121114461EABA
:1021800003065640276A3E44454F3E44304486018C
:1021900046EA9060084460EA02064E40E76B3E441F
:1021A000404F3E4433449E0246EA9353034463EA5D
:1021B00001064640A7693E443B4F3E443244D603A5
:1021C00046EA52421A4462EA00065E40676B3E44A9
:1021D000364F3E4431444E0546EAD121114461EA6E
:1021E0000306564027693E44314F3E443044860141
:1021F00046EA9060084460EA02064E40E76A3E44C0
:102200002C4F3E4433449E0246EA9353034463EA10
:1022100001064640A7683E44274F3E443244D60359
:1022200046EA52421A4462EA00065E40676A3E4449
:10223000224F3E4431444E0546EAD12111442E68D6
:1022400006442E606E680E446E60AE681644AE6042
:10225000EE681E44EE60F0BD604BBBF670BCBFBEC6
:10226000C67E9B28FA27A1EA8530EFD4051D880495
:1022700039D0D4D9E599DBE6F87CA21F6556ACC409
:10228000442229F497FF2A43A72394AB39A093FC57
:10229000C3595B6592CC0C8F7DF4EFFFD15D8485D3
:1022A0004F7EA86FE0E62CFE144301A3A111084E57
:1022B000827E53F735F23ABDBBD2D72A91D386EB53
:1022C0001CB540F225514B4801F0E4F900287ED0BE
:1022D000484801F09BFAC0B2019040F225514548B0
:1022E00001F0A7F944480078022805D19DF80410B0
:1022F000424801F090FA6AE03F480078012805D191
:102300009DF804103E4801F086FA60E03A480078F3
:1023100000285CD13B48008828B100203A49088059
:102320003A4908701CBD9DF804103748028800889F
:10233000401C354B18803548815435480078F8B139
:10234000344800780D2839D19DF804000A2835D189
:102350002E48007847280DD12C484078542809D1C0
:102360001846008827490880002028491A46128804
:10237000885423E0002024490880244908701DE087
:1023800022480078892814D11F480088032815DBCB
:102390001E488078C01C00901B4800880099884225
:1023A0000CD3194800881749088000201649088076
:1023B00004E000201449088014490870124800887D
:1023C000C72804DB0020104908800E4908809DF8CA
:1023D0000400104908700821064801F04EF9012850
:1023E00006D1044801F012FA0821024801F018F958
:1023F00000BF97E7003801402C0000200044004057
:1024000000480040300000202E000020340400204E
:10241000750200203E00002008B540F225512548F5
:1024200001F038F9B0B3234801F0F0F9C0B20090E0
:102430002148007802280AD19DF800101F4801F0B9
:10244000EAF940F225511B4801F0F3F808BD1C4899
:10245000008840F21E21884217DA9DF800001949D1
:10246000194A1288885418480088401C80B21649BE
:10247000088040F21E21884202DB002012490880B9
:102480000F480088401C0E49088040F22551094839
:1024900001F0CFF80821074801F0EFF8012806D134
:1024A000044801F0B3F90821024801F0B9F800BF6F
:1024B000CCE70000004400402C0000200038014020
:1024C00034000020FC0400203600002038B5002431
:1024D00040F22551374801F0DDF800285CD035483E
:1024E00001F094F9C0B2009033480078012805D17A
:1024F0009DF80010314801F08EF944E03048008822
:1025000000283DD19DF800002E492F4A128888549A
:1025100008460078242803D000202B49088004E0D6
:1025200029480088401C2849088027480088B0F5C1
:10253000957F02DD002024490880244800780D287A
:1025400021D19DF800000A281DD11E484078472857
:1025500012D11C48C07852280ED11A48407943281D
:102560000AD1002118480088401E164A1154164806
:1025700000881349088006E000201349088002E023
:1025800000201149088040F225510A4801F051F815
:102590009DF800000D4908700821064801F06DF80B
:1025A000012806D1034801F031F90821014801F062
:1025B00037F838BD004800402C00002000380140AA
:1025C0003C0000201A0700203A0000203F000020B5
:1025D00003498978024A517011468870704700009B
:1025E0004603002038B5054625B100203349087060
:1025F000334908803148007820B1012817D00228DB
:102600003AD11CE02F48007850B92FA0FEF704F90A
:102610003221324805F08EFB01202849087005E080
:10262000002001F013FC02202449087024E02B480C
:1026300005F068FB10B10120FFF7CAFF1CE003F0B2
:10264000B7F90446BCB1214625A001F0F7FEF5F725
:10265000C3FAFBF7B5FC01236E227F210020F5F7BA
:1026600073FB032015490870002001231FA272216B
:102670000090F5F7A3FD00BF00BF104800780328C5
:1026800000D038BD0E48008838B90020012317A2B9
:1026900072210090F5F792FD00E000BF0848008825
:1026A000401C80B206490880B0F5C87F01DB0020DD
:1026B000088001F0F7FC00BFE3E70000C70300203B
:1026C000CC0300205C0800202020C7EBCFC8B5C792
:1026D000C2BC2E2E2E20202000000000C8030020A7
:1026E00074656D703D3D3D25640D0A003CCDCBB356
:1026F000F62020C8B7B6A82020CFC2B7AD3E000054
:10270000F0B591B00646122546B1002094490870F4
:10271000F5F762FA012193A0FDF7AEFF022720240E
:10272000934800689349884201D0002E7DD0002054
:102730008F490860904908708948007818B1884826
:10274000007802283BD17F231A4621460020F5F766
:102750009DFA8A48D0F81D3089A2322101A801F0E3
:102760007DFE0020012301AA214600903846F5F79E
:1027700025FD601984B28148B0F82F3082A2322141
:1027800001A801F06BFE0020012301AA2146009060
:102790003846F5F713FD601984B200237EA232217A
:1027A00001A801F05BFE0020012301AA2146009050
:1027B0003846F5F703FD012069490870CDE0684807
:1027C00000780128FAD10020694908606A49087038
:1027D0007F231A462146F5F759FA724800780228F5
:1027E00005D171A2322101A801F038FE11E06D4837
:1027F000007828B96FA2322101A801F02FFE08E06D
:1028000068480078012804D16DA2322101A801F0A6
:1028100025FE0020012301AA214600903846F5F745
:10282000CDFC601984B2694B00E039E068A2322126
:1028300001A801F013FE0020012301AA2146009007
:102840003846F5F7BBFC601984B200208DF83800DB
:10285000302362A23221009001A801F0FFFD002088
:10286000012301AA214600903846F5F7A7FC60191C
:1028700084B23222002101A8F1F788FC5C4B5DA2F2
:10288000322101A801F0EAFD0020012301AA21461E
:1028900000903846F5F792FC0220314908705CE060
:1028A000334800685549884257D1002030490860B4
:1028B0002B480078012803D02948007802284CD101
:1028C0007F231A4621460020F5F7E0F90020012376
:1028D0004BA2214600903846F5F770FC601984B28F
:1028E0004A4B4BA2322101A801F0B8FD0020012380
:1028F00001AA214600903846F5F760FC601984B2C1
:102900000020012343A2214600903846F5F756FCEB
:10291000601984B2424B3EA2322101A801F09EFD13
:102920000020012301AA214600903846F5F746FC15
:10293000601984B23B48B0F82D333BA2322101A884
:1029400001F08CFD0020012301AA214600903846A9
:10295000F5F734FC00200249087011B0F0BD00000A
:10296000A0010020D6D5B6CBD0C5CFA20000000074
:10297000400000202A04BC00E20200209C1B002032
:1029800050534E3A256C7500D3A6D3C3B0E6B1BE02
:102990003A56256400000000C4DAB2BFB0E6B1BE0A
:1029A0003A2564009C000020C6BDCCA83ACEB4D61F
:1029B000AA000000C6BDCCA83A484753000000005A
:1029C000C6BDCCA83A424E44000000004808002092
:1029D000506F635665723A25730000004D4355D61B
:1029E000F7C6B53A25642E2564204D687A000000AC
:1029F0008A100020C4A3BFE93A2573002A04AC0062
:102A0000BDBBBBBBB7FECEF1C6F73A0070240020B9
:102A100025730000B6A8CEBBB7FECEF1C6F73A00CC
:102A200098240020DE1B0020504F52543A256400A9
:102A300038B50446002C25D0F5F7CEF80020012348
:102A400011A20D210090F5F7B9FB1248408801282A
:102A500007DB1048418800230F4A1048F6F778FF3B
:102A600003E000210846F6F7A3FF002001230CA293
:102A700072210090F5F7A2FB01236E229F21002016
:102A8000F5F762F938BD00002020CEC4B1BECFFBFF
:102A9000CFA20000A8210020FC010020C0240020BB
:102AA0005B50315DB2E9D4C420202020205B50323D
:102AB0005DD1A1CFEE00000070B586B005460426BA
:102AC000002D41D0F5F788F8DC48007830B10128B6
:102AD00009D002280CD0032814D10EE00D21D8A073
:102AE000FDF7CAFD0EE00D21D8A0FDF7C5FD09E0F8
:102AF0000D21D9A0FDF7C0FD04E00D21D9A0FDF7FF
:102B0000BBFD00BF00BFDC4890F8600240B2DB496B
:102B100008700846007830B90E231E226E2164200A
:102B2000F5F770F807E000200123D5A26E21009090
:102B30006420F5F743FB4FF0FF30D34908600020D5
:102B4000D249086006B070BDCB4890F86002CB490E
:102B500091F90010884217D0C74890F8600240B23F
:102B6000C64908700846007830B90E231E226E212F
:102B70006420F5F747F807E000200123C0A26E218A
:102B800000906420F5F71AFBC1480078012805D1B0
:102B9000C0A0FDF741FE322005F0BFF8B64800782E
:102BA00008B9002415E0B448C07838B9B248407973
:102BB00020B901240020BA4908600AE0AE484079F3
:102BC000002801DD022404E0AB48C078002800DDC5
:102BD000032434B1012C17D0022C3AD0032C6AD133
:102BE00052E0A9480068844202D1A948007850B157
:102BF0006C2380221B210020F5F748F8A9A22C2184
:102C00000020F5F77AFA56E09F480068844202D126
:102C10009F480078E0B122237F221B210020F5F796
:102C200035F863237F224B210020F5F72FF8A0A26F
:102C300053210020F5F761FA002010239FA25321B1
:102C400000901846F5F7BAFA01208B4981F8610225
:102C500031E08D480068844202D18D48007828B167
:102C60005F237F224B210020F5F710F895A2532116
:102C70000020F5F742FA0020102395A2532100907E
:102C80001846F5F79BFA16E07F480068844202D1A7
:102C90007F48007850B191A253210020F5F72DFA1A
:102CA00067237F2253211020F4F7F0FF53211020D7
:102CB000FDF784FC00BF00BF002C19DD72480068DE
:102CC000844206D07048006830B16F480068401CEC
:102CD00010B16F48007828B1012223210020FDF7B0
:102CE000E1FC92E0002223211046FDF7DBFC8CE0A2
:102CF0002022142101A8F1F749FA09227BA101A899
:102D0000F1F732FA6148006838B90020012301AABE
:102D10001B210090F5F752FA1EE05C480068642819
:102D20000AD12E208DF80D000020012301AA1B21BD
:102D30000090F5F743FA0FE054480068C8280BD11B
:102D40002E208DF80D008DF80E000020012301AA21
:102D50001B210090F5F732FA474890F86302664964
:102D60000978884203D148480068401C78BB424833
:102D700090F86302012805D160A2142101A801F096
:102D80006DFB36E03C4890F86302022805D15FA253
:102D9000142101A801F062FB2BE0374890F8630290
:102DA000042805D15DA2142101A801F057FB20E001
:102DB000314890F8630205280AD14F48007801286D
:102DC00006D05AA2142101A801F048FB11E01CE032
:102DD000294890F86302062805D157A2142101A8BA
:102DE00001F03CFB05E0244890F86302424908707A
:102DF0000FE0214890F863023F490870002001234A
:102E000001AA2B210090F5F7D9F90020204908707C
:102E100000BF1E480068401C1C490860B0F5967F42
:102E200001DB0020086018480068844204D016487E
:102E3000046000201549086000BF83E6FD02002001
:102E4000D6D0B9FAB5E7D0C500000000D6D0B9FA9F
:102E5000D2C6B6AF00000000D6D0B9FAC1AACDA83C
:102E600000000000B9ABCDF8BCAFC8BAB6D4BDB253
:102E7000CFB5CDB3000000005C0800208503002022
:102E8000B9D2B6CF000000007C03002080030020F0
:102E9000E5020020C7EBCFC8BDE2CBF8A3A100003C
:102EA0005C0300206C6F676F2E626D700000000085
:102EB00050686F6E652E626D70000000BFD5CFD078
:102EC000000000004373656E642E626D70000000A8
:102ED000B1BEBBFAD4DABDB2BBB0000043726563C9
:102EE000656976652E626D7000000000D5FDD4DA4C
:102EF000B5C7C2BD2E00000084030020D5CBBAC5E3
:102F0000D0C5CFA2B4EDCEF300000000CEDECDF8E8
:102F1000C2E7C1ACBDD3202000000000C7EBB2E582
:102F2000BFA820202020202000000000CEDEB7A86F
:102F3000C1ACBDD300000000C3BBD3D0B7FECEF1FF
:102F40000000000010B504461CB102490248FBF71E
:102F5000D5F910BDEC030020B8000020F8B50646F6
:102F6000002500BF2846691CCDB21E4951F820003B
:102F700000780028F6D1681EC5B2002E30D0F4F7D4
:102F80002BFE0D2118A0FDF777FB1A480078A8B199
:102F9000002407E0134850F82400174941F82400A2
:102FA000601CC4B2042CF5DB0E4850F82500124911
:102FB00041F824001148F7F71DFA03E009490F48CA
:102FC000F7F718FA002001230DA272210090F5F7FF
:102FD000F5F801236E227F210020F4F7B5FEF8BD3D
:102FE00000BFFCE788030020CFB5CDB3C9E8D6C346
:102FF000000000009C0000201C260020B8000020DB
:103000003CCDCBB3F62020C8B7B6A82020CFC2B79E
:10301000AD3E0000F8B50646002E56D0F4F7DCFDB4
:1030200002212BA0FDF728FB01236E229F21002007
:10303000F4F78AFE0020012328A272210090F5F700
:10304000BDF82B4890F89C502A48007818B1022D02
:1030500001DBA81EC5B2002409E0AC4203D1012067
:103060002549085502E0002023490855641C042C1A
:10307000F3DD2048007840B91F48204B002220494A
:1030800000902048F6F70AFC1EE0002406E01C48E9
:1030900050F824001C4941F82400641C022CF6DB83
:1030A000174802692046641C174941F8202014483B
:1030B00042692046641C41F820200F480F4B002233
:1030C00000901048F6F7EAFBF8BD00BFFCE70000EF
:1030D000B7FECEF1C6F7C1D0B1ED00005B4558494F
:1030E000545DCDCBB3F65B4D5DC8B7B6A80000000C
:1030F000DE1B00209C000020C8010020A40100204D
:10310000B0010020C0240020141F002038B5044660
:10311000DCB1F4F761FD01210CA0FDF7ADFA0EA3BF
:10312000382228210E48F8F7A3FE0D48F8F7F4FEE0
:103130000123682280210020F4F706FE00200123ED
:1031400008A272210090F5F739F838BDC3DCC2EB54
:10315000D1E9D6A40000000030303030303000001B
:10316000DA2300203CBCD3D6B52020C8B7B6A820AF
:1031700020CFC2B7AD3E000038B5044624B10020D0
:1031800030490870304908802E48007820B1012865
:1031900017D0022835D11CE02C48007850B92CA05B
:1031A000FDF73AFB32212F4804F0C4FD01202549E8
:1031B000087005E0002000F049FE02202149087057
:1031C0001FE0284804F09EFD10B10120FFF700FA2F
:1031D00017E002F0EDFB98B1F4F7FEFCFAF76EFE93
:1031E00001236E229F210020F4F7AEFD0020012371
:1031F0001DA272210090F4F7E1FF0320114908702D
:1032000000BF00BF0F480078032800D038BD0E482B
:10321000008838B90020012313A272210090F4F72E
:10322000CDFF00E000BF08480088401C80B206497E
:103230000880B0F5C87F01DB0020088000F032FF75
:1032400000BFE3E7E3030020E80300205C08002060
:103250002020C7EBCFC8B5C7C2BC2E2E2E20202001
:1032600000000000E40300203CCDCBB3F62020B5E5
:10327000A5BAF42020CFC2B7AD3E000000B5034888
:10328000002101600120FFF7A3F900BD46030020E3
:1032900010B588B002F0D8FC08B908B010BD6F486E
:1032A000007800B1F9E76E480078212872D2DFE893
:1032B00000F0D011407E7B81848791949A97D09DB5
:1032C000A0A3A6ACB2AFD0B5D0B8BBBEC1D0C4A984
:1032D000C7CACD00634800686349084458B1B0F5D7
:1032E000401F24D161480078012800D1D5E7022091
:1032F000FFF76EF91BE05D480078012800D1CCE7AC
:103300005B4890F86002012810D15A48007818B93B
:1033100059A0F8F76FFA09E055485BA21E21036C2B
:10332000684601F09BF86846F8F764FA00BF00BFF2
:1033300090E05B48FBF778F804464A480068594932
:10334000884228D15648407906281CD2DFE800F090
:1033500003070B0F13170420FFF73AF913E00320BC
:10336000FFF736F90FE01120FFF732F90BE01720D5
:10337000FFF72EF907E00620FFF72AF903E0072000
:10338000FFF726F900BF00BF454841794648FAF7E4
:1033900061FC08E05DE0334800684449884202D19E
:1033A0000120FFF715F955E0F4F74CFB52E000F06F
:1033B000A7FE4FE0F7F79EFB4CE0FCF73BFB49E034
:1033C000284800683949884203D125494878FFF7E1
:1033D000FFF83FE0F7F798FA3CE0F7F7F9FA39E041
:1033E000F7F746FA36E0F7F751F933E0FBF73CF927
:1033F00030E0FBF7F1F92DE0FBF728FC2AE0FBF7C2
:1034000089FE27E0FBF7A6FF24E0FCF7CFF921E0D7
:10341000F8F7E2FD1EE0F8F711FE1BE0FBF730FBCA
:1034200018E0FBF7FBFD15E0FCF748FB12E0FCF7AA
:1034300081FA0FE0FCF75CFE0CE0FCF7BDFD09E053
:10344000FBF77CFA06E0FCF78DF803E0FAF770FB77
:1034500000E000BF00BF00BF1FE70000DA0200204D
:103460004603002040000020D6FB43FFE40200207A
:103470005C0800209C00002041542B504F433D35F8
:1034800030303030300D0A0041542B504F433D65F1
:103490006E74657267726F75702C25640D0A00007A
:1034A000B80000202A04EC004A0300202A00FC0097
:1034B00010B500245248007851498978884202D1D9
:1034C0004F48C07838B14E4800784D49487008469A
:1034D00080780870012421460120FDF769FA4848E8
:1034E0000078212818D2DFE800F08811181C202469
:1034F000282C30343C403844484C5058605C886438
:1035000088686C70748878547C8084003D48F5F736
:1035100017F82046FFF7D0FA6FE02046FFF712FDBC
:103520006BE02046FFF728FE67E02046FFF75AF8D9
:1035300063E02046FFF77CFA5FE02046FFF70EFDD0
:103540005BE02046FFF7DCF857E02046F7F708FA83
:1035500053E02046F7F784FA4FE02046F1F7A0FE4B
:103560004BE02046F7F7B2F847E02046F7F79AF924
:1035700043E02046FBF7BEF83FE02046FBF774F936
:103580003BE02046FBF7CEFB37E02046FBF71CFE76
:1035900033E02046FBF70CFF2FE02046FCF754F900
:1035A0002BE02046FFF7B2FD27E02046FFF732FD73
:1035B00023E02046FBF7D6FA1FE02046FBF7D2FCBB
:1035C0001BE02046FCF7D6FA17E02046FCF7E2F9AC
:1035D00013E02046FCF7B6FD0FE02046FCF738FD6F
:1035E0000BE02046FBF7F2F907E02046FCF75AF81B
:1035F00003E02046FAF7CEFA00BF00BF10BD00007E
:10360000460300204A03002010B5FEF759FE10BD06
:1036100010B5FEF701FF10BD10B5FEF757FF10BD46
:1036200001F40072B2F5007F00D100BFCA430280EE
:10363000704710B50022002340F66A14A14200D161
:1036400000BF0A1201249440A3B2DC43048010BDE1
:1036500021B1828942F40052828104E082894DF6D0
:10366000FF731A40828170471AB1838A0B438382A9
:1036700002E0838A8B438382704702460020B1F5C3
:10368000007F00D100BF13880B400BB1012000E088
:103690000020704770B5024600240023002500205A
:1036A00040F66A16B14200D100BFC1F3421501F0E5
:1036B0001F03012606FA03F3012D02D19689334038
:1036C00006E0022D02D1168A334001E0968A33408B
:1036D0000C12012606FA04F41688344013B10CB11A
:1036E000012000E0002070BDF0B503460024002654
:1036F0000025002040F66A17B94200D100BF1846E5
:10370000C1F3421401F01F06012707FA06F5012C48
:1037100001D10C3004E0022C01D1103000E0143053
:103720001AB107682F43076002E00768AF430760DC
:10373000F0BD00002DE9F04786B005460E46002496
:10374000A24600BFA1460027B08900B100BF2F46A6
:103750002C8A4CF6FF700440F08804432C82AC891C
:103760004EF6F3100440B08831890843718908434C
:103770000443AC81AC8A4FF6FF400440B089044357
:10378000AC8201A8FAF7AAFA1F48874202D1DDF8F5
:1037900010A001E0DDF80CA0A88900F4004040B1C1
:1037A0000AEBCA0000EB0A1031684900B0FBF1F8DF
:1037B00007E00AEBCA0000EB0A1031688900B0FB91
:1037C000F1F86420B8FBF0F004012009642101FB4A
:1037D0001089A88900F4004040B1322000EBC900F4
:1037E000B0FBF1F000F00700044308E0322000EBEA
:1037F00009106421B0FBF1F000F00F0004432C81AC
:1038000006B0BDE8F0870000003801400146888816
:10381000C0F308007047C1F30802828070470000BF
:1038200000B585B0012144F20400FAF73DFA4FF4E7
:103830000070ADF8100018208DF8130003208DF8EB
:10384000120004A91C48F2F749FE4FF48060ADF85D
:10385000100004208DF8130003208DF8120004A935
:103860001548F2F73BFE4FF4E13000900020ADF830
:103870000400ADF80600ADF80800ADF80C000C200F
:10388000ADF80A0069460D48FFF754FF01210B48C7
:10389000FFF7DEFE40210948FFF7C2FE002240F29A
:1038A00027710648FFF720FF002240F22551034808
:1038B000FFF71AFF05B000BD0008014000380140C5
:1038C0001FB504464FF4E13000900020ADF804002D
:1038D000ADF80600ADF80800ADF80C000820ADF812
:1038E0000A00A4B1BDF80A0040F00400ADF80A00D7
:1038F00069461148FFF71EFF01210F48FFF7A8FE98
:10390000012240F225510C48FFF7EEFE13E0694614
:103910000948FFF70FFF01210748FFF799FE002232
:1039200040F224410448FFF7DFFE002240F2255117
:103930000148FFF7D9FE1FBD0038014070B50546AC
:103940000E4600240BE0295D0648FFF764FF00BF28
:1039500040210448FFF791FE0028F9D0641CB442CE
:10396000F1DB70BD0038014000B585B001210420B5
:10397000FAF79AF901214804FAF786F90820ADF818
:10398000100048208DF8130003208DF8120004A9C0
:103990002948F2F7A3FD0420ADF8100018208DF897
:1039A000130004A92448F2F799FD4FF4E130009088
:1039B0000020ADF80400ADF80600ADF80800ADF841
:1039C0000C000C20ADF80A0069461C48FFF7B2FE57
:1039D00040211A48FFF724FE002240F227711748C1
:1039E000FFF782FE012240F225511448FFF77CFECA
:1039F000002240F224411148FFF776FE01222821DF
:103A00000E48FFF771FE012260210C48FFF76CFEA3
:103A100001210A48FFF71CFE0020094908800949D6
:103A20000880094908800949088040F21E21084899
:103A3000F0F7B3FB05B000BD0008014000440040B2
:103A40003200002034000020360000203800002022
:103A5000FC0400202DE9F04788B0CC4800880828F5
:103A600002DA08B0BDE8F087C8480088B0F5077FE3
:103A700018DD002240F22551C548FFF735FE002031
:103A8000C4490880C1490880C3490880012240F226
:103A90002551BF48FFF728FE0122C0A11046FDF7BF
:103AA0005DFBDEE7B9480688042E00DAD9E7102E60
:103AB00001DA354600E01025B748078800240DE0FC
:103AC000BA48C05D03A90855781C80B2074640F289
:103AD0001E21884200DD0027601C84B2AC42EFDB6F
:103AE000B3A103A8F8F70CF800287DD0AA480788EE
:103AF00000240EE0AD48C05D0A2800D10BE0781C20
:103B000080B2074640F21E21884200DB0027601C7D
:103B100084B2B442EEDB00BFB44266DA601C85B208
:103B2000B5F5077F41DAA5480580002415E09F48D8
:103B300099490988415CA148801C01559648008834
:103B4000401C80B29449088040F21E21884202DB6A
:103B5000002091490880601C84B2AC42E7DB002160
:103B60009648801C0155002240F225518848FFF7F5
:103B7000BBFD86480088401B84490880012240F232
:103B800025518348FFF7B0FD8C480088401C8B49C5
:103B9000088008460188801CF8F7D2F820B101227D
:103BA00087A10020FDF7DAFA5BE78448058000244E
:103BB0001DE07E487849098810F80190B4F5077F28
:103BC00003DA7E48801C00F8049073480088401C8B
:103BD00080B27149088040F21E21884202DB002039
:103BE0006D490880601C01E025E023E084B2AC420E
:103BF000DFDB0021714880F81F12002240F22551BE
:103C00006348FFF771FD61480088401B5F490880E9
:103C1000012240F225515E48FFF766FD67480188A2
:103C2000801CF8F78DF820B1012269A10020FDF772
:103C300095FA16E715E7102E00DA12E756480788BE
:103C40004FF0000AD046002425E0584810F80790AD
:103C5000B9F12C0F08D1BAF1010F04DA0AF1010011
:103C600000F0FF0A0DE018E0BAF1010F09D1B8F138
:103C7000040F06DA4046411C1FFA81F801A901F839
:103C80000090781C80B2074640F21E21884200DB7B
:103C90000027601C84B2B442D7DB00BFB44200DB13
:103CA000DFE6002001A901F8080001A8F0F71CFBDD
:103CB00085B20A2D02DA4FF001080CE0642D02DA19
:103CC0004FF0020807E0B5F57A7F02DA4FF00308FB
:103CD00001E04FF0040805EB08000E3085B2AE425B
:103CE00000DABEE6B5F5077F41DA344805800024E6
:103CF00015E02E4828490988415C3048801C015550
:103D000025480088401C80B22349088040F21E21CB
:103D1000884202DB002020490880601C84B2AC424B
:103D2000E7DB00212548801C0155002240F2255187
:103D30001748FFF7D9FC15480088401B1349088035
:103D4000012240F225511248FFF7CEFC1B480088A3
:103D5000401C1A49088008460188801CF7F7F0FFCC
:103D600088B101221EA10020FDF7F8F90BE02346DF
:103D70001FA2142103A800F071FB012203A9104621
:103D8000FDF7ECF96DE600BF6BE6000034000020A3
:103D90000044004036000020380000205B5278329A
:103DA000427566204F7665725D000000FC040020BD
:103DB0002B54435052454356000000004A0C00204B
:103DC0004D51756575652046756C6C3100000000BD
:103DD0004D51756575652046756C6C3200000000AC
:103DE0004D51756575652046756C6C33000000009B
:103DF00041744D7367427566204F766572205B256E
:103E0000755D000070B505460E4600240BE0295D87
:103E10000648FFF700FD00BF40210448FFF72DFCD6
:103E20000028F9D0641CB442F1DB70BD00440040AE
:103E3000044948700021034A91701170024A1170C0
:103E400070470000530200205602002003494870CA
:103E50000021024A91700121117070475302002025
:103E6000F8B50446201220B9E0B27F2801DA2046D6
:103E7000F8BD002641F6F2771BE0F01900EBD07197
:103E80004D10A9006B4604220C480078FAF718F987
:103E9000BDF80000A04200DA6E1CBDF80000A04290
:103EA00000DD6F1EBDF80000A04202D1BDF8020087
:103EB000DEE7BE42E1DD3F20DAE70000A00000209F
:103EC0002DE9F0419AB00646274DDFF8A080746ACC
:103ED0006846F6F78DF91EE0B4F5806F10D94FF4FF
:103EE00080624146284603F01DFB4FF4806229465C
:103EF0006846F6F78FF908F58068A4F580640AE053
:103F0000A2B24146284603F00DFB224629466846E8
:103F1000F6F780F90024002CDED16846F6F700F9A8
:103F20002F4630224FF4FF11284603F0FBFA1022EF
:103F300016A907F11400F0F77AF958B1102216A962
:103F400007F11400F0F710F930224FF4FF11284662
:103F500003F05EFB102216A906F11400F0F704F935
:103F60001AB0BDE8F08100009C33002000F01F0073
:103F70002DE9F041DFF8C0C09CF800C04FEA8C008A
:103F8000DFF8B8C01CF80070E04600F1010C18F82A
:103F90000C6000F1020C18F80C50E910B210FB1084
:103FA0004FEAC12C0CEB421C9C441FFA8CF4DFF846
:103FB00090C0ACF80040DFF88CC09CF800C04FEA1D
:103FC0008C00C4461CF8007000F1010C18F80C605D
:103FD00000F1020C18F80C50E910B210FB104FEA77
:103FE000C12C0CEB421C9C441FFA8CF4DFF858C027
:103FF000ACF80040DFF854C09CF800C04FEA8C00D9
:10400000C4461CF8007000F1010C18F80C6000F1B7
:10401000020C18F80C50E910B210FB104FEAC12C3A
:104020000CEB421C9C441FFA8CF4DFF824C0ACF863
:104030000040BDE8F081000011040020FC260020B3
:104040001604002012040020180400201004002090
:10405000140400202DE9F84F0546AC000F4810F875
:1040600004900146601C11F80080A01C0F5C4FEA10
:10407000E70A4FEAA80B4FEAE90000904FEACA208E
:1040800000EB4B110098084486B23012F5F7E2FAC3
:10409000F0B2F5F7DFFABDE8F88F0000FC2600204B
:1040A00000BFFEE710B514480078012802D00228AE
:1040B00020D10FE001F07CFC58B1104800780428B2
:1040C00002D1F9F77DFF01E0F9F7F8FE00200A4977
:1040D00008700FE001F06CFC58B108480078042823
:1040E00002D1F9F76DFF01E0F9F7E8FE002002497F
:1040F000087000BF00BF10BD600300204603002011
:1041000010B58EB04B48007800283ED14A48C08890
:1041100058B94A4800684A49884206D10120FFF749
:1041200095FE01204349087011E04348C088401CB7
:104130004149898888420AD14048006841498842FB
:1041400005D10220FFF782FE02203A4908703A4862
:10415000F5F77AFC0446394800683B4988420DD19E
:1041600000203A4908703A48807918B10120FEF7DA
:104170002FFA5BE00220FEF72BFA57E03548844225
:1041800054D13548D0F8680200B950E00120FFF75B
:104190004FFE32480078012802D131A0F7F72AFB00
:1041A0002E48007801280FD12348C08800EB400139
:1041B00001EBC0012848A03050F821302FA2322155
:1041C00001A800F04BF90EE01B48C08800EB40014D
:1041D00001EBC0012048A03050F821302DA232213F
:1041E00001A800F03BF901A8F7F704FB012201A99F
:1041F0000020FCF7B3FF1048C08800EB400101EB42
:10420000C0011548A03000EB8100431D26A23221D9
:1042100001A800F023F9012201A90020FCF79EFF6C
:104220000120FEF7D5F900200249087000BF00BF49
:104230000EB010BD60030020C0240020400000200C
:104240002A04DC002A04BC002A00FC0053020020DF
:104250004A0300202A04EC005C0800209C00002097
:1042600041542B504F433D6175746F6C65617665A9
:1042700074696D652C33300D0A00000041542B50D9
:104280004F433D73696E676C6563616C6C2C25648C
:104290000D0A000041542B504F433D304130303027
:1042A00030253038780D0A00BAF4BDD03A257300B5
:1042B00010B586B000F036F810211848F2F7EDF985
:1042C0000020ADF804004FF48270ADF80600002025
:1042D000ADF808000220ADF80A000120ADF80C008E
:1042E0004002ADF80E000020ADF81000ADF812004D
:1042F0000720ADF8140001A90948FAF73FF9012198
:104300000748FAF721F94FF47A70F1F778F903F0DA
:1043100037F90446012006B010BD00000008014036
:104320000030014008B501210420F9F7BDFC01214E
:104330000803F9F7B9FC2020ADF8000003208DF840
:10434000020018208DF8030069460F48F2F7C6F8FE
:104350008020ADF8000069460B48F2F7BFF8402016
:10436000ADF8000004208DF8030069460648F2F716
:10437000B5F81020ADF800008DF80300694602483A
:10438000F2F7ACF808BD00000008014010B5024685
:104390000846012A05D1CB1DDC1703EB5474E0104D
:1043A00012E0042A04D14B1C03EBD37460100BE021
:1043B000102A01D1480007E0182A02D101EB410080
:1043C00002E0202A00D1880000E0401C00F0030336
:1043D000002BFAD110BD00002DE9F04705460E462E
:1043E0009046B5F1006F02D31348854201D3BDE872
:1043F000F087C5F3090000B1F9E7F1F717FD28468A
:10440000F1F7AAFC0746042F00D0F0E700240CE0E7
:10441000315D601C305C01EB00201FFA80F9281927
:104420004946F1F7E3FCA01C84B24445F0DBF1F708
:10443000D3FC00BFDBE70000000002080FB4054B0F
:1044400010B503A9044A029800F044F810BC5DF8C6
:1044500014FB00003D590108240400200FB41CB5D2
:104460000A46521ECDE9000207A9054B6A46069886
:1044700000F030F8009A002111701CBC5DF814FBAC
:10448000374901080FB4084B10B504A902AA0398D4
:1044900000F020F8044602A9002000F057FA204658
:1044A00010BC5DF814FB00004D490108004870473E
:1044B0003004002002E008C8121F08C1002AFAD107
:1044C00070477047002001E001C1121F002AFBD194
:1044D000704700002DE9FF4F8DB00F4605460026BE
:1044E00006E025280BD0DDE90F1290476D1C761CE5
:1044F00028780028F5D111B03046BDE8F08F0024AF
:10450000A246A1460122EC4900E0044315F8013F10
:10451000203B02FA03F00842F7D128782A2810D06D
:104520006FF02F022878A0F13001092914D80AEB86
:104530008A0102EB410144F0020400EB010A6D1C08
:10454000F0E701CF5FEA000A03D544F40054CAF152
:10455000000A44F002046D1C28782E2817D115F8A3
:10456000010F44F004042A280ED06FF02F0228789F
:10457000A0F1300109290AD809EB890102EB4101B8
:1045800000EB01096D1CF2E757F8049B6D1C2878BD
:104590006C280FD006DC4C2817D068280DD06A286C
:1045A00014D104E0742810D07A280FD10DE044F41F
:1045B00000140AE044F4801401E044F440146978E3
:1045C000814202D104F580146D1C6D1C2A786E2A7C
:1045D0001FD00CDC632A31D004DC002A8BD0582A8F
:1045E00011D1A3E0642A68D0692A0CD165E0732A4E
:1045F0002ED004DC6F2A73D0702A04D19BE0752A78
:104600006FD0782A6ED01046DDE90F129047761CE5
:1046100050E1C4F30250022806D0032809D0042830
:1046200001CF09D0066045E101CFF117C0E9006173
:1046300040E101CF06803DE106703BE117F8040B35
:104640008DF8000000208DF80100EB46012003E00A
:1046500057F804BB4FF0FF3061074FF0000102D460
:104660000DE008F10101884649450FDA8045F8DB85
:104670001BF808100029F4D108E008F10101884670
:104680008142FADB1BF808100029F6D1DDE90F237F
:10469000AAEB08008146214600F036F9304400EBD1
:1046A000080604E0DDE90F121BF8010B9047B8F192
:1046B0000108F7D221464846F7E00A21C4F3025325
:1046C0004FF0000B0891022B04D001CFC117032B30
:1046D00009D00AE0FF1D27F00707F7E8020108E00C
:1046E00032E01FE020E000B2C117042B01D140B23C
:1046F000C117031E71F1000307DA4FF0000CD0EB75
:104700000C006CEB01012D2302E0230504D52B23C3
:104710008DF82430012303E0E30701D02023F7E7DD
:10472000984658E00A2110E010210EE010204FF0CA
:10473000000B08900CE010214FF0000B44F0040433
:104740004FF00809089103E008214FF0000B089191
:10475000C4F30253022B04D001CF0021032B06D057
:1047600006E0FF1D27F00707F7E8020103E080B22B
:10477000042B00D1C0B24FF0000823072BD5702ABC
:1047800007D0DDF820C08CF0100C5CEA0B0C05D0D3
:104790000EE040238DF82430012308E050EA0103A5
:1047A00006D030238DF824308DF82520022398463A
:1047B000DDF820C08CF0080C5CEA0B0C0BD150EA41
:1047C000010301D1630706D530238DF824304FF063
:1047D0000108A9F10109582A04D038A20B9208AAAD
:1047E0000A920BE03AA2F9E75B46089AEFF748FF16
:1047F0000B9B9B5C0A9A521E0A92137050EA0102AC
:10480000F2D10A98ADEB000000F1200B600702D551
:1048100024F4803401E04FF00109D94502DDA9EB11
:104820000B0000E0002000EB0B0141440890AAEBD4
:10483000010AE00306D4DDE90F232146504600F0CB
:1048400063F806444FF0000908E009A911F80900CF
:10485000DDE90F12904709F10109761CC145F4DB2F
:10486000E0030CD5DDE90F232146504600F04CF85B
:10487000064404E0DDE90F1230209047761C0899C9
:10488000481E08900029F5DC08E00A980A9900788B
:10489000491C0A91DDE90F129047761CBBF100011B
:1048A000ABF1010BF1DC21465046DDE90F2300F0AE
:1048B00019F806446D1C1BE609280100303132331B
:1048C000343536373839616263646566000000004C
:1048D0003031323334353637383941424344454636
:1048E000000000002DE9F041044600251E46174651
:1048F000880404D405E039462020B0476D1C641EAE
:10490000F9D52846BDE8F0812DE9F041044600259F
:104910001E469046C80301D5302700E020278804B2
:1049200004D505E041463846B0476D1C641EF9D5F4
:104930002846BDE8F0814A68002A06D00A68531C60
:104940000B6010704868401E486070470A68531C2E
:104950000B601070704700002DE9F041AAB00025EF
:104960000027A846012119A8F2F78AFE0C2119A8F0
:1049700000F0FCFE064619A807C88DE807000020D5
:10498000039004900590069036A103A8EFF75CFC15
:1049900000210791089109910A9133A107A8EFF727
:1049A00053FC35221CA93248F9F7CAFBDDF88F0009
:1049B000B04202D12AB0BDE8F08146E03DB9B8F17D
:1049C000000F04D100221146302000F06BF8681C63
:1049D0000546032805D3B8F1000F01D1781CC7B2F2
:1049E0000025032F00DD31E0F3F77AFD4FF47A70F4
:1049F000F0F7F3FD1F48008800B926E01D48017854
:104A00001CAB32461C4800F0E5FD04462CB90C22D4
:104A100019A9352000F046F8CCE7042C05D10C226A
:104A200019A9372000F03EF80BE0052C02D14FF019
:104A3000010806E0062C04D12C226946342000F03F
:104A400031F800200B49088000BFB7E700BF07E03E
:104A5000F3F746FD6420F0F7C0FD08A0FFF7EEFC79
:104A6000F6E700005A5400005A5432363000000075
:104A700000FC01083000002034040020706C6561E7
:104A800073652074727920617574682D2D2D2D2D1C
:104A90002D2D2D2D2D2D2D2D2D2D2D2D2D2D0D0A89
:104AA000000000002DE9F04FA1B082468B4617466A
:104AB0000DF10706F81C00F0FF08002589222946A1
:104AC0006D1C01A8425429466D1C00F801A029461E
:104AD0006D1C00F801802B480088021229466D1CCD
:104AE00001A842542748027829466D1C01A8425467
:104AF000002408E01BF804202846691CCDB201A957
:104B00000A54601CC4B2BC42F4DB08F10300C0B21A
:104B10008DF800009DF804008DF801009DF8050057
:104B20008DF8020000240FE0032094FBF0F100FB5D
:104B300011401DF80000315D48403055305D80F077
:104B400086003055601CC4B2A8F10100A042EBDC25
:104B50004FF00009002405E001A8005D80EA090982
:104B6000601CC4B2AC42F7DB2846691CCDB201A977
:104B700001F80090294601A8FEF7E0FE21B0BDE84B
:104B8000F08F0000A002002030B59DB00446012245
:104B900015A10020FCF7E2FA1648B0F80300ADF8C2
:104BA00008001448B0F8010001909DF805008DF848
:104BB0000A009DF804008DF80B000E4840798DF82E
:104BC0000C00052000900C48D0F81D1002AB01220B
:104BD00004A8FCF7A9FE05462A4604A9204602F0CF
:104BE00095FF1DB030BD000062754269616F416381
:104BF0006B000000360200209C1B002030B595B0F1
:104C0000054601220DA10020FCF7A8FA072000901C
:104C10000D48D0F81D100D4B4FF4817201A8FCF720
:104C200083FE84B2224601A9284602F06FFF214686
:104C300001A8F8F7D1FF15B030BD000062754269D8
:104C4000616F4175746800009C1B0020D71E002016
:104C50002DE9F04F97B0044688466178A07861F35B
:104C60001F2082464FF0010B5346A4A232210AA80E
:104C7000FFF7F4FB01220AA90020FCF76FFAAAF65D
:104C8000027000287ED0A0F5E040FF3800287AD0DE
:104C9000FF2804D0A0F2FF20002875D156E0E67B63
:104CA000334699A232210AA8FFF7D8FB01220AA9AC
:104CB0000020FCF753FA052E33D2DFE806F0031A82
:104CC00020262C00072204F110019348EFF7AFFAD9
:104CD00048B1914821690160A18A8180A17D8171DB
:104CE0000020F6F721FF8DA20A2107A8FFF7B6FBE7
:104CF0001DE08BA20A2107A8FFF7B0FB17E08BA2EB
:104D0000012107A8FFF7AAFB11E08AA20A2107A840
:104D1000FFF7A4FB0BE08BA20A2107A8FFF79EFB7D
:104D200005E08BA20A2107A8FFF798FB00BF00BF90
:104D300007A8334688A2322100900AA8FFF78EFB0D
:104D400001220AA90020FCF709FACFE0E5784FF626
:104D5000FF7000EA052505F47F4520790543681EAC
:104D600085B2B5F5C87F01DB4FF4C87540F29111EB
:104D70007E48EFF712FA2A4604F10E017B48EFF75E
:104D8000F3F902E07AE01EE0ADE07848001FA0F8F9
:104D9000965148F203107649A1F80100E07A8DF8A7
:104DA0001800207B8DF81900BDF81800A1F8030049
:104DB000022048716D48001FB0F89601002801DDFF
:104DC000FAF750F892E00FFA88F7F81E215CB81E47
:104DD00014F8009061F31F29781E265C434665A2F3
:104DE00032210AA8CDE90096FFF738FB01220AA973
:104DF0000020FCF7B3F9B9F1020F31D0B9F5817F8A
:104E000007D0B9F5007F25D0A9F60170002833D16D
:104E10002CE076B96048007820F0100010305E4930
:104E200008705EA232210AA8FFF718FB00F086FC8A
:104E30000AE05948007820F01000574908705AA23B
:104E400032210AA8FFF70AFB01220AA90020FCF779
:104E500085F911E0012258A10020FCF77FF90BE051
:104E6000012259A10020FCF779F905E001225AA19D
:104E70000020FCF773F900BF00BF37E0012259A101
:104E80000020FCF76BF9607B8DF81800A07B8DF893
:104E90001900BDF81800ADF81000E07B8DF8120085
:104EA000207C8DF81300607C8DF81400A07C8DF8B8
:104EB0001500E07C8DF81600DDE90401F8F7E6FF47
:104EC0009DF816009DF815109DF81420CDE90021DD
:104ED00002909DF813309DF81220BDF8101044A0E8
:104EE000FFF7ACFA02E04FF0000B00BF00BF00205C
:104EF0004A49087017B0BDE8F08F00000D0A636DD5
:104F0000643D2530347800000D0A726573756C7449
:104F10003D25303278000000D71E00204F6B000086
:104F20004361722045786973740000004E6F2063FE
:104F30006172000044657669636520457869737421
:104F4000000000004E6F205265636F726400000025
:104F50004661696C650000000D0A5B526567697304
:104F60007465725D25642025730000009C1F00207D
:104F7000360200200D0A4C656E3D25642C61636B82
:104F8000436D643D253034782C726573756C743DC7
:104F90002530327800000000281F00200D0A5B41F8
:104FA00054485D4F6B0000000D0A5B4154485D465C
:104FB00061696C65000000000D0A4C6F63617469E3
:104FC0006F6E2041434B00000D0A486561725469C1
:104FD000636B2041434B00000D0A534F5320414364
:104FE0004B0000000D0A54696D6541636B000000C1
:104FF0000D0A4E657754696D653A253032642D256A
:105000003032642D2530326420253032643A253028
:1050100032643A253032640D0A0000003502002067
:1050200030B59BB0044601220AA10020FCF796F897
:10503000002000900A48D0F81D100023022202A888
:10504000FCF772FC85B22A4602A9204602F05EFDFA
:105050001BB030BD62754269616F48656172740052
:105060009C1B002030B59DB0044601220CA10020FD
:10507000FCF774F802A8FCF7E1FC1C2000900C4837
:10508000D0F81D1002AB4FF4007209A8FCF74CFCDD
:1050900085B22A4609A9204602F038FD1DB030BD70
:1050A00062754269616F4C6F636174696F6E000075
:1050B0009C1B002070B588B006460024614800782B
:1050C00040B100205F49087040F273525E4930469B
:1050D000FCF76AF8304602F095FC08B108B070BDE4
:1050E0005A480078C0F30010F8B94FF4FA705849E4
:1050F000088058480078401CC0B2564908701E28E5
:1051000012DB0020087054480078401CC0B252499D
:105110000870032805DB00200870304600F0DEF838
:1051200002E03046FFF76AFDD8E74C4800780628D1
:1051300012DD002049490870731C49A21E216846EF
:10514000FFF78CF96846F6F755FB4048007820F0E9
:1051500010003E490870C1E73C480078C0F34000A9
:1051600030B34448006818B3434890F8F802434904
:1051700031F810004FF6FF7101EA40054048008801
:10518000401C80B23E490880A84204DB0020088011
:1051900001203C4908703B48007848B100F064FDAC
:1051A00030B100203749087001243046FFF75AFF1C
:1051B00027480088401C80B225490880B0F5B47F9C
:1051C0000ADB4CB900F050FD30B1002020490880C6
:1051D0000124304600F004F92B48007800F001006B
:1051E00038B134B900202849087001243046FFF74F
:1051F000CBFC2648007838B134B900202349087028
:105200000124304600F0A8F821480088401C80B2F4
:105210001F490880782809DB44B900F025FD28B132
:1052200000201B4908803046FFF7FAFE3CB10B48CE
:105230000078401C0949087000201549088000BF0B
:105240004CE70000AC00002098240020281F00201C
:10525000400200203F0200203E02002035020020D4
:1052600041542B544350434C4F53453D25640D0A44
:1052700000000000B4000020DE1B00204A7D010871
:1052800044020020460200203602002034020020A2
:105290004202002070B504460D4620787E280DD1CC
:1052A000681E205C7E2809D1691E601C02F0ECF8A3
:1052B00086B231462046FFF7CBFC04E0012202A172
:1052C0000020FBF74BFF70BD4E6F7420427562618A
:1052D000696F2070726F746F6C00000030B5A7B0FA
:1052E0000446012218A10020FBF738FF302102A854
:1052F000EEF753FF1748D0F81D00000E8DF825007B
:105300001448D0F81D00010C02A881771148B0F8AC
:105310001D00010A02A8C1770E48417F8DF82810B0
:105320002E2000900B48D0F81D1002AB4FF4807275
:105330000EA8FCF7F9FA85B22A460EA9204602F01B
:10534000E5FB27B030BD000062754269616F5265B0
:10535000670000009C1B002030B58FB0044601227E
:105360000BA10020FBF7FAFE002000900B48D0F8BC
:105370001D10002340F6017202A8FCF7D5FA85B291
:105380002A4602A9204602F0C1FB0FB030BD000042
:1053900062754269616F536F530000009C1B0020CF
:1053A00010B50446012205A10020FBF7D7FE0848EE
:1053B000007820F010000649087010BD627542693F
:1053C000616F536F636B657420446F776E000000EC
:1053D000281F002010B504462046FFF76BFE10BDC5
:1053E00030B58FB0044601220BA10020FBF7B6FEBA
:1053F000002000900B48D0F81D10002340F60272E8
:1054000002A8FCF791FA85B22A4602A9204602F0CA
:105410007DFB0FB030BD000062754269616F546959
:105420006D6500009C1B0020F0B58BB005460C4656
:10543000AE1D34B9284B29A2282101A8FFF70EF888
:1054400005E0294B29A2282101A8FFF707F82846E3
:10545000EEF7D8FE09280ED327A12846F6F750FB11
:1054600048B101A92846EEF7D4FE20B126A128466E
:10547000F6F746FB08B90BB0F0BD9CB93046EEF725
:10548000C1FE871E3A4631461348EEF76DFE3046A0
:10549000EEF7B8FE801E104900220A541EA0FEF747
:1054A000CDFF16E03046EEF7ADFE871E3A46314698
:1054B0000D48EEF759FE3046EEF7A4FE801E0A496D
:1054C00000220A5419A0FEF7B9FF07491C48EEF75D
:1054D000BBFE00BFCFE70000702400202B475049DF
:1054E000503A25730D0A0000982400202B474749A5
:1054F000503A25730D0A00002B474749503A302E89
:10550000302E302E300000002B475049503A302EBC
:10551000302E302E30000000676574206E657720D5
:105520005049503D3D3D3D25730D0A00676574208F
:105530006E6577204749503D3D3D3D25730D0A007E
:105540003821002070B505460120F3F737FE002012
:1055500011490880012211A1FBF700FE13A0F6F704
:1055600049F915B1012D08D103E014A0FBF754F956
:1055700004E015A0FBF750F900E070BD00BF062461
:1055800006E0F2F7ADFF642002F0C7FB601E04B234
:10559000002CF6DA00BFF0E7B0000020547279204A
:1055A000746F205077724F6666000000415424519A
:1055B00043505752444E0D0A00000000D5FDD4DA86
:1055C000B9D8BBFA00000000B5CDD1B9B9D8BBFA43
:1055D000000000002DE9F84F04468846924699469F
:1055E0004FF0000BE51C2078892802D00120BDE88F
:1055F000F88FA078C01C404501D00220F7E70026B4
:1056000004E0A05D80EA0B0B701CC6B2A8F101009B
:10561000B042F6DC205C584501D00320E7E78DF866
:10562000008020788DF8010060788DF80200002657
:105630000FE0032096FBF0F100FB11601DF8000065
:10564000A95D4840A855A85D80F08600A855701C4B
:10565000C6B26078401EB042EBDC6078312801D1E0
:105660000520C4E76078322801D10620BFE76078C2
:10567000362801D00420BAE7AD1C2846F0F7E6FA38
:105680002F783F0227F0FF07687807433F0227F093
:10569000FF07A87807433F0227F0FF07E878074392
:1056A0002D1D287889F82300C9F81F7000260CE00A
:1056B00015F8010BA179484009F8060004EB080031
:1056C000A84200D82546701CC6B21F2EF0D3002673
:1056D0000DE015F8010B2179484009F124018855A6
:1056E00004EB0800A84200D82546701CC6B2112E53
:1056F000EFD3352249460748FEF76EFE524639463B
:1057000005A0FEF79BFE574501D100206FE704205E
:105710006DE7000000FC01086E657741757468490B
:105720006E666F3A253038782C74617267657463E1
:105730006F64653A253038780D0A000010B5C8212D
:10574000054802F0F7FA012004490870012204A17B
:105750000020FBF703FD10BD4C020020500200208A
:1057600053656E6420656E61626C65002DE9F043DF
:10577000D1B080460F464FF480722B4911A8EEF746
:10578000F3FC0026002408E018F80400464018F84E
:10579000040001A90855601CC4B2BC42F4DB7E4081
:1057A00011A810F8069000240CE001A8005D80EA22
:1057B000090684EA060001A9085511A810F8069008
:1057C000601CC4B2BC42F0DB002413E004EB4400D4
:1057D00001A9085C04EB4401491C01AA515C80EA60
:1057E000010604EB4400801C01A9085C70400855C8
:1057F000601CC4B2042CE9DB9DF804502D0225F096
:10580000FF059DF8050005432D0225F0FF059DF8D5
:10581000060005432D0225F0FF059DF8070005430E
:10582000284651B0BDE8F0832C9201082DE9F047DD
:1058300080460D46680000F0EFFD81464C4600278B
:1058400015B90020BDE8F08769004846EEF7A5FCD1
:1058500000261CE018F806007D2806D104F8010B8C
:10586000012004F8010BBF1C10E018F806007E2888
:1058700007D17D2004F8010B022004F8010BBF1CA6
:1058800004E018F8060004F8010B7F1C761CAE42F9
:10589000E0DB3A4649464046EEF766FC484600F0F3
:1058A0005FF83D462846CDE72DE9F04105460C4618
:1058B000002100200BE0175C15F8018087EA08073B
:1058C00017544F1C3946A74200DB0021401C984268
:1058D000F1DB0021002028E00F4601EBD7784FEAEA
:1058E0006808A1EB4808B8F1000F04D0114F7F5CA5
:1058F00007F00F0C03E00F4F7F5C4FEA171C0E4FB1
:1059000017F80C604F1C3946A74200DB0021074600
:1059100000EBD7784FEA6808A0EB4808B8F1000F11
:1059200002D0175C77401754401C9842D4DBBDE886
:10593000F0810000727D0108787D010870B5044691
:105940000D46E1B20548FDF766FF00BF4021034860
:10595000FDF793FE0028F9D0204670BD00380140C5
:1059600010B5002821D0114B0022001F196803E058
:10597000814203D80A4649680029F9D152B1136817
:10598000841A9C4204D1006818441060104602E05A
:10599000506000E0186039B102680B1A934203D1DD
:1059A0000B681A4402604968416010BD2804002059
:1059B000002004490878097811B10021014A1170CA
:1059C000704700005602002000200A4991F89C1000
:1059D00005290CD2DFE801F0030405070A0006E000
:1059E00005E0054803E00448283000E000BF00BFA0
:1059F00070470000DE1B00206B1D002010B5002446
:105A0000114890F89C0005280ED2DFE800F003064C
:105A100008090A000C4CC53406E00C4C04E003E015
:105A200002E00A4C503400BF00BF1CB900200849F6
:105A3000087003E021460648EEF706FC0120054900
:105A40000870204610BD0000DE1B0020F31C002063
:105A500098240020AC00002070B504462046EEF7E4
:105A6000D1FB851E2A4621460448EEF77DFB002225
:105A700021461046FBF772FB70BD00008A10002023
:105A800010B50024104890F89C00052810D2DFE8DB
:105A900000F00306090B0D000B4C9D3408E00A4C86
:105AA000ED3405E0094C03E0084C01E0084C00BF70
:105AB00000BF28210748EEF770FB21460548EEF7A6
:105AC000C3FB204610BD0000DE1B0020427D010804
:105AD0001B1D00207024002010B50446A07B302838
:105AE00004D10020074981F8640203E00120054940
:105AF00081F86402034890F8641203A0FEF79EFC4C
:105B000010BD00005C080020506F63436F64653A6D
:105B100025640D0A000000002DE9F0418CB0044618
:105B200088462046EEF76EFB07460026002524E057
:105B3000605D0D2815D1002002A988551422114856
:105B4000EEF754FB02AB10A2282102A80094FEF746
:105B500085FC002202A91046FBF700FB0CB0BDE853
:105B6000F081605D302807DB605D392804DC625D10
:105B70003046761C02A90A546D1CBD42D8DB00BF1A
:105B8000ECE7000048080020504F437665723A2544
:105B9000733C2D3E2573000070B5ADF5936D054641
:105BA000302229460DF58D6001F0BCFC2549DDF859
:105BB0009404884203D001200DF5936D70BDDDF88B
:105BC0008C04B0F5805F01D90220F5E705F5805619
:105BD000DDF88C440DF58060F4F70AFB20E0B4F5A5
:105BE000806F11D94FF480623146684601F09AFC0B
:105BF0004FF4806269460DF58060F4F70BFB06F503
